:020000040000FA
:1020000002A4C002D2578F27AFA775A70F8FA77F53
:10201000327E0012CA33E52724FF92B47FDC7E05AE
:1020200002CA3302CB86D286D2872202CE6D7D01D0
:102030007F8012A2F5901B9BE0FEA3E02400FFE44A
:102040003EFEC36480948050066307FF6306FF7CF6
:10205000007D021227FDE51D2FFFE51C3EFE7C00E2
:0A2060007D021227FD8E1C8F1D2249
:10206B0002CE4C7D1AAF16AE1512600B12CF4D126D
:10207B00CC617D18AF16AE1512600B900968740316
:10208B00F09009677409F02202C0B38F27AFA775D0
:10209B00A70F8FA77F327E0012CA33E52724FF924A
:1020AB00B57FC87E0002CA3302CEE3E590540C2301
:1020BB00C0E074CFC0E0C082C08302CF00E5905473
:1020CB000C23C0E074CFC0E0C082C08302CF08E510
:1020DB0090540C23C0E074CFC0E0C082C08302CF09
:1020EB0010E590540C23C0E074CFC0E0C082C083D5
:0A20FB0002CF18EFC40390CF00736A
:1021060002244EE86480F8E933E83360110460F095
:10211600ED33EC337009E8FCE9FDEAFEEBFF22043F
:1021260060DED3EB9FEA9EE99DE8C2E78CF0C2F73A
:1021360095F0400CE8CCF8E9CDF9EACEFAEBCFFB06
:1021460012241985D0F05804700320D5B3E8047022
:10215600075002B2D502245892D5EC0460F7E4CCBD
:10216600C0E0C398F8603B94186008400DD0E0FBCF
:10217600022430E4FBFAC9FC8028E830E406E4C90E
:10218600FBE4CAFCE830E305E4C9CACBFCE8540723
:102196006010F8C3E913F9EA13FAEB13FBEC13FC2E
:1021A600D8F130F52FC3E49CFCEF9BFFEE9AFEEDD1
:1021B60099FDD0E0FBEF4E4D4C701222DB0302245A
:1021C60055EC2CFCEF33FFEE33FEED33FDED30E73F
:1021D600EB022430EF2BFFEE3AFEED39FDD0E0FBAB
:1021E60050130BBB0003022458ED13FDEE13FEEF54
:1021F60013FFEC13FC022430EC4D6011E849701714
:10220600ED33EC3304600DE4FCFFFEFD22E933E818
:10221600330470F802244E12241958046009E4CCE1
:1022260024815006285009022458284003022455C8
:10223600C0E0EB4A7044B98006D0E0FB022444EFCC
:102246004E701CBD8008EBFFEAFEE9FD80EBE98DD0
:10225600F0A4FEE5F00222E7E9CDF9EAFEEBFFEF96
:1022660089F0A4FCE5F0CE89F0A42EFFE435F0CD8C
:1022760089F0A42DFEE435F08067EF4E7005BD8031
:10228600D780C3EF8BF0A4ACF0EE8BF0A42CFCE46B
:1022960035F0F8EF8AF0A42CE5F038FCE433CB8D6A
:1022A600F0A42CFCE5F03BF8EE8AF0A42CFCE5F05B
:1022B60038F8E433CF89F0A42CFCE5F038CF3400AD
:1022C600CE89F0A42FFFE5F03EFEE433C98DF0A4DD
:1022D6002EFEE5F039CD8AF0A42FFFE5F03EFEE4B0
:1022E6003DFD33D0E0FB50070BBB000F022458EC3A
:1022F6002CFCEF33FFEE33FEED33FD0224300224D7
:1023060058EC5D046005E85904700302244E12245B
:1023160019580460F6EC4860F2EC7004FDFEFF22EA
:10232600C860DB2481C85009C398600250060224A5
:10233600559850CAF582E9294B4A7005AB820224AA
:102346004475F0007C1A7880C3EF9BEE9AED9940B5
:102356000DC3EF9BFFEE9AFEED99FDE842F0DC23FC
:10236600ACF0D0E0FFD0E0FED0E0FDAB8220E7107D
:102376001BEB60BAEC2CFCEF33FFEE33FEED33FDC6
:10238600022430E803F830E705C0F075F000EF2FBF
:10239600FFEE33FEED33FD40B830E7C280AA75F09C
:1023A60020800E75F010800575F0087D007E007F98
:1023B600003392D530D5031229E1EC334010EF33C8
:1023C600FFEE33FEED33FDEC33FCD5F0ED22E5F008
:1023D600247EA2D513CC92E7CDCEFF22EDD2E7CD57
:1023E60033EC3392D524814006E4FFFEFDFC22FC4B
:1023F600E4CFCECDCC24E0501174FF80EDC3CC13D6
:10240600CCCD13CDCE13CECF13CF0470F030D5DEA6
:102416000229E1E9D2E7C933E833F892D5EDD2E7EC
:10242600CD33EC33FC5002B2D522EC30E7100FBFAF
:10243600000C0EBE00080DBD00040BEB6014A2D507
:10244600EB13FCED92E7FD2274FFFCFDFEFF22E498
:1024560080F8A2D574FF13FC7D80E480EFF920E7B5
:102466002824F950037907E4F42402FB18DBFDE67F
:1024760024FB5014E9600DE4F618E604F6B40A08E5
:10248600E4F6D9F57401F60A22C2D522ED33EC330F
:1024960092D5FA602AB4FF33EDC2E77BFF60067A75
:1024A6002479B7E4227A2479C020D5047A2479BB2A
:1024B600224E614E002B494E46002D494E4600E401
:1024C6007A08F608DAFC7B00740722E8C0E0ECC064
:1024D600E0EDC0E0EEC0E0EFC0E0EA75F010A4CA9F
:1024E600ABF075F04DA42BFBE435F0FCEA2410FAB2
:1024F600EB34C5FBEC34D9FCEDC2E7FF75F056A40E
:10250600F42411C5F0F434C58FF0A42AE5F03BE4B9
:102516003CF620E7141225C5D0E0FFD0E0FED0E05F
:10252600FDD0E0FC1223078014F4041225C5D0E088
:10253600FFD0E0FED0E0FDD0E0FC1221FED0E0F8B6
:10254600E6FAEDD2E7CD33EC332482FBE4C3CF3396
:10255600CFCE33CECD33CD33DBF37B0775F00A8494
:102566006004F6081B0AE5F0F6088FF0740AA4FF6B
:10257600ACF08EF0740AA42CFEACF050010C8DF079
:10258600740AA42CFDE435F0F608DBDE7407223F5E
:102596008000004120000042C80000447A00004646
:1025A6001C400047C35000497424004B1896804CC9
:1025B600BEBC205A0E1BCA6753C21C749DC5AEFB17
:1025C60060065407601C23231225F3EB5438600978
:1025D6001225DF1225EE1221FEECF8EDF9EEFAEFE8
:1025E600CB22EB1225EE80F1543803241C9025955E
:1025F600FE93FC0EEE93FD0EEE930ECE93FF22E7B6
:1026060009F608DFFA8046E709F208DFFA803E8815
:10261600828C83E709F0A3DFFA8032E309F608DF4C
:10262600FA8078E309F208DFFA807088828C83E307
:1026360009F0A3DFFA806489828A83E0A3F608DFC3
:10264600FA805889828A83E0A3F208DFFA804C80F8
:10265600D280FA80C680D4806980F2803380108070
:10266600A680EA809A80A880DA80E280CA803389D0
:10267600828A83ECFAE493A3C8C582C8CCC583CC0E
:10268600F0A3C8C582C8CCC583CCDFE9DEE7800DE0
:1026960089828A83E493A3F608DFF9ECFAA9F0EDC0
:1026A600FB2289828A83ECFAE0A3C8C582C8CCC51E
:1026B60083CCF0A3C8C582C8CCC583CCDFEADEE8EC
:1026C60080DB89828A83E493A3F208DFF980CC88D1
:1026D600F0EF60010E4E60C388F0ED2402B40400F2
:1026E60050B9F582EB2402B4040050AF232345828F
:1026F6002390265573BB010689828A83E022500205
:10270600E722BBFE02E32289828A83E49322BB018D
:102716000CE58229F582E5833AF583E0225006E945
:102726002582F8E622BBFE06E92582F8E222E5824A
:1027360029F582E5833AF583E49322BB010FF8E598
:102746008229F582E5833AF583E028F0225009C50F
:102756008229F8E58226F622BBFE09C58229F8E21F
:102766002582F222F8EA2583F583E9932822BB0124
:102776000689828A83F0225002F722BBFE01F322E9
:10278600F8BB010DE58229F582E5833AF583E8F089
:10279600225006E92582C8F622BBFE05E92582C835
:1027A600F222BC000BBE0029EF8DF084FFADF022B3
:1027B600E4CCF875F008EF2FFFEE33FEEC33FCEEB9
:1027C6009DEC984005FCEE9DFE0FD5F0E9E4CEFDAC
:1027D60022EDF8F5F0EE8420D21CFEADF075F0087F
:1027E600EF2FFFED33FD4007985006D5F0F222C3D8
:1027F60098FD0FD5F0EA22C2D5EC30E709B2D5E450
:10280600C39DFDE49CFCEE30E715B2D5E4C39FFF03
:10281600E49EFE1227A8C3E49DFDE49CFC800312FF
:1028260027A830D507C3E49FFFE49EFE22C5F0F833
:10283600A3E028F0C5F0F8E582158270021583E062
:1028460038F022A3F8E0C5F025F0F0E58215827095
:10285600021583E0C838F0E822BB0110E58229F5AD
:1028660082E5833AF583E0F5F0A3E0225009E925F5
:1028760082F886F008E622BBFE0AE92582F8E2F530
:10288600F008E222E5832AF583E993F5F0A3E993BC
:1028960022F8BB0111E58229F582E5833AF583E842
:1028A600F0E5F0A3F0225009E92582C8F608A6F063
:1028B60022BBFE09E92582C8F2E5F008F222E88F7C
:1028C600F0A4CC8BF0A42CFCE98EF0A42CFC8AF0AE
:1028D600EDA42CFCEA8EF0A4CDA8F08BF0A42DCCB0
:1028E6003825F0FDE98FF0A42CCD35F0FCEB8EF009
:1028F600A4FEA9F0EB8FF0A4CFC5F02ECD39FEE4EF
:102906003CFCEAA42DCE35F0FDE43CFC2275F00833
:10291600758200EF2FFFEE33FECD33CDCC33CCC521
:102926008233C5829BED9AEC99E58298400CF5823C
:10293600EE9BFEED9AFDEC99FC0FD5F0D6E4CEFBAE
:10294600E4CDFAE4CCF9A88222B800C1B90059BA9C
:10295600002DEC8BF084CFCECDFCE5F0CBF97818CA
:10296600EF2FFFEE33FEED33FDEC33FCEB33FB10C4
:10297600D703994004EB99FB0FD8E5E4F9FA2278DE
:1029860018EF2FFFEE33FEED33FDEC33FCC933C9F0
:1029960010D7059BE99A4007EC9BFCE99AF90FD8FA
:1029A600E0E4C9FAE4CCFB2275F010EF2FFFEE331A
:1029B600FEED33FDCC33CCC833C810D7079BEC9A59
:1029C600E899400AED9BFDEC9AFCE899F80FD5F0E2
:1029D600DAE4CDFBE4CCFAE4C8F922C3E49FFFE4D1
:1029E6009EFEE49DFDE49CFC22EB9FF5F0EA9E42F0
:1029F600F0E99D42F0EC6480C864809845F022EBD3
:102A06009FF5F0EA9E42F0E99D42F0E89C45F022EF
:102A1600E8600FECC313FCED13FDEE13FEEF13FF9E
:102A2600D8F122E8600FEFC333FFEE33FEED33FD3E
:102A3600EC33FCD8F1227401FF3395E0FEFDFC086F
:102A46000808E6CF2FF618E6CE3EF618E6CD3DF698
:102A560018E6CC3CF622ECF0A3EDF0A3EEF0A3EFE3
:102A6600F022A8828583F0D083D082122A7F122A90
:102A76007F122A7F122A7FE473E493A3C583C5F0ED
:102A8600C583C8C582C8F0A3C583C5F0C583C8C5BC
:102A960082C822A42582F582E5F03583F58322FAE1
:102AA600E6FB0808E6F925F0F618E6CA3AF622D05B
:102AB60083D082F8E4937012740193700DA3A393EC
:102AC600F8740193F5828883E4737402936860EF67
:102AD600A3A3A380DFD083D082E493701274019302
:102AE600700DA3A393F8740193F5828883E473743D
:102AF60002936C70127403936D700C7404936E7071
:102B0600067405936F60DDA3A3A3A3A3A380CAE302
:102B1600F5F009E208B5F06D606B80F3E3F5F009B6
:102B2600E608B5F060605E80F387F009E608B5F068
:102B360054605280F487F009E208B5F04860468098
:102B4600F488828C8387F009E0A3B5F0386036807C
:102B5600F488828C8387F009E493A3B5F027602577
:102B660080F388828C83E3F5F009E0A3B5F0166064
:102B76001480F388828C83E3F5F009E493A3B5F01F
:102B860004600280F2022C40808580E7808E80D22D
:102B9600803C8015806C807E809B80B5808B80A178
:102BA600804F8070803A022C4C89828A83ECFAE44A
:102BB60093F5F0A3C8C582C8CCC583CCE493A3C85B
:102BC600C582C8CCC583CCB5F070606E80E18982C1
:102BD6008A83E493F5F0A3E208B5F05E605C80F2C8
:102BE60089828A83E0F5F0A3E608B5F04D604B8054
:102BF600F389828A83E0F5F0A3E208B5F03C603AF7
:102C060080F389828A83E493F5F0A3E608B5F02A77
:102C1600602880F2805389828A83ECFAE493F5F087
:102C2600A3C8C582C8CCC583CCE0A3C8C582C8CC1E
:102C3600C583CCB5F004600280E27FFFB5F0020FD9
:102C46002240027F012289828A83ECFAE0F5F0A312
:102C5600C8C582C8CCC583CCE0A3C8C582C8CCC5CC
:102C660083CCB5F0D560D380E389828A83ECFAE021
:102C7600F5F0A3C8C582C8CCC583CCE493A3C8C568
:102C860082C8CCC583CCB5F0B160AF80E288F0EDE8
:102C96002402B4040050A3F582EB2402B4040050CD
:102CA600992323458223902B8E73EF4E6012EF609B
:102CB600010EEDBB010B89828A83F0A3DFFCDEFAED
:102CC6002289F05007F709DFFCA9F022BBFEFCF3CE
:102CD60009DFFCA9F022EF8DF0A4A8F0CF8CF0A4B8
:102CE60028CE8DF0A42EFE2278A37C097D017BFFE1
:102CF6007ADA7934122C93EF3395E04F700302B7EA
:102D0600DF78A37C097D017BFF7ADA793B122C936D
:102D1600EF3395E04F7003024E1178A37C097D01D5
:102D26007BFF7ADA7948122C93EF3395E04F7003E4
:102D360002C15E78A37C097D017BFF7ADA794D12A8
:102D46002C93EF3395E04F7003028D1178A37C0925
:102D56007D017BFF7ADA7952122C93EF3395E04F9F
:102D6600700302A82078A37C097D017BFF7ADA79BB
:102D760057122C93EF3395E04F700302B3FB78A301
:102D86007C097D017BFF7ADA795F122C93EF33950C
:102D9600E04F700302D26578A37C097D017BFF7A40
:102DA600DA7963122C93EF3395E04F700302CF6408
:102DB60078A37C097D017BFF7ADA7967122C93EF81
:102DC6003395E04F700302672178A37C097D017B70
:102DD600FF7ADA7971122C93EF3395E04F70030284
:102DE600692578A37C097D017BFF7ADA7979122C33
:102DF60093EF3395E04F7003026CF478A37C097D62
:102E0600017BFF7ADA797E122C93EF3395E04F70CF
:102E16000302650978A37C097D017BFF7ADA79854F
:102E2600122C93EF3395E04F700302708778A37CE2
:102E3600097D017BFF7ADA7988122C93EF3395E0CE
:102E46004F70030233E478A37C097D017BFF7ADAB5
:102E5600798E122C93EF3395E04F700302A1B77869
:102E6600A37C097D017BFF7ADA7994122C93EF33E8
:102E760095E04F700302A25678A37C097D017BFF83
:102E86007ADA799A122C93EF3395E04F700302B4F5
:102E96006D78A37C097D017BFF7ADA79A0122C93E9
:102EA600EF3395E04F7003026B1A78A37C097D011E
:102EB6007BFF7ADA79AA122C93EF3395E04F7003F1
:102EC60002D27878A37C097D017BFF7ADA79B51284
:102ED6002C93EF3395E04F7003028F7B78A37C0928
:102EE6007D017BFF7ADA79BF122C93EF3395E04FA1
:102EF600700302C5B478A37C097D017BFF7ADA7979
:102F0600CB122C93EF3395E04F700302460578A35E
:102F16007C097D017BFF7ADA79D1122C93EF339508
:102F2600E04F700302D23578A37C097D017BFF7ADE
:102F3600DA79D8122C93EF3395E04F700302D23E24
:102F460078A37C097D017BFF7ADA79DE122C93EF78
:102F56003395E04F700302CFD178A37C097D017BC6
:102F6600FF7ADA79E2122C93EF3395E04F70030281
:102F7600D18078A37C097D017BFF7ADA79E7122C70
:102F860093EF3395E04F7003027DFC78A37C097DB7
:102F9600017BFF7ADA79F0122C93EF3395E04F70CC
:102FA60002801678A37C097D017BFF7ADA79F61216
:102FB6002C93EF3395E04F700302C96778A37C0921
:102FC6007D017BFF7ADA79FC122C93EF3395E04F83
:102FD6007002801678A37C097D017BFF7ADB79017C
:102FE600122C93EF3395E04F7003025D4678A37C75
:102FF600097D017BFF7ADB790A122C93EF3395E08A
:103006004F7002801678A37C097D017BFF7ADB79FD
:1030160015122C93EF3395E04F700302CCB378A3CF
:103026007C097D017BFF7ADB7920122C93EF3395A7
:10303600E04F700302A07778A37C097D017BFF7ABD
:10304600DB792B122C93EF3395E04F700302A11717
:1030560078A37C097D017BFF7ADB7937122C93EF0D
:103066003395E04F700302813D78A37C097D017B97
:10307600FF7ADB794B122C93EF3395E04F70030206
:10308600977078A37C097D017BFF7ADB795E122C31
:1030960093EF3395E04F700302A70678A37C097D72
:1030A600017BFF7ADB796A122C93EF3395E04F7040
:1030B6000302C1B278A37C097D017BFF7ADB7977B5
:1030C600122C93EF3395E04F700302D1B778A37CAF
:1030D600097D017BFF7ADB7981122C93EF3395E032
:1030E6004F700302C64678A37C097D017BFF7ADB1D
:1030F6007990122C93EF3395E04F700302D1AA78A2
:10310600A37C097D017BFF7ADB799A122C93EF333E
:1031160095E04F700302B13178A37C097D017BFFF6
:103126007ADB79AB122C93EF3395E04F700302965E
:103136001378A37C097D017BFF7ADB79BB122C9384
:10314600EF3395E04F700302D0A578A37C097D018B
:103156007BFF7ADB79D3122C93EF3395E04F700324
:1031660002D0B678A37C097D017BFF7ADB79E91270
:103176002C93EF3395E04F700302740078A37C091B
:103186007D017BFF7ADB79F5122C93EF3395E04FC7
:10319600700302BEA778A37C097D017BFF7ADC79E8
:1031A60007122C93EF3395E04F700302C2AE78A35B
:1031B6007C097D017BFF7ADC7913122C93EF339522
:1031C600E04F700302981D78A37C097D017BFF7A8E
:1031D600DC7920122C93EF3395E04F70030287D5EC
:1031E60078A37C097D017BFF7ADC7931122C93EF81
:1031F6003395E04F700302A5E478A37C097D017B3B
:10320600FF7ADC7941122C93EF3395E04F7003027D
:10321600A79378A37C097D017BFF7ADC794E122C7B
:1032260093EF3395E04F700302ACCE78A37C097D13
:10323600017BFF7ADC7954122C93EF3395E04F70C3
:103246000302AD4C78A37C097D017BFF7ADC7961B2
:10325600122C93EF3395E04F700302CD7978A37C5F
:10326600097D017BFF7ADC7970122C93EF3395E0B0
:103276004F700302CFE578A37C097D017BFF7ADCE2
:103286007981122C93EF3395E04F700302B54E7897
:10329600A37C097D017BFF7ADC7989122C93EF33BD
:1032A60095E04F70030294A778A37C097D017BFF0C
:1032B6007ADC7991122C93EF3395E04F7003029FDD
:1032C6003778A37C097D017BFF7ADC799A122C93EF
:1032D600EF3395E04F7003029FD778A37C097D01F9
:1032E6007BFF7ADC79A3122C93EF3395E04F7003C2
:1032F60002CE0A78A37C097D017BFF7ADC79AC12C9
:103306002C93EF3395E04F700302D0E978A37C0944
:103316007D017BFF7ADC79B2122C93EF3395E04F77
:10332600700302B22478A37C097D017BFF7ADC79E5
:10333600BA122C93EF3395E04F700302B5BD78A314
:103346007C097D017BFF7ADC79C2122C93EF3395E1
:10335600E04F700302D10878A37C097D017BFF7AD8
:10336600DC79CD122C93EF3395E04F7003029973FD
:1033760078A37C097D017BFF7ADC79D9122C93EF47
:103386003395E04F700302C8FD78A37C097D017B6D
:10339600FF7ADC79E8122C93EF3395E04F70030245
:1033A600CCDB78A37C097D017BFF7ADC79F3122CD8
:1033B60093EF3395E04F700302A39278A37C097DC7
:1033C600017BFF7ADC79FB122C93EF3395E04F708B
:1033D6000302AA487BFF7ADD79031241F822901B8B
:1033E60047E0FCA3E0FDA3E0FEA3E02401FFE43EEA
:1033F600FEE43DFDE43CFC901B47122A5C901BA4B6
:10340600122A6800000010E4901BA0F0A3F09009B7
:1034160087E070069009B374FFF0E4901BA0F0A358
:10342600F0900987E0FFC3901BA1E09F901BA0E0EE
:1034360094004003023786E0FEA3E0FF901B677509
:10344600F013122A99EE75F013A42583F583E0FC98
:10345600A3E024B3F58274093CF583E5822FF58257
:10346600E5833EAF82F5228F23901BA0A3E0901B3D
:103476005E75F013122A99EE75F013A42583F58371
:10348600E0FCA3E0FDA3E0FEA3E0F52F8E2E8D2D3C
:103496008C2C7F007E367D6E7C0112C7E3901BA0CC
:1034A600E0FEA3E0FF901B6475F013122A99EE75F7
:1034B600F013A42583F583E0FDD3940174809480F2
:1034C60050030237157C00901B6975F013EF122A22
:1034D60099EE75F013A42583F583E0FEA3E0FF12B1
:1034E60027A8901BA2ECF0A3EDF04C7036901BA021
:1034F600E0FEA3E0FF901B6B75F013122A99EE75A0
:10350600F013A42583F583E07D0070027D01901BF6
:103516006B75F013EF122A99EE75F013A42583F557
:1035260083EDF0901BA0E0FEA3E0FF901B6975F011
:1035360013122A99EE75F013A42583F583E475F02A
:1035460001122833901B5A75F013EF122A99EE7563
:10355600F013A42583F583E0FCA3E0FDA3E0FEA31E
:10356600E0FFE47BB0FAF9F8C3122A0570597F40F0
:103576007E427D0FFC901BA0E0FAA3E0901B5E75D7
:10358600F013122A99EA75F013A42583F583122AFB
:103596005C12D19C901BA0E0FEA3E0901B6B75F023
:1035A60013122A99EE75F013A42583F583E0FF1212
:1035B600D0D812D135901BA2A3E0540F04901BA8BB
:1035C600F044B0F0023696901BA0E0FEA3E0901BFC
:1035D6005A75F013122A99EE75F013A42583F58314
:1035E600E0FCA3E0FDA3E0FEA3E0FFE47BC0FAF964
:1035F600F8C3122A057037901BA0E0FEA3E0901BCB
:103606006B75F013122A99EE75F013A42583F583D2
:10361600E02482F582E43409F583E0FF901BA2A33F
:10362600E0FEEF4E04901BA8F044C0F08062901BB1
:10363600A0E0FEA3E0901B5A75F013122A99EE75CE
:10364600F013A42583F583E0FCA3E0FDA3E0FEA32D
:10365600E0FFE47BA17A16F9F8C3122A05703190CF
:103666001BA0E0FEA3E0901B6B75F013122A99EEE7
:1036760075F013A42583F583E02482F582E43409EA
:10368600F583E0FF901BA2A3E0FEEF4E901BA8F08F
:10369600901BA0E0FEA3E0901B5A75F013122A9926
:1036A600EE75F013A42583F583E0FCA3E0FDA3E00B
:1036B600FEA3E0540FFFE4FBFAF9F8C3122A0570E3
:1036C60019E5232401FFE43522FE901BA8E0FB90B8
:1036D6001BA0A3E0F52EE4FD8017E5232401FFE4FB
:1036E6003522FE901BA8E0FB901BA0A3E0F52E7DE3
:1036F60001125A6D78A97C1B7D017E007F0312267C
:10370600D5901BA8E0852382852283A3F08024E53B
:10371600232401FFE43522FE901BA0A3E0F52E7BB7
:1037260001E4FD125A6D78A97C1B7D017E007F03A2
:103736001226D5901BA9E0852382852283F0901B53
:10374600A4E0F8A3E0F9A3E0FAA3E0FB901BABE04A
:103756002401FF901BAAE03400FEE4FCFDEB2FFFE2
:10376600EA3EFEED39FDEC38FC901BA4122A5C9073
:103776001BA1E004F07006901BA0E004F0023427C1
:103786007E097FA3127829E4901BA8F0FF7E0CFD2A
:10379600FC901BA4E0F8A3E0F9A3E0FAA3E0FBD3B6
:1037A600122A05400A7E097FA37D007C108046E42C
:1037B600FF7E08FDFC901BA4E0F8A3E0F9A3E0FA65
:1037C600A3E0FBD3122A05400A7E097FA37D007C75
:1037D6000C8022E4FF7E04FDFC901BA4E0F8A3E02D
:1037E600F9A3E0FAA3E0FBD3122A0540127E097F73
:1037F600A37D007C0812CC37901BA8EFF0800590C3
:103806001BA8E4F012D0FEE4901BA0F0A3F0901BDE
:10381600A0E0FEA3E0FFC3EE9404501F74A32FF5AF
:103826008274093EF583E0FF12D117901BA1E004D4
:10383600F070DB901BA0E004F080D3E4FF7E04FD73
:10384600FC901BA4E0F8A3E0F9A3E0FAA3E0FBC315
:10385600122A055008901BA8E0FF12D117E4901B0E
:10386600A0F0A3F0901BA0E0FEA3E0FFC3EE94043B
:10387600501C74A32FF58274093EF583E4F0901B67
:10388600A1E004F070DE901BA0E004F080D62212C6
:103896008EB38F118E108D0F8C0E12BCE3EF602746
:1038A6007D09AF16AE1512600B7E087F007D007B8A
:1038B600017A007900122CB07400440060097D1270
:1038C600AF16AE1512600BE4F522F523740025231E
:1038D600F58274003522F583E0FF74A02523F58276
:1038E600741B3522F583EFF00523E52370020522CC
:1038F6006408452270D67E117F947D007B017A098B
:1039060079A3122CB078A37C097D017B017A00791A
:10391600007E047F001226D5E4F52EF52F7F807EEB
:1039260008FDFC12851A7E097F607D007B017A0006
:103936007900122CB012BCE3EF60097D09AF16AE18
:103946001512600B9000B8E09000CAF09000B9E044
:103956009000CBF09000BAE09000CCF09000BBE075
:103966009000CDF09000BCE09000CEF09000BDE05D
:103976009000CFF09000BEE09000D0F0900991E06A
:10398600FF9000D3F0900992E0FE9000D4F09009E9
:1039960093E0FD9000D5F0900994E0FC9000D6F0FD
:1039A600900995E0FB9000D7F0900996E0F9900019
:1039B600D8F0900997E0FA9000D9F0E4900031F041
:1039C600900025EFF0A3EEF0A3EDF0A3ECF0A3EB4F
:1039D600F0A3E9F0A3EAF0900991E09000DCF09002
:1039E6000992E09000DDF0900993E09000DEF090FF
:1039F6000994E09000DFF0900995E09000E0F0A3D4
:103A0600E9F0900997E09000E2F07E087F007D00E3
:103A16007B017A0979A3122CB0E4F522F523740010
:103A26002523F58274003522F583E0FF74A3252350
:103A3600F58274093522F583EFF00523E52370023C
:103A46000522B400D9E522B404D47E097FA37DFE05
:103A56007C0312CC37900DA1EFF07B017A0979A394
:103A66007DFF7C0312C932900DA2EFF0E4FFFE1237
:103A76009E96E4F52EF52F7F907E08FDFC12851AA2
:103A86007E087F007D007B017A0979A3122CB0E5C0
:103A9600112470FFE51034F7FEE50F34FFFDE50E47
:103AA60034FFFCE4FB7A08F9F81228C48F278E2627
:103AB6008D258C24780E122A3CE4F52EF52F1285DE
:103AC6001AAF11AE10AD0FAC0EE4F52EF52F128520
:103AD6001AAD19AC18AF16AE1512A937AD19AC1838
:103AE600AF16AE1512A9C2900979E07E008E22F5B6
:103AF6002375F020A4FF90097BE07C002FFDEC35B8
:103B0600F0FC900978E02414FFEF7F0025E0FEEF3B
:103B16002DFFEC3E901BC8F0A3EFF090097DE075F9
:103B2600F020A4FFA3E0C3137C002FFDEC35F0FCCE
:103B360090097CE07F0033333354F8FEEF2DFFEC21
:103B46003E901BCAF0A3EFF078A87C1B7D017BFF9B
:103B56007AE079E67E007F201226D5901BCAE0FE29
:103B6600A3E0F9901BB6F0EEFDA3F0901BC8E0FEB3
:103B7600A3E0901BB8F0EEFFFCA3F0901BC8A3E0F7
:103B8600FB901BBAF0A3ECF0901BBEE9F0A3EDF09E
:103B9600A3EBF0A3EFF078A37C097D017B017A1BF0
:103BA60079A87E007F201226D578A87C1B7D017B14
:103BB600FF7AE079C67E007F201226D5901BCAE0E8
:103BC600FEA3E0F9901BB6F0EEFDA3F0901BC8E053
:103BD600FEA3E0901BB8F0EEFFFCA3F0901BC8A379
:103BE600E0FB901BBAF0A3ECF0901BBEE9F0A3ED4E
:103BF600F0A3EBF0A3EFF078C37C097D017B017A9B
:103C06001B79A87E007F201226D578A87C1B7D0113
:103C16007BFF7AE179067E007F201226D5901BCAAB
:103C2600E0FEA3E0F9901BB6F0EEFDA3F0901BC8F2
:103C3600E0FEA3E0901BB8F0EEFFFCA3F0901BC8DB
:103C4600A3E0FB901BBAF0A3ECF0901BBEE9F0A337
:103C5600EDF0A3EBF0A3EFF078E37C097D017B01A7
:103C66007A1B79A87E007F201226D59009FFE527CA
:103C7600F0FFAE26AD25AC247808122A16A3EFF085
:103C8600AF27AE26AD25AC247810122A16A3EFF086
:103C9600AF27AE26AD25AC247818122A16A3EFF06E
:103CA600E4F522F52374A02523F582741B3522F54D
:103CB60083E0700F74A02523F582741B3522F583EB
:103CC6007420F00523E5237002052264084522705E
:103CD600D4E4F522F52374A02523F582741B35223E
:103CE600F583E0FF74E32523F58274093522F58315
:103CF600EFF00523E523700205226408452270D6FD
:103D0600E4F52EF52FFF7E08FDFC12851A02C4D6B7
:103D1600C3E51A94085054901B47E0FCA3E0FDA3AA
:103D2600E0FEA3E02401FFE43EFEE43DFDE43CFCAE
:103D3600901B47122A5C900981E0FBE4FAF9F8909F
:103D46001B47E0FCA3E0FDA3E0FEA3E0FF12294F22
:103D5600AC00AD01AE02AF03E4FBFAF9F8C3122AD8
:103D66000570AD127249127CD980A512D2847D02EB
:103D7600AF16AE1512600B12BCE3E4FFFE74002F03
:103D8600F58274003EF583E0FD74A02FF582741B66
:103D96003EF583EDF00FBF00010EEF64084E70DDB7
:103DA6009000B8E09000CAF09000B9E09000CBF027
:103DB6009000BAE09000CCF09000BBE09000CDF00F
:103DC6009000BCE09000CEF09000BDE09000CFF0F7
:103DD6009000BEE09000D0F0900991E0FF9000D3F3
:103DE600F0900992E0FE9000D4F0900993E0FD90E7
:103DF60000D5F0900994E0F99000D6F0900995E08E
:103E06009000D7F0900996E09000D8F0900997E0DE
:103E16009000D9F0E4900031F0900025EFF0A3EE89
:103E2600F0A3EDF0A3E9F0900995E0FF900029F0EA
:103E3600900996E0FE90002AF0900997E0FD900028
:103E46002BF0900991E09000DCF0900992E0900050
:103E5600DDF0900993E09000DEF0A3E9F0A3EFF027
:103E6600A3EEF0A3EDF07E087F007D007B017A09CA
:103E760079A3122CB0E4FEFF74002FF58274003E85
:103E8600F583E0FD74A32FF58274093EF583EDF00A
:103E96000FBF00010EE4B507DFEEB404DB7E097F39
:103EA600A37DFE7C0312CC37900DA1EFF07B017A47
:103EB6000979A37DFF7C0312C932900DA2EFF0E4CD
:103EC600FFFE129E9612BB6BE4F52EF52F7F907EB9
:103ED60008FDFC12851A12BA487B017A0979A312E9
:103EE600C05DE4F52EF52F7F407E08FDFC12851A95
:103EF600752E08752F007F417E087D007C00128597
:103F06001A7E087F007D007B017A0979A3122CB006
:103F1600E5112470FFE51034F7FEE50F34FFFDE5EB
:103F26000E34FFFCE4FB7A08F9F81228C48F268EBB
:103F3600258D248C23E5112401F511E43510F510A7
:103F4600E4350FF50FE4350EF50E12B9E5AD19ACF3
:103F560018AF16AE1512A937AD19AC18AF16AE15B7
:103F660012A9C2900979E075F020A4FF90097BE0C0
:103F76007C002FFDEC35F0FC900978E02414FFEF6F
:103F86007F0025E0FEEF2DFFEC3E901BC8F0A3EF6F
:103F9600F090097DE075F020A4FFA3E0C3137C0038
:103FA6002FFDEC35F0FC90097CE07F003333335471
:103FB600F8FEEF2DFFEC3E901BCAF0A3EFF078A8B9
:103FC6007C1B7D017BFF7AE079E67E007F2012264E
:103FD600D5901BCAE0FEA3E0F9901BB6F0EEFDA358
:103FE600F0901BC8A3E0901BB8F0901BC8E0FF90B0
:103FF6001BB9F0901BC8A3E0FE901BBAF0A3EFF02C
:10400600901BBEE9F0A3EDF0A3EEF0901BC8E09084
:104016001BC1F078A37C097D017B017A1B79A87E00
:10402600007F201226D578A87C1B7D017BFF7AE0D5
:1040360079C67E007F201226D5901BCAE0FEA3E03B
:10404600F9901BB6F0EEFDA3F0901BC8A3E0901B01
:10405600B8F0901BC8E0FF901BB9F0901BC8A3E016
:10406600FE901BBAF0A3EFF0901BBEE9F0A3EDF0B3
:10407600A3EEF0901BC8E0901BC1F078C37C097DCD
:10408600017B017A1B79A87E007F201226D578A8AD
:104096007C1B7D017BFF7AE179067E007F2012265C
:1040A600D5901BCAE0FEA3E0F9901BB6F0EEFDA387
:1040B600F0901BC8A3E0901BB8F0901BC8E0FF90DF
:1040C6001BB9F0901BC8A3E0FE901BBAF0A3EFF05B
:1040D600901BBEE9F0A3EDF0A3EEF0901BC8E090B4
:1040E6001BC1F078E37C097D017B017A1B79A87EF0
:1040F600007F201226D59009FFE526F0FFAE25ADFC
:1041060024AC237808122A16A3EFF0AF26AE25AD0D
:1041160024AC237810122A16A3EFF0AF26AE25ADF5
:1041260024AC237818122A16A3EFF0E4FEFF74A03D
:104136002FF582741B3EF583E0700D74A02FF58277
:10414600741B3EF5837420F00FBF00010EEF640868
:104156004E70DBE4FEFF74A02FF582741B3EF583E0
:10416600E0FD74E32FF58274093EF583EDF00FBF91
:1041760000010EEF64084E70DDE4F52EF52FFF7E8C
:1041860008FDFC12851A12CC619009687403F022AE
:10419600E54A2436F8E6054A2278333007027836AF
:1041A600E475F001122AA50226FB2000EB7F2ED231
:1041B600008018EF540F2490D43440D4FF30040B01
:1041C600EF24BFB41A0050032461FFE54B600215CB
:1041D6004B054EE54E7002054D30070D7833E475FC
:1041E600F001122AA5EF02277402D1267403D20722
:1041F6008003E4C207F54A8B338A348935E4F54BEC
:10420600F54DF54EE54B60077F201241D180F575DF
:104216004CFFC201C200C202C203C205C206C208E6
:1042260012419FFF700D3007057F001241E2AF4E2D
:10423600AE4D22B4255FC2D5C20412419FFF24D0E1
:10424600B40A00501A75F00A784B30D50508B6FF47
:104256000106C6A426F620D5047002D20380D9240E
:10426600CFB41A00EF5004C2E5D2040244CFD20103
:1042760080C6D20080C0D20280BCD2D580BAD20518
:1042860080B47F201241D12002077401B54B004053
:10429600F1124196FF1241D102420AD208D206809B
:1042A60095124196FB124196FA124196F94A4B70C5
:1042B6000679C67A457BFF20022EE54B602A7E00F2
:1042C6008E8275830012271460060EEE654C70F020
:1042D600C2D5EBC0E0EAC0E0E9C0E0EE12452FD05F
:1042E600E0F9D0E0FAD0E0FB1226FBFF60AAEBC0B3
:1042F600E0EAC0E0E9C0E01241D1D0E02401F9D003
:10430600E03400FAD0E0FBE54C0460DCD54CD98003
:1043160087D20280A212451260F7E54C70010412A2
:104326002463A94C600DE54C600914F54C1245B99F
:10433600EF60F3EA30E702F404C3995077EAF42514
:104346004C0430E701E404F54C800D12451260C1BF
:10435600EA054C254C122463EA7849F630E701E475
:10436600254C04D54C042005011412452FE4C0E069
:104376001245B97849E6601320E70714F61241B9E9
:10438600802204F6D0E014C0E07F001241B9E54C6B
:1043960060071241B0154C800B3005031241B0D0B6
:1043A600E002420AD0E00480C512451260A0E54C46
:1043B600041224637849EAF6E54C200502600104FC
:1043C600240412452F74FF04C0E01245B91241B906
:1043D600E54C20050260031241B0D0E0B54CE87F01
:1043E600451241C37849E67F2B30E7047F2DF4045C
:1043F600C0E01241D1D0E075F00A84C0F01241BA93
:10440600D0E01241BA02420A791080027908C20647
:10441600C2088008D2D5790A8004790AC2D5E54C4B
:10442600047002F54CE4FAFDFEFF124196FC7B088F
:10443600200113124196FD7B1030000A124196FEB0
:10444600124196FF7B20EC3382D592D55013C3E4FC
:104456003000069FFFE49EFEE42001039DFDE49CE0
:10446600FCE4CBF8C201EC700CCFCECDCCE824F83E
:10447600F870F38017C3EF33FFEE33FEED33FDEC38
:1044860033FCEB33FB994002FB0FD8E9EB30010517
:10449600F8D0E0C448B201C0E00AEC4D4E4F782097
:1044A6007B0070C2EAB54C0040BCC0E0124531D07A
:1044B600F0D0E0200104C4C0E0C4B201C0F0124153
:1044C600BAD0F0D5F0EB02420A122AB542A75344FD
:1044D6000E5842784C42744244124F441A44441ACD
:1044E60049428D4344205543514643AF45431B47FC
:1044F60045E650427C2D42802E42A32B4284234225
:10450600A12045CF2A423C480000429BE54CB4FF1F
:1045160003754C06124196FC124196FD124196FE19
:10452600124196FF7842022492790AA2D5200314FA
:10453600300509B910020404B9080104A2D5200601
:10454600025001042002689202B54B005034C0E0CC
:104556007F203003197F30A20272067205500F12B7
:104566004588C202C206C205C2087F30800F3005E8
:1045760003E9C0E01241D1300503D0E0F9D0E0B53F
:104586004BCC3005177F30B9100C1241D17F583013
:1045960004077F788003B908031241D13002057FF2
:1045A6002D0241D17F202008F87F2B2006F322928E
:1045B6000280CF7F00B4070050052442F8E6FF22B0
:1045C600286E756C6C2900D2011241963001F8C232
:1045D60001784B30D50108F602423C2D504349582C
:1045E6001241962403B405004001E49045E193127C
:1045F60041C2743A1241C2D203754B0402440EE41E
:10460600901BA0F0A3F0901BA0E0FEA3E024A3F56E
:104616008274093EF583E06010901BA1E004F070FF
:10462600E5901BA0E004F080DD901BA1E004F07093
:1046360006901BA0E004F0901BA0E0FEA3E024A3DC
:10464600F974093EFA7B011296C2901BA4EEF0A300
:10465600EFF0EE6003024A40EF14B40D004003028F
:104666004A4090467675F003A4C58325F0C583734A
:1046760002469D0246D70248E00248F002490E0271
:10468600492B0249AB0249D50249D90249DE024902
:10469600E2024A400249E81293F090097EE0FF9058
:1046A6001BA2E4F0A3EFF07FD07E0712CA33AD1948
:1046B600AC18AF16AE1512A9C290097EE0FF901B8A
:1046C600A2E07003A3E06F7F31700302492502491F
:1046D600DB12D28490097CE0FFE4FCFDFE7B3CFA11
:1046E600F9F81228C4A804A905AA06AB0790097D03
:1046F600E0FFE4FCFDFEEB2FFFEE3AFEED39FDECAC
:1047060038FC901BA6122A5C901BA6E0FCA3E0FDD9
:10471600A3E0FEA3E0FFE47B3CFAF9F81228C4907C
:104726001BA6122A5C901BA6E0F8A3E0F9A3E0FA08
:10473600A3E0FB90097EE0FFE4FCFDFEEB2FFFEE1D
:104746003AFEED39FDEC38FC901BA6122A5C901B54
:10475600A6E0FCA3E0FDA3E0FEA3E02408FFE43E00
:10476600FEE43DFDE43CFC901BA6122A5CE47B3C87
:10477600FAF9F8901BA6E0FCA3E0FDA3E0FEA3E097
:10478600FF12294FAC00AD01AE02AF03901BAA1277
:104796002A5C901BAAA3A3A3E090098EF0901BA607
:1047A600E0FCA3E0FDA3E0FEA3E0FFA3E0F8A3E0A6
:1047B600F9A3E0FAA3E0FBC3EF9BFFEE9AFEED99A7
:1047C600FDEC98FC901BA6122A5C901BA6E0FCA3AD
:1047D600E0FDA3E0FEA3E0FFE47B3CFAF9F8122932
:1047E6004F901BA6122A5CE47B3CFAF9F8901BA6B4
:1047F600E0FCA3E0FDA3E0FEA3E0FF12294FAC001E
:10480600AD01AE02AF03901BAA122A5C901BAAA3AD
:10481600A3A3E090098DF0901BA6E0FCA3E0FDA306
:10482600E0FEA3E0FFA3E0F8A3E0F9A3E0FAA3E02B
:10483600FBC3EF9BFFEE9AFEED99FDEC98FC901BF7
:10484600A6122A5C901BA6E0FCA3E0FDA3E0FEA353
:10485600E0FFE47B3CFAF9F812294F901BA6122AD6
:104866005C901BA6A3A3A3E0FF90098CF0A3E0FD38
:10487600A3E0FB12C857900978E0FFA3E0FD90097A
:104886007BE0FB90097AE0F52512C56A12CF1C126F
:10489600D00D12CEFC12D048E47FF87E2AFDFCAB88
:1048A6000DAA0CA90BA80AC3122A057F0050027F85
:1048B60001E5147E0070027E01EF5E70DB12D2010C
:1048C60012D27112CF4DE51464017F32700512CBFE
:1048D600B4800312CBE0E4F5142212B0B6EC4D4ED0
:1048E6004F7F3370030249DB803512BBC9EF70136B
:1048F60012BC27EF700D12C3A3EF7F347003024979
:10490600DB801C7F340249A612BBC9EF701312BCB0
:1049160027EF700D12C3A3EF7F3570030249DB80CA
:104926007F7F35807BE4901BA0F0A3F0901BAA123A
:104936002A6800000000E4FFFE7D0FFC901BAAE041
:10494600F8A3E0F9A3E0FAA3E0FBC3122A05503F5F
:10495600901BAAE0FCA3E0FDA3E0FEA3E0FF1293F8
:1049660039901BA1E02FF0901BA0E03EF0901BAA0F
:10497600E0FCA3E0FDA3E0FEA3E02400FFEE34018B
:10498600FEE43DFDE43CFC901BAA122A5C80A7C312
:10499600901BA1E0945A901BA0E094007F36400340
:1049A60002CBE08030E4901BA4F0A3F0FF12CFA668
:1049B600E4752F80752E25F52DF52CFF7E367D6E40
:1049C6007C0112C7E37F3712CBB47F0102CFA67FEB
:1049D6003880027F3902CBB47D3080027D317F3151
:1049E6008052E4901BA0F0A3F0FF12CFA6127249EA
:1049F600D3901B3EE09488901B3DE09413400890B2
:104A06001BA0E4F0A304F07F0112CFA6127249C3E3
:104A1600901B3EE09488901B3DE094135008901B39
:104A2600A0E4F0A304F0901BA0E07002A3E07D33A5
:104A36007F31700302CAC812CAF82212BD3EEF7057
:104A460003024ADE12D28412BCE3EF60097D09AF8D
:104A560016AE1512600B900991E09000CAF090090D
:104A660092E09000CBF0900993E09000CCF0900992
:104A760094E09000CDF0900995E09000CEF090097A
:104A860096E09000CFF0900997E09000D0F07E0875
:104A96007F007D007B017A0979A3122CB078A37C74
:104AA600097D017B017A0079007E047F001226D5FC
:104AB6007E097FA37DFE7C0312CC37900DA1EFF01B
:104AC6007B017A0979A37DFF7C0312C932900DA27E
:104AD600EFF0E4FFFE129DF512BCE3EF60097D09DD
:104AE600AF16AE1512600B7B017A0079137D0412A6
:104AF600BB0DE47B7DFAF9F812294F900981EFF09E
:104B06007B017A0079177D0212BB0D900985EEF0C4
:104B1600A3EFF09003BDE0900987F0E4F524F525B6
:104B2600900987E0FFC3E5259FE524940040030232
:104B36004D49E525C4F8540FC868FFE524C454F070
:104B460048FE74BE2FF974033EFA7B017D0412BB46
:104B56000D901B5A75F013E525122A99E52475F078
:104B660013A42583F583122A5CE525C4F8540FC8DF
:104B760068FFE524C454F048FE74C22FF974033E5E
:104B8600FA7B017D0412BB0D901B5E75F013E525C3
:104B9600122A99E52475F013A42583F583122A5C5D
:104BA600E525C4F8540FC868FFE524C454F048FE50
:104BB60074C62FF974033EFA7B017D0212BB0D9079
:104BC6001B6275F013E525122A99E52475F013A4E6
:104BD6002583F583EEF0A3EFF0E525C4F8540FC85E
:104BE60068FFE524C454F048FE74C82FF5827403A8
:104BF6003EF583E0FD901B6475F013E525122A99B6
:104C0600E52475F013A42583F583EDF074C92FF917
:104C160074033EFA7B017D0212BB0DE5252FFFE5ED
:104C2600243EFE901B6775F013E525122A99E524AC
:104C360075F013A42583F583EEF0A3EFF0901B6BBC
:104C460075F013E525122A99E52475F013A425833A
:104C5600F5837401F0901B6975F013E525122A9906
:104C6600E52475F013A42583F583E4F0A3F0901BE7
:104C76005A75F013E525122A99E52475F013A42533
:104C860083F583E0FCA3E0FDA3E0FEA3E0FF122A88
:104C9600DB4CAD000000B04CDE000000C04D200033
:104CA6000016A100004D3E9000A8E0FF7E007007B0
:104CB60090098274BC800BEF64014E700A900982E1
:104CC60074BDF0A3F08071EF64024E706B900982A0
:104CD60074BCF0A304F080609000A8E0FD75F00AB3
:104CE60084FE25E025E0540C900982F0ED75F00A6B
:104CF60084AFF0EF25E025E0540CA3F09000B1E07E
:104D0600FF901B6C75F013E525122A99E52475F0C2
:104D160013A42583F583EFF0801E9000A8E0FD75AF
:104D2600F00A84FEC45470900982F0ED75F00A848E
:104D3600AFF0EFC45470A3F00525E52570020524F5
:104D4600024B26E4F51AF51B901B47122A68000051
:104D560000007508097509A3E4900975F0A3F090A1
:104D66000974F0F524F525900987E0FFC3E5259F32
:104D7600E52494004003024E10901B5A75F013E58B
:104D860025122A99E52475F013A42583F583E0FC02
:104D9600A3E0FDA3E0FEA3E0FFE47BC0FAF9F8C3BD
:104DA600122A05705A901B5E75F013E525122A9992
:104DB600E52475F013A42583F583E0FCA3E0FDA3A9
:104DC600E0FEA3E0FF752F00752E36752D6E752C4F
:104DD6000112C7E312D19C901B6C75F013E52512E6
:104DE6002A99E52475F013A42583F583E0FF12D0F4
:104DF600D812D1357F407E0D7D037C0012CE8D0505
:104E060025E52570020524024D6D22901BA3745FD3
:104E1600F074B52409F582E434D6F583E493F99069
:104E26001BA4F074B5240AF582E434D6F583E49322
:104E3600FF901BA5F0A3742EF090D6B5E493FE6404
:104E46004F6009EE644E6004EEB444047E31800285
:104E56007E30901BA7EEF090D6B5E493B44A17A324
:104E6600E493B4611115827583D6A3A3E493B46E5B
:104E7600057E31024F5190D6B5E493FEB446057EC9
:104E860032024F51EEB44D1A90D6B5A3E493B461F5
:104E96001115827583D6A3A3E493B472057E3302FB
:104EA6004F5190D6B5E493B4410BA3E493B4700587
:104EB6007E34024F5190D6B5E493FEB44D16A3E46A
:104EC60093B4611015827583D6A3A3E493B47904D1
:104ED6007E358077EEB44A1990D6B5A3E493B475BF
:104EE6001015827583D6A3A3E493B46E047E368030
:104EF6005A90D6B5E493B44A16A3E493B475101544
:104F0600827583D6A3A3E493B46C047E37803C9069
:104F1600D6B5E493FEB4410AA3E493B475047E388F
:104F26008029EEB453047E39802190D6B5E493FEF1
:104F3600B44F047E308014EEB44E047E31800C9063
:104F4600D6B5E4937E3FB444027E32901BA8EEF0C1
:104F560074B52404F582E434D6F583E493FEFD3378
:104F660095E0FCC3ED9430EC6480948040028002AE
:104F76007E30901BA9EEF0E4A3F0C3ED9430EC6410
:104F8600809480401074B52404F582E434D6F58309
:104F9600E493FE80027E30901BABEEF074B52405E0
:104FA600F582E434D6F583E493901BACF0A3742E1B
:104FB600F090D6B5E493FE644F6009EE644E60044B
:104FC600EEB444047E3180027E30901BAEEEF0904B
:104FD600D6B5E493B44A17A3E493B4611115827568
:104FE60083D6A3A3E493B46E057E310250C990D64E
:104FF600B5E493FEB446057E320250C9EEB44D1AAE
:1050060090D6B5A3E493B4611115827583D6A3A394
:10501600E493B472057E330250C990D6B5E493B4D6
:10502600410BA3E493B470057E340250C990D6B503
:10503600E493FEB44D16A3E493B461101582758310
:10504600D6A3A3E493B479047E358077EEB44A19E7
:1050560090D6B5A3E493B4751015827583D6A3A331
:10506600E493B46E047E36805A90D6B5E493B44A7F
:1050760016A3E493B4751015827583D6A3A3E4939F
:10508600B46C047E37803C90D6B5E493FEB4410AF6
:10509600A3E493B475047E388029EEB453047E39B4
:1050A600802190D6B5E493FEB44F047E308014EE92
:1050B600B44E047E31800C90D6B5E4937E3FB44462
:1050C600027E32901BAFEEF0A3742EF0A3E9F0A39C
:1050D600EFF0E4A3F078A37C097D017BFF7ADA790F
:1050E6000FFE7F081226D578AB7C097D017B017AFD
:1050F6001B79AB7E007F091226D578B47C097D0129
:105106007BFF7ADA79077E007F081226D5E4901BAA
:10511600A2F07E097FA37D19FC12CC37901BA2EF6B
:10512600F012D0FEE4901BA0F0A3F0901BA0E0FECE
:10513600A3E0FFC39419EE9400501F74A32FF582C9
:1051460074093EF583E0FF12D117901BA1E004F02D
:1051560070D9901BA0E004F080D1901BA2E0FF0262
:10516600D1178E228F238D24129B68901BEB122A57
:105176005CAF241275788B2C8A2D892E7F007E4099
:105186007D017C00901BEBE0F8A3E0F9A3E0FAA315
:10519600E0FBC3122A0540030254887E007F407D4F
:1051A600007B017A1B79A0122CB08523828522838D
:1051B600A3A3A3E0C3940A7480948050127538FFA9
:1051C6007539D2753A877B017A1B79A012BF57854C
:1051D6002382852283A3A3A3E0FF7E007B017A1BA3
:1051E60079E0127BB575380175391B753AE07B019C
:1051F6007A1B79A012BF577538FF7539D2753A896F
:105206007B017A1B79A012BF57852382852283A34F
:10521600E0C3940A7480948050127538FF7539D2B1
:10522600753A877B017A1B79A012BF578523828541
:105236002283A3E0FF7E007B017A1B79E0127BB517
:1052460075380175391B753AE07B017A1B79A01216
:10525600BF577538FF7539D2753A897B017A1B7944
:10526600A012BF57852382852283E0FF7E007B0143
:105276007A1B79E0127BB575380175391B753AE0F2
:105286007B017A1B79A012BF577538FF7539D27525
:105296003A8B7B017A1B79A012BF57E5232404F5CC
:1052A60082E43522F583E0C3940A74809480501218
:1052B6007538FF7539D2753A877B017A1B79A0124A
:1052C600BF57E5232404F582E43522F583E0FF7E0B
:1052D600007B017A1B79E0127BB575380175391BA5
:1052E600753AE07B017A1B79A012BF577538FF75B6
:1052F60039D2753A8D7B017A1B79A012BF57E52307
:105306002405F582E43522F583E0C3940A7480947B
:105316008050127538FF7539D2753A877B017A1B32
:1053260079A012BF57E5232405F582E43522F583DB
:10533600E0FF7E007B017A1B79E0127BB5753801B0
:1053460075391B753AE07B017A1B79A012BF577538
:1053560038FF7539D2753A8D7B017A1B79A012BF59
:1053660057E5232406F582E43522F583E0C3940A43
:105376007480948050127538FF7539D2753A877BE0
:10538600017A1B79A012BF57E5232406F582E4357E
:1053960022F583E0FF7E007B017A1B79E0127BB564
:1053A60075380175391B753AE07B017A1B79A012B5
:1053B600BF57E52E452D452C6012852C38852D3995
:1053C600852E3A7B017A1B79A012BF577E007F0B90
:1053D6007D007B017A1B79E0122CB0AF28AE27AD99
:1053E60026AC257B017A1B79E0127A8F7538017518
:1053F600391B753AE07B017A1B79A012BF577538C5
:10540600FF7539D2753A8B7B017A1B79A012BF578B
:10541600E52B452A4529600B852938852A39852BB0
:105426003A80097538FF7539D2753A8B7B017A1B3C
:1054360079A012BF577B017A1B79A012CFBCC3EFAC
:10544600943EEE9400501474A02FF582741B3EF522
:10545600837420F00FBF00010E80E3901BDE740DF5
:10546600F0A3740AF0901BEBE0FCA3E0FDA3E0FEC2
:10547600A3E0FF7B017A1B79A0753C00753D4012C5
:10548600B77322E4F522F523900987E0FFC3E523ED
:105496009FE5229400400302578B901B6775F0131B
:1054A600E523122A99E52275F013A42583F583E0F6
:1054B600FEA3E0FF74B3251BF5827409351AF58344
:1054C600E5822FF582E5833EF583E5822523F58285
:1054D600E5833522AF82F5268F27901B5E75F01384
:1054E600E523122A99E52275F013A42583F583E0B6
:1054F600FCA3E0FDA3E0FEA3E0F52F8E2E8D2D8C00
:105506002C7F007E367D6E7C0112C7E3901B64758E
:10551600F013E523122A99E52275F013A42583F5E5
:1055260083E0FFD39401748094805003025768EFA0
:10553600FD7C00901B6975F013E523122A99E5227C
:1055460075F013A42583F583E0FEA3E0FF1227A8D8
:105556008D24E5247033901B6B75F013E523122A16
:1055660099E52275F013A42583F583E07F00700288
:105576007F01901B6B75F013E523122A99E52275BE
:10558600F013A42583F583EFF0901B6975F013E5FE
:1055960023122A99E52275F013A42583F583E47571
:1055A600F001122833901B5A75F013E523122A993D
:1055B600E52275F013A42583F583E0FCA3E0FDA3A3
:1055C600E0FEA3E0FFE47BB0FAF9F8C3122A056017
:1055D6002E901B5E75F013E523122A99E52275F0CD
:1055E60013A42583F583E0FCA3E0FDA3E0FEA3E07E
:1055F600FF7B407A42790F7800C3122A0570461263
:10560600D19C901B6B75F013E523122A99E5227540
:10561600F013A42583F583E02482F582E43409F5AA
:1056260083E0FF12D0D812D135E4FFFE0FBF000190
:105636000EBE1FF8BF40F5E524540F04F52543259B
:10564600B0E40256F2901B5A75F013E523122A991C
:10565600E52275F013A42583F583E0FCA3E0FDA302
:10566600E0FEA3E0FFE47BC0FAF9F8C3122A057056
:105676002A901B6B75F013E523122A99E52275F023
:1056860013A42583F583E02482F582E43409F583A7
:10569600E0452404F5254325C08051901B5A75F03A
:1056A60013E523122A99E52275F013A42583F583C1
:1056B600E0FCA3E0FDA3E0FEA3E0FFE47BA17A16F5
:1056C600F9F8C3122A057024901B6B75F013E523B5
:1056D600122A99E52275F013A42583F583E0248226
:1056E600F582E43409F583E04524F525901B5A75C7
:1056F600F013E523122A99E52275F013A42583F504
:1057060083E0FCA3E0FDA3E0FEA3E0540FFFE4FB6F
:10571600FAF9F8C3122A057012E5272401FFE435C9
:1057260026FE85232EAB25E4FD8010E5272401FF08
:10573600E43526FE85232EAB257D01125A6D78A011
:105746007C1B7D017E007F031226D5852782852658
:1057560083A3E525F0901BA0E0852782852683F0AC
:105766008018AD23AC22AF27AE2612C99B78A07C49
:105776001B7D017E007F031226D50523E5237002DB
:10578600052202548E901BA0E0FF22901C9AE0FF97
:1057960090097EE0FE6F7003025866901C9AEEF048
:1057A600901C80E0FCA3E0FDA3E0FEA3E02401FF43
:1057B600E43EFEE43DFDE43CFC901C80122A5C9035
:1057C6001C84E0FCA3E0FDA3E0FEA3E02401FFE4CB
:1057D6003EFEE43DFDE43CFC901C84122A5C901CD9
:1057E60088E0FCA3E0FDA3E0FEA3E02401FFE43E85
:1057F600FEE43DFDE43CFC901C88122A5C901C8C67
:10580600E0FCA3E0FDA3E0FEA3E02401FFE43EFEEE
:10581600E43DFDE43CFC901C8C122A5C901C90E05C
:10582600FCA3E0FDA3E0FEA3E02401FFE43EFEE4CA
:105836003DFDE43CFC901C90122A5C901C94E0FC1C
:10584600A3E0FDA3E0FEA3E02401FFE43EFEE43D69
:10585600FDE43CFC901C94122A5C901C99E004F038
:10586600D3901B38E094E8901B37E094034043E460
:105876007F107E0EFDFC901C84E0F8A3E0F9A3E007
:10588600FAA3E0FBD3122A054028901C84122A684A
:1058960000000000901B37E0FEA3E0FFE48F288E97
:1058A60027F526F5257529FF752AE1752B267D0531
:1058B6008057C3901B3EE09488901B3DE0941350A4
:1058C6005AE47F107E0EFDFC901C90E0F8A3E0F9F0
:1058D600A3E0FAA3E0FB122A054040901C90122A8E
:1058E6006800000000901B3FE0FEA3E0FFC3948821
:1058F600EE9413501DE48F288E27F526F52575297D
:10590600FF752AE1752B2A7D0EAF16AE151251686A
:1059160080097D0FAF16AE1512600BC3901B38E0E1
:10592600941E901B37E094005047E47F107E0EFDD6
:10593600FC901C88E0F8A3E0F9A3E0FAA3E0FB12D0
:105946002A05402D901C88122A6800000000901B32
:1059560037E0FEA3E0FFE48F288E27F526F52575B0
:1059660029FF752AE1752B267D06AF16AE15125155
:1059760068901B55E06403702D7F107E0EFDFC9031
:105986001C80E0F8A3E0F9A3E0FAA3E0FBD3122A17
:10599600054013901C80122A68000000007D04AFA9
:1059A60016AE1512600B901B55E06401702D7F102A
:1059B6007E0EFDFC901C8CE0F8A3E0F9A3E0FAA3B0
:1059C600E0FBD3122A054013901C8C122A680000B3
:1059D60000007D07AF16AE1512600BC3901B3AE0B0
:1059E60094E0901B39E0942E5047E47F087E07FD33
:1059F600FC901C94E0F8A3E0F9A3E0FAA3E0FB1204
:105A06002A05402D901C94122A6800000000901B65
:105A160039E0FEA3E0FFE48F288E27F526F52575ED
:105A260029FF752AE1752B2A7D10AF16AE15125186
:105A360068C3901B40E09488901B3FE09413502667
:105A4600901C98E0700804F0E4A3F0FF8015901C09
:105A560099E0D3940274809480400BE4F0901C98F3
:105A6600F07F0112CFA6228E2A8F2B8D2C8B2D78BC
:105A7600AE7C1B7D017BFF7AE179637E007F03129A
:105A860026D5E4F52FE52E75F013A4245EF582E401
:105A9600341BF583E0FCA3E0FDA3E0FEA3E0FF12C8
:105AA6002ADB5AB20000258000005B2DE52E75F03A
:105AB60013A4245EF582E4341BF583E0F8A3E0F931
:105AC600A3E0FAA3E0FB7F807E967D987C001229F6
:105AD6004FE47BFAFAF9F812294FE47B02FAF9F857
:105AE600D3122A054008E47F02FEFDFC802EE52E37
:105AF60075F013A4245EF582E4341BF583E0F8A365
:105B0600E0F9A3E0FAA3E0FB7F807E967D987C0017
:105B160012294FE47BFAFAF9F812294FEF240AF515
:105B260031E43EF5308074E52E75F013A4245EF55D
:105B360082E4341BF583E0F8A3E0F9A3E0FAA3E0DE
:105B4600FB7F807E967D987C0012294FE47BFAFAD3
:105B5600F9F812294FE47B02FAF9F8D3122A054024
:105B660008E47F02FEFDFC802EE52E75F013A424CA
:105B76005EF582E4341BF583E0F8A3E0F9A3E0FACE
:105B8600A3E0FB7F807E967D987C0012294FE47B04
:105B9600FAFAF9F812294F8E308F3112D19CE52E80
:105BA60075F013A4245AF582E4341BF583E0FCA3B4
:105BB600E0FDA3E0FEA3E4FFE4FBFAF9F8C3122A32
:105BC60005704AE52E75F013A4245AF582E4341BB9
:105BD600F583A3A3A3E0FBEB452DFFE4901BB1EFF8
:105BE600F0E52E75F013A4245EF582E4341BF583EC
:105BF600E0FCA3E0FDA3E0FEA3E0FF7B407A427950
:105C06000F7800C3122A05901BB1025CA8E52E7519
:105C1600F013A4245AF582E4341BF583A3A3E0FE13
:105C2600A3E4FFE4FDFC7808122A16901BB1EFF0FE
:105C3600E52E75F013A4245AF582E4341BF583A3EC
:105C4600A3A3E0FFE4901BB2EFF0E52C6031A3E5DF
:105C56002DF07E1B7FB17D037C0012CC37901BB4E8
:105C6600EFF0901BB1E0FF12D0D8901BB2E0FF120C
:105C7600D0D8901BB3E0FF12D0D8901BB480237EFF
:105C86001B7FB17D027C0012CC37901BB3EFF090E6
:105C96001BB1E0FF12D0D8901BB2E0FF12D0D89013
:105CA6001BB3E0FF12D0D812D135AB2BAA2AAD31E7
:105CB600AC307F647E0012BEFF901BAFEEF0A3EF08
:105CC600F04E7007901BAE7403806DE52E75F013D1
:105CD600A4245AF582E4341BF583E0FCA3E0FDA37B
:105CE600E0FEA3E4FFE4FBFAF9F8C3122A05702CE0
:105CF600F52FFFFED3901BB0E09F901BAFE09E40B8
:105D060016E52B2FF582E52A3EF583E0252FF52FA4
:105D16000FBF00010E80DD532F7F8011901BAFE077
:105D2600FCA3E0FDAF2BAE2A12CC378F2FE52F7FD9
:105D3600017001FF901BAEEFF07B017A1B79AE225A
:105D4600E4901BA0F0A3F0901BA0E475F0011228CC
:105D560049FE74A325F0F58274093EF583E070E7E9
:105D6600901BA0E0FEA3E024A3F974093EFA7B0190
:105D7600128B5C901BA2122A5CE4FFFEFDFC901BBA
:105D8600A2E0F8A3E0F9A3E0FAA3E0FBC3122A0518
:105D9600704A12C48A7E097FA37D007C0412CC3728
:105DA6008F2212D0FEE4901BA0F0A3F0901BA0E07F
:105DB600FEA3E0FFC3EE9404501F74A32FF5827474
:105DC600093EF583E0FF12D117901BA1E004F070A5
:105DD600DB901BA0E004F080D3026005E47B02FAAE
:105DE600F9F8901BA2E0FCA3E0FDA3E0FEA3E0FF10
:105DF60012294FEF24FFFFEE34FFFEED34FFFDECDA
:105E060034FFFC901BA6122A5C90096CE0640170BA
:105E160038FF7E08FDFC901BA6E0F8A3E0F9A3E09E
:105E2600FAA3E0FBD3122A05401F901BA6E0FCA3B1
:105E3600E0FDA3E0FEA3E02470FFE43EFEE43DFDAA
:105E4600E43CFC901BA6122A5C901BA6E0FCA3E097
:105E5600FDA3E0FEA3E0FF12AEC4EF600302600AFA
:105E6600901BA6E0FCA3E0FDA3E0FEA3E0FF122A40
:105E7600DB5E8D000000005ED3000008005F0A00B4
:105E860000089000005F10E4901BA0F0A3F0901BA8
:105E9600A0E0FEA3E0FF2400F58274003EF583E057
:105EA600FD74A32FF58274093EF583EDF0901BA1D6
:105EB600E004F07006901BA0E004F0901BA0E0B494
:105EC60004CCA3E0B400C712CB58025FC1E4901B18
:105ED600A0F0A3F0901BA0E0FEA3E0FFC3EE9404A5
:105EE600501C74A32FF58274093EF583E4F0901BD1
:105EF600A1E004F070DE901BA0E004F080D6129CB6
:105F0600B1025FC112CB28025FC1901BA2A3A3A35B
:105F1600E05401FFE4FEFDFCFBFAF9F8C3122A0582
:105F26007041901BA0F0A3F0901BA0E0FEA3E0FF41
:105F36002400F58274003EF583E0FD74A32FF582FC
:105F460074093EF583EDF0901BA1E004F070069015
:105F56001BA0E004F0901BA0E0B404CCA3E0B400C6
:105F6600C78058901BA2A3A3A3E05401FFE4FEFD43
:105F7600FCFBFAF9F8C3122A056040E4901BA0F076
:105F8600A3F0901BA0E0FEA3E0FF2400F5827404BA
:105F96003EF583E0FD74A32FF58274093EF583ED8B
:105FA600F0901BA1E004F07006901BA0E004F090B6
:105FB6001BA0E0B404CCA3E0B400C77E097FA37D98
:105FC600007C0412CC378F2212D0FEE4901BA0F086
:105FD600A3F0901BA0E0FEA3E0FFC3EE9404501FC5
:105FE60074A32FF58274093EF583E0FF12D1179052
:105FF6001BA1E004F070DB901BA0E004F080D3AF9F
:106006002212D117228E2A8F2B8D2C129B68901C60
:1060160014122A5CAF2C1275788B328A3389347F3E
:10602600007E407D017C00901C14E0F8A3E0F9A3FB
:10603600E0FAA3E0FBC3122A0540030262C07E0019
:106046007F407D007B017A1B79D4122CB0852B8290
:10605600852A83A3A3A3E0C3940A74809480501274
:106066007538FF7539D2753A877B017A1B79D41258
:10607600BF57852B82852A83A3A3A3E0FF7E007BDF
:10608600007A00792D127BB5753800753900753A9E
:106096002D7B017A1B79D412BF577538FF7539D21B
:1060A600753A897B017A1B79D412BF57852B828575
:1060B6002A83A3E0C3940A7480948050127538FF33
:1060C6007539D2753A877B017A1B79D412BF578509
:1060D6002B82852A83A3E0FF7E007B007A00792D40
:1060E600127BB5753800753900753A2D7B017A1B20
:1060F60079D412BF577538FF7539D2753A897B0145
:106106007A1B79D412BF57852B82852A83E0FF7EBE
:10611600007B007A00792D127BB575380075390041
:10612600753A2D7B017A1B79D412BF577538FF75E6
:1061360039D2753A8B7B017A1B79D412BF57E52B7E
:106146002404F582E4352AF583E0C3940A74809426
:106156008050127538FF7539D2753A877B017A1BE4
:1061660079D412BF57E52B2404F582E4352AF5834A
:10617600E0FF7E007B007A00792D127BB575380032
:10618600753900753A2D7B017A1B79D412BF577584
:1061960038FF7539D2753A8D7B017A1B79D412BFD7
:1061A60057E52B2405F582E4352AF583E0C3940AE6
:1061B6007480948050127538FF7539D2753A877B92
:1061C600017A1B79D412BF57E52B2405F582E435F5
:1061D6002AF583E0FF7E007B007A00792D127BB5DD
:1061E600753800753900753A2D7B017A1B79D41202
:1061F600BF577538FF7539D2753A8D7B017A1B7991
:10620600D412BF57E52B2406F582E4352AF583E040
:10621600C3940A7480948050127538FF7539D2750C
:106226003A877B017A1B79D412BF57E52B2406F5F2
:1062360082E4352AF583E0FF7E007B007A00792D23
:10624600127BB5753800753900753A2D7B017A1BBE
:1062560079D412BF57E5344533453260128532385A
:1062660085333985343A7B017A1B79D412BF577B43
:10627600017A1B79D412CFBCC3EF943EEE94005042
:106286001474D42FF582741B3EF5837420F00FBF6F
:1062960000010E80E3901C12740DF0A3740AF0A3A3
:1062A600E0FCA3E0FDA3E0FEA3E0FF7B017A1B79FF
:1062B600D4753C00753D4012B77322E55A65597096
:1062C60003026506AF59055974002FF582E43400C0
:1062D600F583E0F522E5556003026488E52224F69D
:1062E600606424FD70030263F624ED604024F560CB
:1062F6001D24F1700302640624FD606924CA6058F7
:10630600246B600302646EE4F54FF55080AD0550D2
:10631600E550AE4F7002054F1424A3F58274093E72
:10632600F583E4F0F553F554755501808E0550E577
:1063360050AE4F7002054F1424A3F58274093EF542
:1063460083E4F00262C174A32550F5827409354FC7
:10635600F583E4F0F555FF220550E550AE4F700287
:10636600054F0264780550E550AE4F7002054F1494
:1063760024A3F58274093EF583E4F075550175563C
:1063860001F551F552F553F55474A32552F582746F
:10639600093551F583E0600A0552E55270EB055167
:1063A60080E70552E5527002055174A32552F58225
:1063B60074093551F583E0600A0552E55270EB0524
:1063C6005180E70552E5527002055174A32552F536
:1063D6008274093551F583E0600A0552E55270EB87
:1063E600055180E70552E5527002055124A38066E7
:1063F60074A32550F5827409354FF583E4F0FF2226
:106406000550E550AE4F7002054F1424A3F5827473
:10641600093EF583E4F0755501755601F551F552BF
:10642600F553F5540552E552AE5170020551142448
:10643600A3F58274093EF583E070E90552E552AE94
:1064460051700205511424A3F58274093EF583E0C8
:1064560070E974A32552F974093551FA7B01129635
:10646600C28E578F580262C10550E550AE4F70027A
:10647600054F1424A3F58274093EF583E522F00244
:1064860062C1E55660340554E55470020553055063
:10649600E550AE4F7002054F1424A3F58274093EF1
:1064A600F583E522F0C3E5549558E5539557500317
:1064B6000262C1E4F555F55680300554E554700284
:1064C60005530550E550AE4F7002054F1424A3F551
:1064D6008274093EF583E522F0C3E5549401E55341
:1064E600940450030262C1E4F55574A32550F58265
:1064F6007409354FF583E522F0E4F54FF550FF2298
:106506007F0122E4901BA0F0A3F0901BA0E0FEA365
:10651600E024A3F58274093EF583E06010901BA188
:10652600E004F070E5901BA0E004F080DD901BA075
:10653600E475F001122849FE74A325F0F58274096A
:106546003EF583742BF0901BA0E0FEA3E024A3F598
:106556008274093EAF82FE7D017C0412CC37901B0B
:10656600A2EFF0901BA0E0FEA3E024A3F58274093D
:106576003EF583E0900987F0E4901BA3F09009872D
:10658600E0FF901BA3E0FEC39F400302670DEE757C
:10659600F010A424A4F9740935F0FA7B01901BA02D
:1065A600E0FEA3E029F9EA3EFA7D0412BB0D901B3A
:1065B600A3E0FB75F013A4245AF582E4341BF5839B
:1065C600122A5CEB75F010A424A8F9740935F0FAC8
:1065D6007B01901BA0E0FEA3E029F9EA3EFA7D04C8
:1065E60012BB0D901BA3E0FB75F013A4245EF5828D
:1065F600E4341BF583122A5CEB75F010A424ACF985
:10660600740935F0FA7B01901BA0E0FEA3E029F99E
:10661600EA3EFA7D0212BB0D901BA3E0FD75F01356
:10662600A42462F582E4341BF583EEF0A3EFF09028
:106636001BA0E0FEA3E0FF75F010EDA42FF582E5A8
:10664600F03EF583E58224AEF582E5833409F583D1
:10665600E0FFED75F013A42464F582E4341BF583A2
:10666600EFF0ED75F010A424AFF9740935F0FA7B5C
:1066760001901BA0E0FEA3E029F9EA3EFA7D021292
:10668600BB0D901BA3E0FD7A002FFFEA3EFEED75E1
:10669600F013A42467F582E4341BF583EEF0A3EF30
:1066A600F0901BA3E0FF75F013A4246BF582E4348D
:1066B6001BF5837401F0901BA0E0FCA3E0901B691E
:1066C60075F013122A99EC75F013A42583F583E46B
:1066D600F0A3F0EF75F013A42462F582E4341BF501
:1066E60083E0FEA3E04E7016901BA3E075F013A4A2
:1066F6002462F582E4341BF583E4F0A304F0901BD6
:10670600A3E004F0026583E4900982F0A3F0900907
:1067160085740FF0A374FFF002D081E4901BA0F003
:10672600A3F0901BA0E475F001122849FE74A3257E
:10673600F0F58274093EF583E070E7901BA0E475DE
:10674600F001122849FE74A325F0F58274093EF57E
:1067560083E070E7901BA075F001122849FE74A330
:1067660025F0F58274093EF583E075F00AA4FF90E2
:106776001BA0E475F001122849FC74A325F0F582EC
:1067860074093CF583E02F24F0900988F0901BA053
:10679600E475F001122849FE74A325F0F582740908
:1067A6003EF583E075F00AA4FF901BA0E475F001A6
:1067B600122849FC74A325F0F58274093CF583E0A0
:1067C6002F24F0900989F0901BA0E475F00112289F
:1067D60049FE74A325F0F58274093EF583E075F051
:1067E6000AA4FF901BA0E475F001122849FC74A3CB
:1067F60025F0F58274093CF583E02F24F090098A90
:10680600F0901BA0E475F001122849FE74A325F050
:10681600F58274093EF583E075F00AA4FF901BA08B
:10682600E475F001122849FC74A325F0F582740979
:106836003CF583E02F24F090098BF0901BA0E475C3
:10684600F001122849FE74A325F0F58274093EF57D
:1068560083E075F00AA4FF901BA0E475F0011228EE
:1068660049FC74A325F0F58274093CF583E02F24D6
:10687600F090098CF0901BA0E475F001122849FEF7
:1068860074A325F0F58274093EF583E075F00AA439
:10689600FF901BA0E475F001122849FC74A325F0B3
:1068A600F58274093CF583E02F24F090098DF09071
:1068B6001BA0E475F001122849FE74A325F0F582A9
:1068C60074093EF583E075F00AA4FF901BA0E475F9
:1068D600F001122849FC74A325F0F58274093CF5F1
:1068E60083E02F24F090098EF090098CE0FFA3E05E
:1068F600FDA3E0FB12C857900988E0FFA3E0FD90D6
:10690600098BE0FB90098AE0F52512C56A12CF1CB7
:1069160012D153EF6401700302D08112D09322E4A6
:10692600901BA0F0A3F0901BA0E475F0011228497B
:10693600FE74A325F0F58274093EF583E070E790B6
:106946001BA0E475F001122849FE74A325F0F58218
:1069560074093EF583E070E7901BA075F0011228DC
:1069660049FE74A325F0F58274093EF583E075F0BF
:106976000AA4FF901BA0E475F001122849FC74A339
:1069860025F0F58274093CF583E02F24F090097810
:10699600F0901BA0E475F001122849FE74A325F0BF
:1069A600F58274093EF583E075F00AA4FF901BA0FA
:1069B600E475F001122849FC74A325F0F5827409E8
:1069C6003CF583E02F24F0900979F0901BA0E47544
:1069D600F001122849FE74A325F0F58274093EF5EC
:1069E60083E075F00AA4FF901BA0E475F00112285D
:1069F60049FC74A325F0F58274093CF583E02F2445
:106A0600F090097AF0901BA0E475F001122849FE77
:106A160074A325F0F58274093EF583E075F00AA4A7
:106A2600FF901BA0E475F001122849FC74A325F021
:106A3600F58274093CF583E02F24F090097BF090F1
:106A46001BA0E475F001122849FE74A325F0F58217
:106A560074093EF583E075F00AA4FF901BA0E47567
:106A6600F001122849FC74A325F0F58274093CF55F
:106A760083E02F24F090097CF0901BA0E475F001D0
:106A8600122849FE74A325F0F58274093EF583E0C9
:106A960075F00AA4FF901BA0E475F001122849FCCA
:106AA60074A325F0F58274093CF583E02F24F09059
:106AB600097DF0901BA0E475F001122849FE74A32D
:106AC60025F0F58274093EF583E075F00AA4FF907F
:106AD6001BA0E475F001122849FC74A325F0F58289
:106AE60074093CF583E02F24F090097EF090097C30
:106AF600E0FFA3E0FDA3E0FB12CA65900978E0FF82
:106B0600A3E0FD90097BE0FB90097AE0F52512C72A
:106B1600A102D081E4901BA0F0A3F0901BA0E0FEA0
:106B2600A3E024A3F58274093EF583E06010901B70
:106B3600A1E004F070E5901BA0E004F080DD901B5E
:106B4600A1E004F07006901BA0E004F0901BA0E00A
:106B5600FEA3E024A3F58274093EF583E064316068
:106B660003026C5D901BA1E004F07006901BA0E090
:106B760004F0E47FC0FEFDFC901B5AE0F8A3E0F9A8
:106B8600A3E0FAA3E0FBC3122A05601AE47FC0FE65
:106B9600FDFC901B6DE0F8A3E0F9A3E0FAA3E0FB8F
:106BA600C3122A05704A901BA0E0FEA3E024A3F9B5
:106BB60074093EFA7B011296C27C007D0A1227FDFB
:106BC600EF25E025E0540C900982F0901BA0E0FE32
:106BD600A3E024A3F974093EFA7B011296C27C0055
:106BE6007D0A1227FDAF05EF25E025E0540C8060F5
:106BF600E47FA17E16FDFC901B5AE0F8A3E0F9A302
:106C0600E0FAA3E0FBC3122A056003026CF0901BB6
:106C1600A0E0FEA3E024A3F974093EFA7B011296D4
:106C2600C27C007D0A1227FDEFC45470900982F0E1
:106C3600901BA0E0FEA3E024A3F974093EFA7B01B1
:106C46001296C27C007D0A1227FDAF05EFC4547070
:106C5600900983F0026CF0901BA0E0FEA3E024A351
:106C6600F58274093EF583E0B43225901BA1E00459
:106C7600F07006901BA0E004F0901BA0E0FEA3E0DD
:106C860024A3F58274093EF583E0900984F0805AC6
:106C9600901BA0E0FEA3E024A3F58274093EF583D1
:106CA600E064337048901BA1E004F07006901BA0CE
:106CB600E004F0901BA0E0FEA3E024A3F582740993
:106CC6003EF583E0FFB4300790098274BC8009EF7B
:106CD600B4310A90098274BDF0A3F0800DEFB4328E
:106CE6000990098274BCF0A304F012D08122E490CA
:106CF6001BA0F0A3F0901BA0E475F001122849FE3A
:106D060074A325F0F58274093EF583E070E7901BC5
:106D1600A0E0FEA3E024A3F974093EFA7B01128BDE
:106D26005C901B5A122A5C901BA0E0FEA3E024A3F1
:106D3600F58274093EF583E06010901BA1E004F033
:106D460070E5901BA0E004F080DD901BA1E004F04C
:106D56007006901BA0E004F0901BA0E0FEA3E024C8
:106D6600A3F974093EFA7B01128B5C901B5E122A12
:106D76005C901BA0E0FEA3E024A3F58274093EF517
:106D860083E06010901BA1E004F070E5901BA0E08A
:106D960004F080DD901BA1E004F07006901BA0E0DB
:106DA60004F0901BA0E0FEA3E024A3F974093EFAC8
:106DB6007B01128B5C901B62EEF0A3EFF0901BA0A0
:106DC600E0FEA3E024A3F58274093EF583E060109B
:106DD600901BA1E004F070E5901BA0E004F080DDBC
:106DE600900985740FF0A374FFF0901B5EE0FCA37E
:106DF600E0FDA3E0FEA3E0F52F8E2E8D2D8C2C7FDB
:106E0600007E367D6E7C0112C7E37E097FA3E4F522
:106E16002EFBFD125A6D78A37C1B7D017E007F033D
:106E26001226D512D0FE901BA4A3E0FF12D1179014
:106E36001BA4E0FF12D117901BA274FFF0901BA4B5
:106E4600A3E0FD7FFF12D247901BA2EFF0901BA498
:106E5600E0FD12D247901BA2EFF0E4901BA0F0A336
:106E6600F0901BA4E0FEA3E0FF901BA0E0FCA3E0D3
:106E7600FDC39FEC9E503E74A32DF58274093CF52C
:106E860083E0FF12D117901BA2E0FF901BA0E0FC4D
:106E9600A3E024A3F58274093CF583E0FD12D247F2
:106EA600901BA2EFF0901BA1E004F070B4901BA021
:106EB600E004F080AC901BA2E0FF02D1177F037EB6
:106EC6000012CA33C3E51A94085003027036E51B54
:106ED6007004E51A64087033AF11AE10AD0FAC0E36
:106EE600F52EF52F12851AEF601E851128851027BD
:106EF600850F26850E257529FF752AE1752B2E7DB2
:106F060016AF16AE1512516802700E900981E0C3D5
:106F16009402748094805079AF11AE10AD0FAC0E10
:106F2600E4F52EF52F12851AEF601E8511288510BF
:106F360027850F26850E257529FF752AE1752B2EC7
:106F46007D16AF16AE15125168E5112401F511E450
:106F56003510F510E4350FF50FE4350EF50EAF11CB
:106F6600AE10AD0FFC752608752700128603EF607C
:106F76001E851128851027850F26850E257529FF64
:106F8600752AE1752B2E7D16AF16AE151251688047
:106F960077AF11AE10AD0FAC0EE4F52EF52F1285BE
:106FA6001AEF601E851128851027850F26850E2568
:106FB6007529FF752AE1752B2E7D16AF16AE1512B3
:106FC6005168E5112401F511E43510F510E4350F8B
:106FD600F50FE4350EF50EAF11AE10AD0FFC752EA4
:106FE60008752F0012851AEF601E85112885102757
:106FF600850F26850E257529FF752AE1752B2E7DB1
:1070060016AF16AE15125168E5112401F511E435D7
:1070160010F510E4350FF50FE4350EF50EE4F51A0C
:10702600F51B7E117F94FD7B017A0979A3122CB0A2
:1070360012B707EF64037008901C9CE004F080050B
:10704600E4901C9CF0901C9CE0D3940A748094807D
:10705600400C7D1EAF16AE1512600B123D167FFB5F
:107066007E457D1E7C00AB11AA10A90FA80EC31287
:107076002A05400C7D0BAF16AE1512600B123D169D
:1070860022901B47E0FCA3E0FDA3E0FEA3E0240161
:10709600FFE43EFEE43DFDE43CFC901B47122A5C07
:1070A600901BA2122A6800000010900987E0700663
:1070B6009009B374FFF0E4901BA0F0A3F090098749
:1070C600E0FFC3901BA1E09F901BA0E0940040034B
:1070D6000271B9E0FEA3E0FF901B6775F013122A58
:1070E60099EE75F013A42583F583E0FCA3E024B3A1
:1070F600F58274093CF583E5822FF582E5833EAF80
:1071060082F5228F23901BA0A3E0901B5E75F013DF
:10711600122A99EE75F013A42583F583E0FCA3E00B
:10712600FDA3E0FEA3E0F52F8E2E8D2D8C2C7F0087
:107136007E367D6E7C0112C7E3901BA0E0FCA3E0C7
:10714600FD901B6475F013122A99EC75F013A425B3
:1071560083F583E0D39401748094805056AF23AEB8
:107166002212C99B78A67C1B7D017E007F03122616
:10717600D5901BA2E0F8A3E0F9A3E0FAA3E0FB9008
:107186001BA8E02401FF901BA7E03400FEE4FCFDF1
:10719600EB2FFFEA3EFEED39FDEC38FC901BA21208
:1071A6002A5C901BA1E004F07006901BA0E004F09E
:1071B6000270C37E097FA3127829E47F3FFEFDFC9F
:1071C600901BA2E0F8A3E0F9A3E0FAA3E0FBD31238
:1071D6002A057E0040047F7F80027F3F901BA91214
:1071E600D0F9E4901BA0F0A3F0901BA9E0FEA3E069
:1071F600FF901BA0E0FCA3E0FDC39FEC9E501F7414
:10720600A32DF58274093CF583E0FF12D117901B7C
:10721600A1E004F070D3901BA0E004F080CB7E09BF
:107226007FA3901BA9E0FCA3E0FD12CC3712D11777
:10723600901BA9E0FEA3E0FF7D007B017A0979A3FC
:10724600022CB012CC8A901B41EEF0A3EFF0E4F5CD
:1072560027C3E527940374809480501912202EE5E5
:107266002725E024CEF582E4341BF583EEF0A3EF68
:10727600F0052780DC901BD0E0FEA3E0FF901BCF3B
:10728600E02FFF901BCEE03EFE901BD3E02FFF9039
:107296001BD2E03EFE7C007D031227A8901B37EE32
:1072A600F0A3EFF07F1612B980EF24C0FDEE34F99B
:1072B600FC1223A9E4FBFA79C0783F1221FE1223BF
:1072C600E2901B4BEEF0A3EFF07F1712B980EF248C
:1072D600C0FDEE34F9FC1223A9E4FBFA79C0783F2D
:1072E6001221FE1223E2901B4DEEF0A3EFF07F1366
:1072F60012B980EE3395E0FDFCE47B0BFAF9F81247
:1073060028C4901B39EEF0A3EFF07F1212B980EE7D
:107316003395E0FDFCE47B0BFAF9F81228C4901BC8
:107326003BEEF0A3EFF07F1512B980EE3395E0FD4A
:10733600FCE47B0BFAF9F81228C4901B3DEEF0A38F
:10734600EFF07F1412B980EE3395E0FDFCE47B0B81
:10735600FAF9F81228C4901B3FEEF0A3EFF07F3045
:1073660012B980901BCCEEF0A3EFF0FDAC06EC1248
:1073760023A97B337AB3796078C412210D7BB87A5E
:107386001E795578401223071223E2901BCCEEF0AB
:10739600A3EFF0901BCCE0FCA3E0FD901B45ECF0C6
:1073A600A3EDF0EC1223A97B3D7A0A7937784012D7
:1073B60021FEE4FBFA7942784412210D7B007AF033
:1073C600797F78451221FEE4FBFA79167845122377
:1073D600071223E2901BCCEEF0A3EFF0901B43EED6
:1073E600F0A3EFF012899FEF600F12899FEF6009FB
:1073F6007D1FAF16AE1512600B22E4901BA0F0A302
:10740600F0901BA0E475F001122849FE74A325F044
:10741600F58274093EF583E070E7901BA0E0FEA3B9
:10742600E024A3F974093EA801FC7D017BFF7AD60E
:10743600798D122C93EF3395E04F7006128DE6028C
:107446007523901BA0E0FEA3E024A3F974093EA8CF
:1074560001FC7D017BFF7AD67994122C93EF33954C
:10746600E04F700612C25A027523901BA0E0FEA3DD
:10747600E024A3F974093EA801FC7D017BFF7AD6BE
:10748600799A122C93EF3395E04F700612C20602DA
:107496007523901BA0E0FEA3E024A3F974093EA87F
:1074A60001FC7D017BFF7AD679A0122C93EF3395F0
:1074B600E04F7071901BA0E475F001122849FE742C
:1074C600A325F0F58274093EF583E070E7901BA0D2
:1074D600E0FEA3E024A3F974093EFA7B011296C2EA
:1074E600901BA2EEF0A3EFF0901BA0E475F0011242
:1074F6002849FE74A325F0F58274093EF583E070F1
:10750600E7901BA0E0FEA3E024A3F58274093EAF3A
:1075160082FE901BA2E0FCA3E0FD12A8AC901BA487
:10752600EEF0A3EFF0901BA4E07002A3E0603F1220
:10753600D0FEE4901BA0F0A3F0901BA4E0FEA3E015
:10754600FF901BA0E0FCA3E0FDC39FEC9E502274BD
:10755600002DF58274003CF583E0FF12D117901BD5
:10756600A1E004F070D3901BA0E004F080CB12D011
:107576009322EFB4210040030276CB907588F82859
:1075860028730275EB0275F20275F902760002762F
:107596000702760E02761502761C02762302762AFA
:1075A60002763102763802763F0276CB02764602C2
:1075B600764D02765402765B027662027669027630
:1075C6007002767702767E02768502768C02769354
:1075D60002769A0276A10276A80276AF0276B60203
:1075E60076BD0276C47BFF7AD2798F227BFF7AD270
:1075F60079AB227BFF7AD279C8227BFF7AD279E8EF
:10760600227BFF7AD3790A227BFF7AD37926227BE3
:10761600FF7AD37942227BFF7AD3795E227BFF7A87
:10762600D37983227BFF7AD579A9227BFF7AD37916
:10763600B2227BFF7AD379D9227BFF7AD379F122E2
:107646007BFF7AD379FF227BFF7AD4791E227BFFD8
:107656007AD4793D227BFF7AD4795F227BFF7AD573
:1076660079C9227BFF7AD47980227BFF7AD479B9D3
:10767600227BFF7AD47998227BFF7AD479E2227B27
:10768600FF7AD57906227BFF7AD57929227BFF7A84
:10769600D57952227BFF7AD57964227BFF7AD57918
:1076A60088227BFF7AD579EA227BFF7AD679072270
:1076B6007BFF7AD6792D227BFF7AD6794B227BFF08
:1076C6007AD67967227BFF7AD379A0228F408E3FC4
:1076D6008D3E8C3D85A74575A710AB44AA43A942AC
:1076E600A841AF40AE3FAD3EAC3D12294FE47B0210
:1076F600FAF9F812294FE47BFFFAF9F8D3122A05B2
:10770600402AAB44AA43A942A841AF40AE3FAD3E92
:10771600AC3D12294FE47B02FAF9F812294F1229DF
:10772600E18F8D538EF4438E08027816AB44AA433C
:10773600A942A841AF40AE3FAD3EAC3D12294FE451
:107746007B02FAF9F812294FE47B04FAF9F81229B8
:107756004FE47BFFFAF9F8D3122A054033AB44AA6B
:1077660043A942A841AF40AE3FAD3EAC3D12294FC2
:10777600E47B02FAF9F812294FE47B04FAF9F812CD
:10778600294F1229E18F8D538EF4438E010278160C
:10779600AB44AA43A942A841AF40AE3FAD3EAC3D83
:1077A60012294FE47B02FAF9F812294FE47B0CFA0E
:1077B600F9F812294FE47BFFFAF9F8D3122A05AB40
:1077C60044AA43A942A841AF40AE3FAD3EAC3D40BE
:1077D6001F12294FE47B02FAF9F812294FE47B0CB9
:1077E600FAF9F812294F1229E18F8D538EF4802071
:1077F60012294FE47B02FAF9F812294FE47B30FA9A
:10780600F9F812294F1229E18F8D538EF4438E0217
:10781600858D8B53890F438920D28ED29DD29C852C
:1078260045A7228E278F28901B47A3A3A3E0852870
:1078360082852783F0901B47E0FCA3E0FDA3E0FED2
:10784600A3E0FF7808122A16852882852783A3EFEE
:10785600F0901B4BE0FEA3E0852882852783A3A337
:10786600F0EEFF852882852783A3A3A3EFF0901B64
:107876004DE0FEA3E0FDE5282404F582E43527F576
:1078860083EDF0EEFFE5282405F582E43527F58340
:10789600EFF0901B51E0FEA3E0FF12ABD0901B4F20
:1078A600EEF0A3EFF0E4A3F0A3F0901B4FE0FEA3ED
:1078B600E0FDE5282406F582E43527F583EDF0EEB4
:1078C600FFE5282407F582E43527F583EFF0901BC2
:1078D60037E0FEA3E0FDE5282408F582E43527F528
:1078E60083EDF0EEFFE5282409F582E43527F583DC
:1078F600EFF0901B39E0FEA3E0FDE528240AF582AF
:10790600E43527F583EDF0EEFFE528240BF582E458
:107916003527F583EFF0901B43E0FEA3E0FDE52855
:10792600240CF582E43527F583EDF0EEFFE52824F7
:107936000DF582E43527F583EFF0901B3BE0FEA3BF
:10794600E0FDE528240EF582E43527F583EDF0EE1B
:10795600FFE528240FF582E43527F583EFF02212A0
:10796600D1F612CDC512D27E12CC6112D1441220AC
:107976002612CC0C7F0112200612CF35C297E49056
:10798600096AF090096CF09009687403F090096731
:107996007409F0127F1E90096F122A5C90096AE042
:1079A600C394067480948050147525017526097554
:1079B60027647B017A1B793712910180DF127249A5
:1079C60012D15390096BEFF064017012900966E0D2
:1079D6006402600512206E800812B312800312B88A
:1079E60049900968E0147003027A7A14601A24FD3B
:1079F600605224FE7003027A83147003027A89248B
:107A06000570DE12B03A80D912A675128A7EEF4E44
:107A160060CF7F0112200612D284901B53E0FEA392
:107A2600E0FFE48F288E27F526F5257529FF752AB0
:107A3600E1752B667D08AF16AE15125168E4FF128C
:107A46002006809D12903E128A7EEF4E6093901B18
:107A560053E0FEA3E0FFE48F288E27F526F5257573
:107A660029FF752AE1752B667D08AF16AE151251F2
:107A7600680279E712AFBE128A7E0279E712B4DE97
:107A86000279E712CD030279E78F328E318D308C81
:107A96002F8B338A348935901BF1740AF0E4901BDE
:107AA600EFF0901BF1E0FF901BEFE0C39F505BE40B
:107AB6007B0AFAF9F8AF32AE31AD30AC2F12294F4E
:107AC600EB2430FF901BF1E024FFFDE434FFFC9033
:107AD6001BEFE0FBC3ED9BFDEC9400AB33AA34A98E
:107AE600358D82F583EF122786AF32AE31AD30ACDD
:107AF6002FE47B0AFAF9F812294F8F328E318D3036
:107B06008C2F901BEFE004F08098E4901BEFF0AB15
:107B160033AA34A935901BEFE0FFF5827583001276
:107B26002714B43013901BF1E014FEEFC39E5008E7
:107B3600901BEFE004F080D7901BEFE0D394007425
:107B4600809480404AE4A3F0901BEFE0FF901BF185
:107B5600E0C39FFE901BF0E0FDC39E5027ED2FF57E
:107B660082E433F583AB33AA34A935122714FF9088
:107B76001BF0E0F582758300EF122786901BF0E07C
:107B860004F080C4AB33AA34A935901BF08009AB4E
:107B960033AA34A935901BF1E0F582758300E4120F
:107BA6002786901BEFE0FF901BF1E0C39FFF228E1C
:107BB600358F368B378A3889397C007D0A1227FD46
:107BC600900004ED122786AE35AF367C007D0A1292
:107BD60027FD8E358F367C007D0A1227FDAB37AA2E
:107BE60038A939900003ED122786AE35AF367C00F2
:107BF6007D0A1227FD8E358F367C007D0A1227FD01
:107C0600AB37AA38A939900002ED122786AE35AFF8
:107C1600367C007D0A1227FD8E358F367C007D0A64
:107C26001227FDAB37AA38A939900001ED12278635
:107C3600AE35AF367C007D0A1227FD8E358F367C39
:107C4600007D0A1227FDAB37AA38A939ED12277431
:107C5600E4901C18F0AB37AA38A939901C18E0FF3D
:107C6600F582758300122714FD3395E04D70089058
:107C76001C18E004F080DEEF6405700DAB37AA38FF
:107C8600A9397430122774803FE4901C19F0901CB7
:107C960018E0FFC374059FFEA3E0FDC39E5029EDC7
:107CA6002FF582E433F583AB37AA38A939122714A6
:107CB6002430FF901C19E0F582758300EF122786A9
:107CC600901C19E004F080C6901C18E0FFC37405F0
:107CD6009FFF22901B47E0FCA3E0FDA3E0FEA3E08C
:107CE600FFC007900981E0FBE4FAF9F8D0071229F2
:107CF6004F901B47122A5C74A3251BF58274093525
:107D06001AAF82FE127829901B47E0F8A3E0F9A388
:107D1600E0FAA3E0FB900981E0FFE4FCFDFE1228F7
:107D2600C4901B47122A5C900986E024EEFF900956
:107D360085E034FFFE74A3251BF5827409351AF518
:107D460083E5822FF582E5833EAF82FE12B91A9053
:107D56000986E024F6FF900985E034FFFE74A3252A
:107D66001BF5827409351AF583E5822FF582E583C2
:107D76003EAF82FE12BAAB900985E0FEA3E0FF7427
:107D860091251BF5827409351AF583E5822FF58254
:107D9600E5833EAF82FE7D107C0012CC37900985CC
:107DA600E0FCA3E0FD251BFBE51A3CFA74A12BF5CC
:107DB6008274093AF583EFF074A3251BF5827409E2
:107DC600351AAF82FEED24FFFDEC34FFFC12CC37F2
:107DD600900985E0FCA3E0FD251BFBE51A3CFA743F
:107DE600A22BF58274093AF583EFF0ED251BF51BFE
:107DF600EC351AF51A221293F0E4901BA0F0A3F0CA
:107E0600901BA0E475F001122849FE74A325F0F535
:107E16008274093EF583E070E7901BA2F0901BA2E6
:107E2600E0C3940874809480505F901BA0E475F0C2
:107E360001122849FE74A325F0F58274093EF583E4
:107E4600E0FF12CEAC901BA3EFF0E0C454F0F0902C
:107E56001BA0E475F001122849FE74A325F0F582F3
:107E660074093EF583E0FF12CEAC901BA3E02FF021
:107E7600E0FF901BA2E02493F582E4341BF583EF28
:107E8600F0901BA2E004F0809412BB6BEF600B1223
:107E9600D0FE7BFF7AD87966807512BD99EF600BAC
:107EA60012D0FE7BFF7AD87979806412AC4F7E04BB
:107EB6007F007D007B017A0D79A3122CB078A37C1C
:107EC600097D017B017A0079007E047F001226D5A8
:107ED6007E097FA37DFE7C0312CC37900DA1EFF0C7
:107EE6007B017A0979A37DFF7C0312C932900DA22A
:107EF600EFF0E4F526F5277F907E08FDFC1286EC70
:107F0600EF700302D08112D0FE7BFF7AD8798712F8
:107F160041F8E4FF12D11722E4F525F524F523F5FF
:107F2600227F3812D1C4901BA0EFF07F3912D1C442
:107F3600901BA1EFF07F3A12D1C4901BA2EFF07F05
:107F46003B12D1C4901BA3EFF07F3C12D1C4901B0F
:107F5600A4EFF07F3D12D1C4901BA5EFF07F3E1237
:107F6600D1C4901BA6EFF07F3F12D1C4901BA7EFA0
:107F7600F07E1B7FA07D037C0012CC37901BA3E014
:107F8600B50731901BA1E0FFE4FCFDFE7808122A3C
:107F960029A804A905AA06AB07901BA0E0FFEB4F92
:107FA600FFEAFEE9FDE8FCC004C005C006C0079074
:107FB6001BA280417E1B7FA47D037C0012CC3790E0
:107FC6001BA7E0B50754901BA5E0FFE4FCFDFE7877
:107FD60008122A29A804A905AA06AB07901BA4E043
:107FE600FFEB4FFFEAFEE9FDE8FCC004C005C00652
:107FF600C007901BA6E0FFE4FCFDFE7810122A29BC
:10800600D003D002D001D000EF4BF525EE4AF5247F
:10801600ED49F523EC48F5228009E4F525F524F52C
:1080260023F522AF25AE24AD23AC222212BCE3EF0A
:1080360060097D09AF16AE1512600B7E117F947D27
:10804600007B017A0979A3122CB078A37C097D0103
:108056007B017A0079007E097F601226D5E4F52E31
:10806600F52F7F807E08FDFC12851A7E117F947D98
:10807600007B017A0979A3122CB078A37C097D01D3
:108086007B017A0079007E097F601226D5E4F52E01
:10809600F52F7F907E08FDFC12851A12D27B8F2960
:1080A6008E288D278C26E47F517E08FDFCAB29AAFD
:1080B60028A927A826C3122A0550037F0422E529EA
:1080C6002470FFE52834F7FEE52734FFFDE5263466
:1080D600FFFCE4FB7A08F9F81228C48F258E248D5C
:1080E600238C227E117F947D007B017A0979A3126D
:1080F6002CB0900A3FE525F0FFAE24AD23AC2278E4
:1081060008122A16A3EFF0AF25AE24AD23AC2278D1
:1081160010122A16A3EFF0AF25AE24AD23AC2278B9
:1081260018122A16A3EFF0E4F52EF52FFF7E08FDB0
:10813600FC12851A7F0022E4901BA0F0A3F0901B8E
:10814600A0E475F001122849FE74A325F0F58274A7
:10815600093EF583E070E7901BA0E0FEA3E024A3B0
:10816600F974093EFA7B01128B5C901BA2122A5C01
:10817600901BA0E475F001122849FE74A325F0F5C2
:108186008274093EF583E070E7901BA0E0FEA3E051
:1081960024A3F974093EFA7B011296C2901BA6EE3F
:1081A600F0A3EFF0901BA0E475F001122849FE74CD
:1081B600A325F0F58274093EF583E070E77E097F1A
:1081C60060FD7B017A007900122CB0E4901BA8F0C8
:1081D600A3F0901BA2E0FCA3E0FDA3E0FEA3E0FF5A
:1081E600901BA0E0F526A3E0F527901BA6E0F52856
:1081F600A3E0F529128C3AEF703812D0FE901BA836
:10820600E0FEA3E02400F58274003EF583E0601DE5
:10821600901BA8E475F001122849FE740025F0F5BC
:108226008274003EF583E0FF12D11780D0E4FF127E
:10823600D117228F458E448D438C4285A747A2AF26
:10824600920085F548C2AFE4F5A7FF7E80FDFCAB42
:1082560045AA44A943A842C3122A05500B8544499E
:1082660085454A53F5CF8076E4FFFE7D01FCAB459C
:10827600AA44A943A842C3122A055020E545F5455C
:10828600E5444480F544E543F543E542F54285443B
:108296004985454A53F5CF43F51080427F007E80DD
:1082A6007D017C00AB45AA44A943A842C3122A0516
:1082B6005020E545F545E5444480F544E543F5435E
:1082C600E542F54285444985454A53F5CF43F520B5
:1082D600800C85444985454A53F5CF43F530E4F58E
:1082E600EF75FFA0FFEFC394FF7480948050030FD7
:1082F60080F3E5FF20E6037F002275EF0275B7A540
:1083060075B7F1438F0175FFA075EF02854A828527
:108316004983E546F0E4F5EF75FF8075EF02538F6C
:10832600FE8548F58547A7A20092AF7F01228F25DB
:108336008E248D238C2285A726A2AF920085F52751
:10834600C2AFE4F5A7FF7E80FDFCAB25AA24A923D6
:10835600A822C3122A05500B85242885252953F502
:10836600CF8076E4FFFE7D01FCAB25AA24A923A8D5
:1083760022C3122A055020E525F525E5244480F57B
:1083860024E523F523E522F522852428852529538E
:10839600F5CF43F51080427F007E807D017C00ABE7
:1083A60025AA24A923A822C3122A055020E525F5CB
:1083B60025E5244480F524E523F523E522F52285E9
:1083C600242885252953F5CF43F520800C852428BC
:1083D60085252953F5CF43F530E4F5EF75FFA0FF6A
:1083E600EFC394FF7480948050030F80F3E5FF2061
:1083F600E6037F002275EF0275B7A575B7F1438FC7
:108406000375FFA075EF02852982852883E4F0F5C0
:10841600EF75FF8075EF02538FFC8527F58526A73C
:10842600A20092AF7F01228B238A248925AB26AA3C
:1084360027A9281226FBFFAB23AA24A9251226FB6F
:10844600FE6F600AEEC39F7F0150027FFF22AB26BC
:10845600AA27A928900001122714FFAB23AA24A952
:1084660025900001122714FE6F600AEEC39F7F015C
:1084760050027FFF22AB26AA27A9289000031227C5
:1084860014FFAB23AA24A925900003122714FE6F1C
:10849600600AEEC39F7F0150027FFF22AB26AA2708
:1084A600A928900004122714FFAB23AA24A925901B
:1084B6000004122714FE6F600AEEC39F7F0150026C
:1084C6007FFF22AB26AA27A928900005122714FFB2
:1084D600AB23AA24A925900005122714FE6F600A73
:1084E600EEC39F7F0150027FFF22AB26AA27A92851
:1084F600900006122714FFAB23AA24A92590000694
:10850600122714FE6F600AEEC39F7F0150027FFFA1
:10851600227F00227536FF7537DD7538158F3C8E44
:108526003B8D3A8C397B017A1C79761241F28F3277
:10853600753A607539E37538167537007F007E36F3
:108546007D6E7C0112C81DE4F530F53174CA253103
:10855600F58274DE3530F583E493FF12D0D8053109
:10856600E53170020530C3940AE530940040DDE43D
:10857600F530F531C3E5319532E5309400501B7482
:10858600762531F582741C3530F583E0FF12D0D89C
:108596000531E53170DE053080DAE4FF12D0D8858A
:1085A6002E30852F31E4252FFFE52E3408FEC3E556
:1085B600319FE5309E501B74A32531F58274093531
:1085C60030F583E0FF12D0D80531E53170D705309C
:1085D60080D37F647E007D007C0012AACCEF701AE7
:1085E60078007C007D017BFF7ADD791C122C93EFED
:1085F6003395E04F7F017004FF227F01227536FF1D
:108606007537DD7538158F3C8E3B8D3A8C397B017D
:108616007A1C79761241F28F2A753A607539E375BC
:1086260038167537007F007E367D6E7C0112C81DB8
:10863600E4F528F52974D42529F58274DE3528F564
:1086460083E493FF12D0D80529E52970020528C3D3
:10865600940BE528940040DDE4F528F529C3E529C7
:10866600952AE5289400501B74762529F582741CFA
:108676003528F583E0FF12D0D80529E52970DE05F7
:108686002880DAE4FF12D0D8852628852729E42514
:1086960027FFE5263408FEC3E5299FE5289E501BE3
:1086A60074A32529F58274093528F583E0FF12D0D5
:1086B600D80529E52970D7052880D37F967E007DC9
:1086C600007C0012AACCEF701A78007C007D017B3A
:1086D600FF7ADD791C122C93EF3395E04F7F017002
:1086E60004FF227F01227536FF7537DD7538158F39
:1086F6003C8E3B8D3A8C397B017A1C79761241F29D
:108706008F2A753A607539E37538167537007F001C
:108716007E367D6E7C0112C81DE4F528F52974CAE3
:108726002529F58274DE3528F583E493FF12D0D827
:108736000529E52970020528C3940AE52894004016
:10874600DDE4F528F529C3E529952AE528940050A6
:108756001B74762529F582741C3528F583E0FF12F3
:10876600D0D80529E52970DE052880DAE4FF12D085
:10877600D8852628852729E42527FFE5263408FEFF
:10878600C3E5299FE5289E501B74A32529F582740D
:10879600093528F583E0FF12D0D80529E52970D7D9
:1087A600052880D37FB87E0B7D007C0012AACCEF13
:1087B600701A78007C007D017BFF7ADD791C122C13
:1087C60093EF3395E04F7F017004FF227F0122E48F
:1087D600901BA0F0A3F0901BA0E475F001122849AD
:1087E600FE74A325F0F58274093EF583E070E790E8
:1087F6001BA0E0FEA3E024A3F974093EFA7B011254
:108806008B5C901BA2122A5C901BA0E475F00112EF
:108816002849FE74A325F0F58274093EF583E070BD
:10882600E7901BA0E0FEA3E024A3F974093EFA7BBF
:10883600011296C2901BA6EEF0A3EFF0901BA0E4E7
:1088460075F001122849FE74A325F0F58274093EDD
:10885600F583E070E77E097F60FD7B017A00790091
:10886600122CB0E4901BA8F0A3F0901BA2E0FCA38E
:10887600E0FDA3E0FEA3E0FF901BA0E0F52EA3E041
:10888600F52F12851AEF700B12D0FE7BFF7AD7797F
:108896000F800912D0FE7BFF7AD7792F901BA2E0BA
:1088A600FCA3E0FDA3E0FEA3E0F5398E388D378CFE
:1088B600361241F822901C9EE004F07006901C9D32
:1088C600E004F0D3901C9EE094E0901C9DE094019F
:1088D600500302899E90096FE0FCA3E0FDA3E0FE31
:1088E600A3E02401FFE43EFEE43DFDE43CFC9009E8
:1088F6006F122A5CE4901C9DF0A3F090096FE0FCD7
:10890600A3E0FDA3E0FEA3E0FF901BA0EFF090091B
:108916006FA3A3A3E07808122A16901BA1EFF0908C
:10892600096FE0FCA3E0FDA3E0FEA3E0FF781012D0
:108936002A16E4901BA2EFF07E1B7FA07D037C002D
:1089460012CC37901BA3EFF0901BA0E0FD7F3812EE
:10895600D1D1901BA1E0FD7F3912D1D1901BA2E0AD
:10896600FD7F3A12D1D1901BA3E0FD7F3B12D1D1FE
:10897600901BA0E0FD7F3C12D1D1901BA1E0FD7FB2
:108986003D12D1D1901BA2E0FD7F3E12D1D1901BAA
:10899600A3E0FD7F3F12D1D1227E1B7FD47C1B7DBD
:1089A600EF12A9377E1B7FD47C1B7DEF12A9C27EF6
:1089B6001B7FDD7C1B7DF812A9377E1B7FDD7C1BB0
:1089C6007DF812A9C27E1B7FE67C1C7D0112A937A9
:1089D6007E1B7FE67C1C7D0112A9C27E1B7FEF7C7D
:1089E6001B7DF812A42BEF700C7FEF7C1C7D01120F
:1089F600A42BEF602178917C097D017B017A1B799C
:108A0600EF7E007F091226D578787C097D017B01EF
:108A16007A1B79D4802D7E1B7FF87C1C7D0112A4E5
:108A26002BEF602878917C097D017B017A1B79F810
:108A36007E007F091226D578787C097D017B017A34
:108A46001B79DD7E007F091226D5802978917C0965
:108A56007D017B017A1C79017E007F091226D5787B
:108A6600787C097D017B017A1B79E67E007F0912FD
:108A760026D57F01227F00227F1812C8C6901BA22E
:108A8600EEF0A3EFF07F1912C8C6901BA4EEF0A378
:108A9600EFF0901BA2E0FCA3E02400FDEC34FAFC0E
:108AA600901BA6F0A3EDF0E42FFFEE34FAA3F0A39B
:108AB600EFF0C3EC648094805015901BA6E0FEA3F3
:108AC600E0FFC3E49FFFE49E901BA6F0A3EFF090A7
:108AD6001BA8E0FEA3E0FFC3EE64809480500DC3A4
:108AE600E49FFFE49E901BA8F0A3EFF0901BA8E084
:108AF600FEA3E0FF901BA6E0FCA3E0FDD39FEE647F
:108B060080F8EC6480984006AE04AF058000901BA8
:108B1600A0EEF0A3EFF0C3901B52E09F901B51E034
:108B26009E500F901BA0E0FFA3E0901B51CFF0A337
:108B3600EFF0901BA0E0FEA3E0FFC394BFEE94010C
:108B4600401012C75F901B53EEF0A3EFF07E007F3C
:108B56000122E4FEFF228B238A248925AB23AA2443
:108B6600A9251226FBFF12D06E500D74012525F59E
:108B760025E43524F52480E4D200AB23AA24A925D4
:108B86001226FBFF642B6004EFB42D1BAB230525D7
:108B9600E525AA247002052414F91226FB642D602B
:108BA60003D38001C39200E4F529F528F527F526BD
:108BB600AB23AA24A9251226FBFF12D171505CE42F
:108BC6007F0AFEFDFCAB29AA28A927A8261228C4DD
:108BD600C8ECC8EDC0E0EEC0E0EFC0E0AB23AA24CD
:108BE600A9251226FBFF3395E0FEEF24D0FFEE34D5
:108BF600FFFEE4FCFDD0E0FBD0E0FAD0E0F9EB2F7D
:108C0600F529EA3EF528ED39F527EC38F526740105
:108C16002525F525E43524F524809530000AAF296D
:108C2600AE28AD27AC26800BAF29AE28AD27AC26E3
:108C36001229E1228F258E248D238C227536FF750D
:108C460037DD7538158F3C8E3B8D3A8C397B017A32
:108C56001C79761241F28F2C753A607539E37538B6
:108C6600167537007F007E367D6E7C0112C81DE4C6
:108C7600F52AF52B745C252BF58274DE352AF583EF
:108C8600E493FF12D0D8052BE52B7002052AC39476
:108C96000DE52A940040DDAF2512D0D8AF25AE24CD
:108CA600AD23AC227808122A1612D0D8AF25AE24EE
:108CB600AD23AC227810122A1612D0D8AF25AE24D6
:108CC600AD23AC227818122A1612D0D885262A850A
:108CD600272BE5292527FFE5283526FEC3E52B9F0B
:108CE600E52A9E501B74A3252BF5827409352AF5B7
:108CF60083E0FF12D0D8052BE52B7002052A80D21F
:108D06007F647E007D007C0002AACC12A5529009E9
:108D16006412D0F97F6412D117E4FF12D1177F6471
:108D260012D117E4FF12D1177F6412D117E4FF1294
:108D3600D117E4901BA0F0A3F0E4FF12D117901B0B
:108D4600A1E004F07006901BA0E004F0C3901BA104
:108D5600E0940B901BA0E0940040DEE4FF12D117D4
:108D66007F1212D1177F7A12D117E4FF12D117E4BE
:108D7600901BA0F0A3F0901BA0E0FEA3E0FFC3941D
:108D860007EE9400502074072FF58274DA3EF583BF
:108D9600E493FF12D117901BA1E004F070D8901B4A
:108DA600A0E004F080D0E4901BA0F0A3F0E4FF1252
:108DB600D117901BA1E004F07006901BA0E004F010
:108DC600C3901BA1E09410901BA0E0940040DE909D
:108DD6000964A3E0FF12D117900964E0FF02D117DE
:108DE60078A67C1B7D017BFF7ADE79037E007F08F7
:108DF6001226D5E4901BAEF0901BAEE0C39402742D
:108E06008094804003028EAF7E097F607D007B01E7
:108E16007A007900122CB0901BAEE025E025E02404
:108E2600A6F582E4341BF583E0FCA3E0FDA3E0FE97
:108E3600A3E0F53A8E398D388C377F007E367D6E0D
:108E46007C0112C81DE4F522F52374FB2523F58267
:108E560074DD3522F583E493FF12D0D80523E5238C
:108E660070020522C39408E522940040DDE4FF1257
:108E7600D0D87F327E007D007C0012AACCEF702015
:108E8600F522F5230523E523AE22700205221424DC
:108E960000F58274003EF583E070E9AE22AF23222E
:108EA600901BAEE004F0028DFEE4FEFF22753A60F0
:108EB6007539E37538167537007F007E367D6E7C12
:108EC6000112C81DE4F52AF52B7472252BF5827460
:108ED600DD352AF583E493FF12D0D8052BE52B70F8
:108EE60002052AC3940FE52A940040DD7F987E3A56
:108EF6007D007C0012AACCEF706C900002E0FFE4CB
:108F0600FCFDFE7810122A29E4FFFEE4FCA804A961
:108F160005AA06AB07900001E0FE900000E02400E1
:108F2600FFEC3EFEE4FDEB2FFFEA3EFEED39FDECE5
:108F360038FCC004C005C006C007900003E0FFE48B
:108F4600FCFDFE7818122A29E4FFFEFDD003D002AC
:108F5600D001D000EF2BF52FEE3AF52EED39F52D99
:108F6600E83CF52C8006E4FFFEFDFC22AF2FAE2E7A
:108F7600AD2DAC2C22E4901BA0F0A3F0901BA0E436
:108F860075F001122849FE74A325F0F58274093E96
:108F9600F583E070E7901BA0E0FEA3E024A3F9743C
:108FA600093EFA7B01128B5C901BA2122A5CE47BC1
:108FB60002FAF9F8901BA2E0FCA3E0FDA3E0FEA3F1
:108FC600E0FF12294FEF24FFFFEE34FFFEED34FFE2
:108FD600FDEC34FFFC901BA6122A5C901BA6E0FC5D
:108FE600A3E0FDA3E0FEA3E02470FFE43EFEE43D23
:108FF600FDE43CFC901BA6122A5C901BA0E475F0D5
:1090060001122849FE74A325F0F58274093EF58302
:10901600E070E7901BA6E0FCA3E0FDA3E0FEA3E062
:10902600FF901BA0E0F52EA3E0F52F12851AEF7036
:109036000302D08112D09322E5177003029100E457
:10904600F5171288BB901C9BE004F0E0D3941E74C5
:109056008094804002E4F0901C9BE0C31390E133BF
:109066009324FF9297901B47E0FCA3E0FDA3E0FE4C
:10907600A3E02401FFE43EFEE43DFDE43CFC901B3E
:1090860047122A5C900981E0FBE4FAF9F8901B4745
:10909600E0FCA3E0FDA3E0FEA3E0FF12294FAC0035
:1090A600AD01AE02AF03E4FBFAF9F8C3122A05706C
:1090B60014127249125489901B55EFF0127CD91282
:1090C6006EC31257917525017526097527647B01B4
:1090D6007A1B793712910190096AE0D3940674805D
:1090E60094804016E4F0900966E06402600C7D1DF1
:1090F600AF16AE1512600B123D16228B228A2389FB
:1091060024AB25AA26A9279000041227146405700B
:1091160008901CA17404F0801590000A12271460B0
:109126000D90000AE4122786901CA1E004F0901C22
:10913600A1E0C394047480948050030291C2E4F0C9
:10914600AB22AA23A92412C300AB22AA23A92490E6
:10915600000212285FFFAEF090000412285FFDACFB
:10916600F0D39FEC9E4011D3ED9470EC94177F01E1
:1091760040027F038F28801DAB22AA23A9249000DA
:109186000412285FFFAEF090000212285FD39FE51D
:10919600F09E752802AB25AA26A927900002122761
:1091A600146528600F900002E528122786900006B5
:1091B600E40227869000067401122741228F458E0D
:1091C600448D438C4285A746A2AF920085F547C2DF
:1091D600AFE4F5A7FF7E80FDFCAB45AA44A943A8F2
:1091E60042C3122A05500B85444885454953F5CF9D
:1091F6008076E4FFFE7D01FCAB45AA44A943A84264
:10920600C3122A055020E545F545E5444480F5445A
:10921600E543F543E542F54285444885454953F51E
:10922600CF43F51080427F007E807D017C00AB45F8
:10923600AA44A943A842C3122A055020E545F5458C
:10924600E5444480F544E543F543E542F54285446B
:109256004885454953F5CF43F520800C854448851C
:10926600454953F5CF43F530854982854883E493D4
:10927600FF8547F58546A7A20092AF229000B8E089
:10928600FF12D026900988EFF09000B9E0FF12D0C7
:1092960026900989EFF09000BAE0FF12D0269009D7
:1092A6008AEFF09000BBE0FF12D02690098BEFF01A
:1092B6009000BCE0FF12D02690098CEFF09000BD24
:1092C600E0FF12D02690098DEFF09000BEE0FF126D
:1092D600D02690098EEFF09000C1E0FF12D02690C4
:1092E600099AEFF09000C2E0FF12D02690099BEF9A
:1092F600F09000C3E0FF12D02690099CEFF090009A
:10930600C4E0FF12D02690099DEFF09000C5E0FF63
:1093160012D02690099EEFF09000C6E0FF12D026EC
:1093260090099FEFF09000C7E0FF12D0269009A0A9
:10933600EFF0227536FF7537DD7538158F3C8E3B9D
:109346008D3A8C397B017A1C79761241F28F24751D
:109356003A607539E37538167537007F007E367DBD
:109366006E7C0112C81DE4F522F52374CA2523F587
:109376008274DE3522F583E493FF12D0D80523E507
:109386002370020522C3940AE522940040DDE4F529
:1093960022F523C3E5239524E5229400501B747619
:1093A6002523F582741C3522F583E0FF12D0D805FB
:1093B60023E52370DE052280DAE4FF12D0D87F642D
:1093C6007E007D007C0012AACCEF701978007C002C
:1093D6007D017BFF7ADD791C122C93EF3395E04FEC
:1093E6007003FEFF227E007F01227D0A7FAC12A25F
:1093F600F5901B9BE0F526900995E526F0FF12D027
:109406002690097CEFF0E48F25F524F523F522AEAE
:1094160024AD23AC227810122A298F258E248D2381
:109426008C227D097FAC12A2F5901B9BE0F526905D
:109436000996E526F0FF12D02690097DEFF0AF26BB
:1094460012D026EF7F00FE3395E0FDFCEF2525F5D3
:1094560025E5243EF524E5233DF523E5223CF522CA
:109466007D087FAC12A2F5901B9BE0F5269009972C
:10947600E526F0FF12D02690097EEFF0AF2612D037
:1094860026E4FCFDFEE5252FF525EE3524F524ED35
:109496003523F523EC3522F522AF25AE24AD23FC8A
:1094A60022E4901BA0F0A3F0901BA0E475F001123B
:1094B6002849FE74A325F0F58274093EF583E07011
:1094C600E7901BA0E0FEA3E024A3F974093EFA7B13
:1094D60001128B5C901BA2122A5C7E097F607D00C4
:1094E6007B017A007900122CB0901BA2E0FCA3E06D
:1094F600FDA3E0FEA3E0FF12AEC4EF704D901BA0EB
:10950600F0A3F0901BA0E0FEA3E0FFC3EE9408508A
:109516004574002FF58274003EF583E0FF12D16298
:10952600501812D0FE901BA0E0FEA3E02400F582A6
:1095360074003EF583E0FF12D117901BA1E004F002
:1095460070C1901BA0E004F080B912D0FE7BFF7AB8
:10955600D879391241F8227536FF7537DD75381519
:109566008F3C8E3B8D3A8C397B017A1C7976124181
:10957600F28F24753A607539E37538167537007FB2
:10958600007E367D6E7C0112C81DE4F522F523743B
:10959600DB2523F58274DD3522F583E493FF12D0B3
:1095A600D80523E52370020522C39411E522940011
:1095B60040DDE4F522F523C3E5239524E522940056
:1095C600501B74762523F582741C3522F583E0FF43
:1095D60012D0D80523E52370DE052280DAE4FF12D7
:1095E600D0D87F647E007D007C0012AACCEF701A72
:1095F60078007C007D017BFF7ADD793D122C93EFAC
:109606003395E04F7F017004FF227F0122E4901B17
:10961600A0F0A3F0901BA0E475F001122849FE7497
:10962600A325F0F58274093EF583E070E7901BA050
:10963600E0FEA3E024A3F974093EFA7B01128B5CD9
:10964600901BA2122A5C901BA2E0FCA3E0FDA3E003
:10965600FEA3E0FF12AF41EF705512D0FE7BFF7AFA
:10966600D97922901BA2E0FCA3E0FDA3E0FEA3E0D3
:10967600F5398E388D378C361241F8E4901BA0F000
:10968600A3F0901BA0E0FEA3E0FFC3EE9408502BCE
:1096960074002FF58274003EF583E0FF12D1179017
:1096A6001BA1E004F070DB901BA0E004F080D31255
:1096B600D0FE7BFF7AD979341241F8228B238A2493
:1096C6008925AB23AA24A9251226FBFF12D06E50AA
:1096D6000D74012525F525E43524F52480E4D20012
:1096E600AB23AA24A9251226FBFF642B6004EFB442
:1096F6002D1BAB230525E525AA247002052414F9A4
:109706001226FB642D6003D38001C39200E4F52684
:10971600F527AB23AA24A9251226FBFF12D17150E7
:1097260036AB23AA24A9251226FBFF3395E0FEEFCC
:1097360024D0FBEE34FFFAAE26AF277C007D0A125A
:109746002CDCEF2BF527EE3AF52674012525F525B9
:10975600E43524F52480BB300006AE26AF27800909
:10976600C3E49527FFE49526FE22E4901BA0F0A310
:10977600F0901BA0E475F001122849FE74A325F0B1
:10978600F58274093EF583E070E7901BA0E0FEA326
:10979600E024A3F974093EFA7B01128B5C901BA2AC
:1097A600122A5C7E097F607D007B017A00790012B7
:1097B6002CB0E4901BA0F0A3F0A3E0FCA3E0FDA373
:1097C600E0FEA3E0FF12ADCAEF703F12D0FEE490B8
:1097D6001BA0F0A3F0900960E0FEA3E0FF901BA0A1
:1097E600E0FCA3E0FDC39FEC9E502B74002DF58298
:1097F60074003CF583E0FF12D117901BA1E004F042
:1098060070D3901BA0E004F080CB12D0FE7BFF7AD1
:10981600D779861241F822128032EF600C12D0FE00
:109826007BFF7AD879E70298C112C520EF600C1247
:10983600D0FE7BFF7AD879FB0298C178007C007D48
:10984600017BFF7AD9791C122C93EF3395E04F6098
:10985600617E117F947D007B017A0979A3122CB079
:1098660078A37C097D017B017A0079007E097F60FF
:109876001226D5E4901BA0F0A3F012D0FE901BA0F8
:10988600E475F001122849FE74A325F0F5827409E7
:109896003EF583E0602D901BA0E0FEA3E024A3F537
:1098A6008274093EF583E0FF12D117E4FF12D11747
:1098B60080CB12D0FE7BFF7AD9791F1241F8E4FFE4
:1098C60012D117228B228A2389248F288E278D2650
:1098D6008C2585A729E4F52AF52BF52CF52DF560C1
:1098E600F55FF55EF55DD2ADF5A7D2CA75A710C2D4
:1098F60098AF28AE27AD26AC25AB60AA5FA95EA8B7
:109906005DC3122A055051E52C704D30982CC29833
:10991600AB22AA23A924052BE52BAE2A7002052A21
:1099260014F5828E83E599122786E4F560F55FF5D6
:109936005EF55DE52D7003752D01E52D640170B1B1
:109946007F02FEFDFCAB60AA5FA95EA85DD3122A6A
:1099560005409E752C018099C2ADE4F5A7C2CA8563
:1099660029A7E52C64017F007002AF2B221293F029
:10997600E4901BA0F0A3F012BB6BEF600C12D0FEBC
:109986007BFF7AD87966029A1612D0FE7BFF7AD9C7
:10999600796D1241F812BD99EF60087BFF7AD8798C
:1099A60079806D7BFF7AD979831241F812AC4F7EAC
:1099B600047F007D007B017A0D79A3122CB078A379
:1099C6007C097D017B017A0079007E047F001226E6
:1099D600D57E097FA37DFE7C0312CC37900DA1EFC7
:1099E600F07B017A0979A37DFF7C0312C932900DC1
:1099F600A2EFF0E4F526F5277F907E08FDFC12869F
:109A0600ECEF7BFF70067AD9799480047AD979AD28
:109A16001241F82290096F122A680000000090098E
:109A26006FE0FCA3E0FDA3E0FEA3E0FF901BA0EF28
:109A3600F090096FA3A3A3E07808122A16901BA141
:109A4600EFF090096FE0FCA3E0FDA3E0FEA3E0FFCA
:109A56007810122A16E4901BA2EFF07E1B7FA07DE1
:109A6600037C0012CC37901BA3EFF0901BA0E0FD07
:109A76007F3812D1D1901BA1E0FD7F3912D1D19050
:109A86001BA2E0FD7F3A12D1D1901BA3E0FD7F3BE4
:109A960012D1D1901BA0E0FD7F3C12D1D1901BA129
:109AA600E0FD7F3D12D1D1901BA2E0FD7F3E12D199
:109AB600D1901BA3E0FD7F3F02D1D18E228F23E4FC
:109AC600FD7FAC12A2F5901B9BE0901BA4F044F71F
:109AD600F0FB7A00E4FD7FAC12B3878007901BA4ED
:109AE600E030E7117D037FAC12A2F5901B9BE0905E
:109AF6001BA4F080E8AB23AA227D287FAC12B38793
:109B06008007901BA4E030E71412C1097D037FACE7
:109B160012A2F5901B9BE0901BA4F080E5E5227A4B
:109B260000FB7D297FAC12B3878007901BA4E03031
:109B3600E71412C1097D037FAC12A2F5901B9BE0CE
:109B4600901BA4F080E5E4FD7FAC12A2F5901B9B70
:109B5600E0901BA4F04408F0FB7A00E4FD7FAC0221
:109B6600B387901C1F122A6800014000901C18122F
:109B76002A68000130007F007E407D017C00901C39
:109B860018E0F8A3E0F9A3E0FAA3E0FBC3122A0564
:109B96005066901C18E0FCA3E0FDA3E0FEA3E0FFE6
:109BA6007B017A1C791C753C00753D0312B62C901E
:109BB6001C1CE0F47020A3E0F4701BA3E0F4701604
:109BC600901C18E0FCA3E0FDA3E0FEA3E0FF901CC0
:109BD6001F122A5C8022901C18E0FCA3E0FDA3E083
:109BE600FEA3E02440FFE43EFEE43DFDE43CFC90A1
:109BF6001C18122A5C029B7C901C1FE0FCA3E0FD53
:109C0600A3E0FEA3E0FF228B228A2389248F288EDD
:109C1600278D268C2585A7297531007530C2752FAD
:109C260001752E007F007E367D6E7C0112CA977507
:109C3600A710C298901BA4122A6800000000AF2843
:109C4600AE27AD26AC25901BA4E0F8A3E0F9A3E06F
:109C5600FAA3E0FBC3122A05503B901BA4A3A3E082
:109C6600FEA3E0AB22AA23A924F5828E8312271431
:109C7600FF12D0D8901BA4E0FCA3E0FDA3E0FEA356
:109C8600E02401FFE43EFEE43DFDE43CFC901BA421
:109C9600122A5C80A9C299C2988529A7901BA4E0C4
:109CA600FCA3E0FDA3E0FEA3E0FF22900020E06419
:109CB600547052A3E06441704CA3E064537046A311
:109CC600E0B44B41E4901BAAF0A3F0901BAAE0FE7F
:109CD600A3E0FF2420F58274003EF583E0FD74A323
:109CE6002FF58274093EF583EDF0901BABE004F08E
:109CF6007006901BAAE004F0901BAAE0B404CCA363
:109D0600E0B400C72290096CE064017040901BAA81
:109D1600F0A3F0901BAAE0FEA3E0FF24C6F5827430
:109D2600E03EF583E493FD74A32FF58274093EF5B6
:109D360083EDF0901BABE004F07006901BAAE004E4
:109D4600F0901BAAE07004A3E0642070C6228E2265
:109D56008F23753A607539E37538167537007F00BD
:109D66007E367D6E7C0112C81DE4F524F525742C23
:109D76002525F58274DF3524F583E493FF12D0D8C8
:109D86000525E52570020524C3940CE524940040BE
:109D9600DD852224852325E42523FFE5223404FEE0
:109DA600C3E5259FE5249E501B74A32525F58274E3
:109DB600093524F583E0FF12D0D80525E52570D7AF
:109DC600052480D37FB07E047D007C0012AACCEFF0
:109DD600701A78007C007D017BFF7ADD791C122CDD
:109DE60093EF3395E04F7F017004FF227F01228EAF
:109DF600268F27753A607539E37538167537007FF3
:109E0600007E367D6E7C0112C81DE4F528F52974A6
:109E1600482529F58274DF3528F583E493FF12D0AF
:109E2600D80529E52970020528C39413E52894006E
:109E360040DD852628852729E42527FFE5263404E5
:109E4600FEC3E5299FE5289E501B74A32529F582AC
:109E560074093528F583E0FF12D0D80529E5297065
:109E6600D7052880D37FB07E047D007C0012AACC63
:109E7600EF701A78007C007D017BFF7ADD791C1279
:109E86002C93EF3395E04F7F017004FF227F012270
:109E96008E288F29753A607539E37538167537003F
:109EA6007F007E367D6E7C0112C81DE4F52AF52BF7
:109EB600745B252BF58274DF352AF583E493FF1254
:109EC600D0D8052BE52B7002052AC3940BE52A94FE
:109ED6000040DD85282A85292BE42529FFE528343D
:109EE60004FEC3E52B9FE52A9E501B74A3252BF584
:109EF600827409352AF583E0FF12D0D8052BE52BAD
:109F060070D7052A80D37FB07E047D007C0012AA1C
:109F1600CCEF701A78007C007D017BFF7ADD791C1E
:109F2600122C93EF3395E04F7F017004FF227F01DF
:109F360022E4901BA0F0A3F0901BA0E475F00112A0
:109F46002849FE74A325F0F58274093EF583E07076
:109F5600E7901BA0E0FEA3E024A3F974093EFA7B78
:109F660001128B5C901BA2122A5C7E097F607D0029
:109F76007B017A007900122CB0901BA2E0FCA3E0D2
:109F8600FDA3E0FEA3E0FF12AEC4EF703712D0FED1
:109F9600E4901BA0F0A3F0901BA0E0FEA3E0FFC39B
:109FA600EE9404502B74002FF58274003EF583E086
:109FB600FF12D117901BA1E004F070DB901BA0E00C
:109FC60004F080D312D0FE7BFF7AD879391241F89B
:109FD60022E4901BA0F0A3F0901BA0E475F0011200
:109FE6002849FE74A325F0F58274093EF583E070D6
:109FF600E7901BA0E0FEA3E024A3F974093EFA7BD8
:10A0060001128B5C901BA2122A5C7E097F607D0088
:10A016007B017A007900122CB0901BA2E0FCA3E031
:10A02600FDA3E0FEA3E0FF12AEC4EF703712D0FE30
:10A03600E4901BA0F0A3F0901BA0E0FEA3E0FFC3FA
:10A04600EE9404502B74002FF58274043EF583E0E1
:10A05600FF12D117901BA1E004F070DB901BA0E06B
:10A0660004F080D312D0FE7BFF7AD879391241F8FA
:10A0760022E4901BA0F0A3F0901BA0E475F001125F
:10A086002849FE74A325F0F58274093EF583E07035
:10A09600E77B017A0979A3901BA0E0FEA3E0FFE429
:10A0A600FCFD129C0D7B017A0979A37F947E117DBC
:10A0B600007C0012D2757E00901BA0EEF0A3EFF09C
:10A0C600603D12D0FEE4901BA2F0A3F0901BA0E02E
:10A0D600FEA3E0FFA3E0FCA3E0FDC39FEC9E50229D
:10A0E60074A32DF58274093CF583E0FF12D1179015
:10A0F6001BA3E004F070D5901BA2E004F080CD1203
:10A10600D0937E117F947D007B017A0979A3022C7E
:10A11600B0E4901BA0F0A3F0901BA0E475F0011230
:10A126002849FE74A325F0F58274093EF583E07094
:10A13600E77B017A0979A3901BA0E0FEA3E0FFE488
:10A14600FCFD129C0D7B017A0979A37F947E117D1B
:10A15600007C0012D2757E00901BA0EEF0A3EFF0FB
:10A16600603D12D0FEE4901BA2F0A3F0901BA0E08D
:10A17600FEA3E0FFA3E0FCA3E0FDC39FEC9E5022FC
:10A1860074A32DF58274093CF583E0FF12D1179074
:10A196001BA3E004F070D5901BA2E004F080CD1262
:10A1A600D0937E117F947D007B017A0979A3022CDE
:10A1B600B012D0FEE4901BA0F0A3F0901BA0E0FE2E
:10A1C600A3E0FFC3EE9404501F74A32FF582740D11
:10A1D6003EF583E0FF12D117901BA1E004F070DB7F
:10A1E600901BA0E004F080D3E4FF7E08FDFC901BEA
:10A1F600A3E0F8A3E0F9A3E0FAA3E0FBC3122A0563
:10A20600501CE4FF7E04FDFC901BA3E0F8A3A3A36F
:10A21600E0122A054008901BA2E0FF12D117E49035
:10A226001BA0F0A3F0901BA0E0FEA3E0FFC3EE94FA
:10A2360004501C74A32FF582740D3EF583E4F09050
:10A246001BA1E004F070DE901BA0E004F080D62293
:10A2560012D0FEE4901BA0F0A3F0901BA0E0FEA39A
:10A26600E0FFC3EE9404501F74A32FF58274113ED1
:10A27600F583E0FF12D117901BA1E004F070DB908C
:10A286001BA0E004F080D3E4FF7E0CFDFC901BA233
:10A29600E0F8A3E0F9A3E0FAA3E0FBC3122A055015
:10A2A6001CE4FF7E08FDFC901BA2E0F8A3A3A3E03C
:10A2B600122A054008901BA6E0FF12D117E4901B56
:10A2C600A0F0A3F0901BA0E0FEA3E0FFC3EE940471
:10A2D600501C74A32FF58274113EF583E4F0901B95
:10A2E600A1E004F070DE901BA0E004F080D6228F7F
:10A2F6002C8D2D85A72E75A710E52C64AC703B120E
:10A30600D035E4FDAF2C12C6DDEF7010AF2D12CDA7
:10A3160052EF700512D00080067F01227F012212C3
:10A32600D0357D01AF2C12C6DDEF700B12CD2B9010
:10A336001B9B12CFF980037F0122E52C64807046B7
:10A3460012D035E4FDAF2C12C6DDEF7010AF2D1222
:10A35600CD52EF700512CFFB80067F01227F0122CE
:10A3660012D0357D01AF2C12C6DDEF701612CD2B43
:10A37600901B9BEFF0E4FF12CE3312CD2BA312CF2E
:10A38600F980037F0122852EA77F0022E4901BA07F
:10A39600F0A3F0901BA0E475F001122849FE74A307
:10A3A60025F0F58274093EF583E070E7901BA0E086
:10A3B600FEA3E024A3F974093EFA7B01128B5C909C
:10A3C6001BA2122A5C901BA2E0FCA3E0FDA3E0FE08
:10A3D600A3E0FF12AE47EF703F12D0FEE4901BA041
:10A3E600F0A3F0900960E0FEA3E0FF901BA0E0FC64
:10A3F600A3E0FDC39FEC9E502B74002DF5827400E4
:10A406003CF583E0FF12D117901BA1E004F070D356
:10A41600901BA0E004F080CB12D0FE7BFF7AD779A8
:10A42600DA1241F8228D828C83E0FB8F828E83E0E4
:10A436006B600302A4BD8D828C83A3E0FB8F828EAA
:10A4460083A3E06B70718D828C83A3A3E0FB8F8264
:10A456008E83A3A3E06B705F8D828C83A3A3A3E09E
:10A46600FB8F828E83A3A3A3E06B704BED2404F5D0
:10A4760082E43CF583E0FBEF2404F582E43EF583B9
:10A48600E06B7033ED2405F582E43CF583E0FBEFE9
:10A496002405F582E43EF583E0B5031BED2406F5BD
:10A4A60082E43CF583E0FDEF2406F582E43EF58385
:10A4B600E0B505037F01227F002212D25E787FE499
:10A4C600F6D8FD75816412CF0002A50D02D24FE4C5
:10A4D60093A3F8E493A34003F68001F208DFF48027
:10A4E60029E493A3F85407240CC8C333C4540F4477
:10A4F60020C8834004F456800146F6DFE4800B0151
:10A506000204081020408090BE4EE47E019360BC99
:10A51600A3FF543F30E509541FFEE493A360010EE8
:10A52600CF54C025E060A840B8E493A3FAE493A30F
:10A53600F8E493A3C8C582C8CAC583CAF0A3C8C530
:10A5460082C8CAC583CADFE9DEE780BEE4FD7FAC08
:10A5560012A2F5901B9BE0901BA6F044F7F0FB7A45
:10A5660000E4FD7FAC12B3878007901BA6E030E7BE
:10A57600117D037FAC12A2F5901B9BE0901BA6F009
:10A5860080E87D287FAC12A2F5901B9BE0901BA66D
:10A59600F07D297FAC12A2F5901B9BE0FF901BA2D9
:10A5A600E4F0A3EFF0E0FE901BA6E07C002400FFA1
:10A5B600EC3E901BA4F0A3EFF0E4FD7FAC12A2F5F5
:10A5C600901B9BE0901BA6F04408F0FB7A00E4FD8C
:10A5D6007FAC12B387901BA4E0FEA3E0FF22E490B9
:10A5E6001BA0F0A3F0901BA0E475F001122849FE11
:10A5F60074A325F0F58274093EF583E070E7901B9D
:10A60600A0E0FEA3E024A3F974093EFA7B01128BB5
:10A616005C901BA2122A5C7E097F607D007B017A1A
:10A62600007900122CB0901BA2E0FCA3E0FDA3E091
:10A63600FEA3E0FF12AEC412D0FEE4901BA0F0A36E
:10A64600F0901BA0E0FEA3E0FFC3EE9408501F7439
:10A65600002FF58274003EF583E0FF12D117901BA0
:10A66600A1E004F070DB901BA0E004F080D322E5AB
:10A6760017700302A705E4F517901CA0E004F0E0AC
:10A68600D3941E748094804002E4F0901CA0E0FFF6
:10A69600C31390E1539324FF9297E5146401700568
:10A6A6007F1312B29B7525017526097527647B01F8
:10A6B6007A1B793712910190096AE0D39406748067
:10A6C6009480403BE4F0900966E06402603112CF6A
:10A6D6004D900966E06401700F12CC6190096874B0
:10A6E60007F09009677409F0900966E06403700F3B
:10A6F60012CC619009687401F09009677409F02220
:10A70600E4901BA0F0A3F0901BA0E475F0011228C2
:10A7160049FE74A325F0F58274093EF583E070E7DF
:10A72600901BA0E0FEA3E024A3F974093EFA7B0186
:10A736001296C2901BA2EEF0A3EFF012B8B3EF7020
:10A746003F12D0FEE4901BA0F0A3F0900960E0FE5B
:10A75600A3E0FF901BA0E0FCA3E0FDC39FEC9E508E
:10A766002B74002DF58274003CF583E0FF12D1179F
:10A77600901BA1E004F070D3901BA0E004F080CB06
:10A7860012D0FE7BFF7AD779B41241F822E4901BEF
:10A79600A0F0A3F0901BA0E475F001122849FE7406
:10A7A600A325F0F58274093EF583E070E7901BA0BF
:10A7B600E0FEA3E024A3F974093EFA7B011296C2D7
:10A7C600901BA2EEF0A3EFF07B017A0979A312C0E9
:10A7D6005D12D0FEE4901BA0F0A3F0901BA0E0FC5D
:10A7E600A3E0FDC3EC94045030901BA3E07F00254A
:10A7F600E025E0FEEF2DFFEC3EFE74A32FF58274FC
:10A80600093EF583E0FF12D117901BA1E004F0701A
:10A81600CA901BA0E004F080C222E4901BA0F0A323
:10A82600F0901BA0E475F001122849FE74A325F0F0
:10A83600F58274093EF583E070E7901BA0E475F09D
:10A8460001122849FE74A325F0F58274093EF583AA
:10A85600E070E7901BA0E475F001122849FE74A38E
:10A8660025F0F58274093EF583E070E7901BA0E4BD
:10A8760075F001122849FE74A325F0F58274093E8D
:10A88600F583E070E7901BA0E0FEA3E024A3F97433
:10A89600093EFA7B011296C2901BA2EEF0A3EFF0DE
:10A8A600129AC102D0818E228F238C248D257E0997
:10A8B6007F607D007B017A007900122CB0753AE04A
:10A8C6007539937538047537007F007E367D6E7C4A
:10A8D6000112C81DE4F526F527C3E5279525E526CB
:10A8E6009524501BE5232527F582E5223526F58399
:10A8F600E0FF12D0D80527E52770DE052680DA7F2F
:10A90600327E007D007C0012AACCEF7020F526F581
:10A91600270527E527AE2670020526142400F582B2
:10A9260074003EF583E070E9AE26AF2722E4FEFF11
:10A93600228E288F298C2A8D2B7D0E7FAC12A2F5B4
:10A9460012D021852982852883EFF0901B9BE08514
:10A956002B82852A83F07D0D7FAC12A2F512D021C1
:10A96600852982852883A3EFF0901B9BE0852B82A7
:10A97600852A83A3F07D0B7FAC12A2F512D0218528
:10A986002982852883A3A3A3EFF0901B9BE0852B48
:10A9960082852A83A3A3A3F07D0C7FAC12A2F512B5
:10A9A600D021852982852883A3A3EFF0901B9BE005
:10A9B600852B82852A83A3A3F07F00228E288F29E8
:10A9C6008C2A8D2B7D0A7FAC12A2F512D021E529A7
:10A9D6002404F582E43528F583EFF0901B9BE0FF15
:10A9E600E52B2404F582E4352AF583EFF07D097F13
:10A9F600AC12A2F512D021E5292405F582E435280A
:10AA0600F583EFF0901B9BE0FFE52B2405F582E430
:10AA1600352AF583EFF07D087FAC12A2F512D0211E
:10AA2600E5292406F582E43528F583EFF0901B9B93
:10AA3600E0FFE52B2406F582E4352AF583EFF07F67
:10AA4600002212D2847536FF7537D97538E790091A
:10AA560078E0753900F53AA3E0753B00F53C9009BE
:10AA66007BE0753D00F53EA3E0753F00F540A3E0B1
:10AA7600754100F542A3E0754300F5447B017A0970
:10AA860079A31241F2901BA012D0F9E4901BA2F018
:10AA9600A3F0901BA0E0FEA3E0FFA3E0FCA3E0FD73
:10AAA600C39FEC9E501F74A32DF58274093CF58359
:10AAB600E0FF12D117901BA3E004F070D5901BA203
:10AAC600E004F080CD228F368E358D348C33E4F55C
:10AAD60037F538F560F55FF55EF55D7E007F007D44
:10AAE600607C0912D18EE47F04FEFDFCAB36AA35EC
:10AAF600A934A8331228C4AB60AA5FA95EA85DC3B7
:10AB0600122A055006E55C455B60DBE47F08FEFD26
:10AB1600FCAB60AA5FA95EA85DC3122A0540EC5390
:10AB2600E7F7900960E55BF0A3E55CF0AE5FAF6028
:10AB3600A3EEF0A3EFF0D3900961E09400900960D2
:10AB4600E094007F0140027F00227E097F607D0045
:10AB56007B017A007900122CB0753A607539E3757D
:10AB660038167537007F007E367D6E7C0112C81D53
:10AB7600E4F522F52374EC2523F58274DD3522F500
:10AB860083E493FF12D0D80523E52370020522C380
:10AB9600940FE522940040DD7F647E007D007C00FA
:10ABA60012AACCEF7020F522F5230523E523AE2269
:10ABB60070020522142400F58274003EF583E070CD
:10ABC600E9AE22AF2322E4FEFF22E48F2C8E2BF582
:10ABD6002AF529900968E06401702CAD2AAC297B1E
:10ABE60037FAF9F81228C48F2C8E2B8D2A8C29E47B
:10ABF6007BE87A03F9F81228C48F2C8E2B8D2A8CC9
:10AC060029E4FB7A0C8030AF2CAE2BAD2AAC29E4BC
:10AC16007B37FAF9F81228C48F2C8E2B8D2A8C29B3
:10AC2600E47BE87A03F9F81228C48F2C8E2B8D2A40
:10AC36008C29E47B997A09F9F812294F8F2C8E2BEF
:10AC46008D2A8C29AE2BAF2C229000317401F09006
:10AC56001B93E0900025F0901B94E0900026F09066
:10AC66001B95E0900027F0901B96E0900028F0904E
:10AC76001B97E0900029F0901B98E090002AF09036
:10AC86001B99E090002BF0901B9AE090002CF0901E
:10AC96000991E09000DCF0900992E09000DDF090E0
:10ACA6000993E09000DEF0900994E09000DFF090C8
:10ACB6000995E09000E0F0900996E09000E1F090B0
:10ACC6000997E09000E2F022E4901BA0F0A3F012B6
:10ACD600C3F0EF704412D0FEE4901BA0F0A3F090F6
:10ACE6000960E0FEA3E0FF901BA0E0FCA3E0FDC32B
:10ACF6009FEC9E501F74002DF58274003CF583E096
:10AD0600FF12D117901BA1E004F070D3901BA0E0B6
:10AD160004F080CBE4FF02D11712D0FEE4901BA012
:10AD2600F0A3F0E4FF12D117901BA1E004F0700627
:10AD3600901BA0E004F0C3901BA1E09410901BA010
:10AD4600E0940040DE22E4901BA0F0A3F012C43D84
:10AD5600EF704412D0FEE4901BA0F0A3F0900960BF
:10AD6600E0FEA3E0FF901BA0E0FCA3E0FDC39FEC88
:10AD76009E501F74002DF58274003CF583E0FF128F
:10AD8600D117901BA1E004F070D3901BA0E004F053
:10AD960080CBE4FF02D11712D0FEE4901BA0F0A3F3
:10ADA600F0E4FF12D117901BA1E004F07006901B8F
:10ADB600A0E004F0C3901BA1E09410901BA0E094C7
:10ADC6000040DE227536FF7537DD7538158F3C8EEF
:10ADD6003B8D3A8C397B017A1C79761241F28F23AE
:10ADE600753A607539E37538167537007F007E361B
:10ADF6007D6E7C0112C81DE4F522C3E522940C7415
:10AE0600809480500EE52290DE6993FF12D0D8051B
:10AE16002280E7E4F522E522C395235014747625B3
:10AE260022F582E4341CF583E0FF12D0D805228097
:10AE3600E5E4FF12D0D87FC87E007D007C0002AA20
:10AE4600CC7536FF7537DD7538158F3C8E3B8D3AE0
:10AE56008C397B017A1C79761241F28F23753A6020
:10AE66007539E37538167537007F007E367D6E7C42
:10AE76000112C81DE4F522C3E52294107480948063
:10AE8600500EE52290DEAA93FF12D0D8052280E765
:10AE9600E4F522E522C39523501474762522F58223
:10AEA600E4341CF583E0FF12D0D8052280E5E4FFE8
:10AEB60012D0D87F807EEE7DFF7CFF02AACC75364D
:10AEC600FF7537DD7538158F3C8E3B8D3A8C397B97
:10AED600017A1C79761241F28F24753A607539E34E
:10AEE6007538167537007F007E367D6E7C0112C878
:10AEF6001DE4F523C3E523940974809480500EE580
:10AF06002390DEC193FF12D0D8052380E7E4F52312
:10AF1600E523C39524501474762523F582E4341C66
:10AF2600F583E0FF12D0D8052380E5E4FF12D0D8E0
:10AF36007FC87E007D007C0002AACC7536FF75377F
:10AF4600DD7538158F3C8E3B8D3A8C397B017A1C2A
:10AF560079761241F28F23753A607539E3753816A2
:10AF66007537007F007E367D6E7C0112C81DE4F5C4
:10AF760022C3E522941074809480500EE52290DD61
:10AF8600CB93FF12D0D8052280E7E4F522E522C351
:10AF96009523501474762522F582E4341CF583E05B
:10AFA600FF12D0D8052280E5E4FF12D0D87FC87EF4
:10AFB600007D007C0002AACC900967E06401603342
:10AFC6007401F012CA0112D1F61220267FB07E71EA
:10AFD6007D0B7C0012C0067F011220967F01122095
:10AFE600067F0112CFA612A552900964EEF0A3EFD8
:10AFF600F0D297E5176006E4F5171288BB1262C116
:10B00600EF700C12D221122CEE12D22B127249754D
:10B0160025017526097527647B017A1B79371291FC
:10B026000190096AE0D39402748094804005E4F0AC
:10B0360012C88F22900967E0640360037403F0E589
:10B0460017606CE4F517901C9FE004F0E0D3941EA3
:10B05600748094804002E4F0901C9FE0FFC313903C
:10B06600E1439324FF929775250175260975276498
:10B076007B017A1B793712910190096AE0D3940615
:10B08600748094804029E4F0900966E06402601FB1
:10B09600A37409F0900966E064017006900968746B
:10B0A60007F0900966E06403700590096804F022D1
:10B0B6007F3812D1C4901B93EFF07F3912D1C49020
:10B0C6001B94EFF07F3A12D1C4901B95EFF07F3BB3
:10B0D60012D1C4901B96EFF07F3C12D1C4901B97FF
:10B0E600EFF07F3D12D1C4901B98EFF07F3E12D156
:10B0F600C4901B99EFF07F3F12D1C4901B9AEFF0DA
:10B106007E1B7F937D047C0012CC378F227E1B7FB3
:10B11600977D047C0012CC37E52270028003EF7025
:10B1260003FF8003E47F01FEFDFC22E4901BA0F0F8
:10B13600A3F0901BA0E475F001122849FE74A32524
:10B14600F0F58274093EF583E070E7901BA0E0FEFF
:10B15600A3E024A3F974093EFA7B01128B5C901BD1
:10B16600A2122A5C901BA2E0FCA3E0FDA3E0FEA3D2
:10B17600E0FF12955DEF702012D0FE7BFF7AD87942
:10B18600BE901BA2E0FCA3E0FDA3E0FEA3E0F53920
:10B196008E388D378C36800912D0FE7BFF7AD879AF
:10B1A600DA1241F82212928212D28412D27B8F11C5
:10B1B6008E108D0F8C0E12B7078F22EF640270452A
:10B1C600FFFEFDFCAB11AA10A90FA80EC3122A059B
:10B1D600700A12CC6190096874038021900966E0B8
:10B1E600640160277F0112CFA612D2847D03AF16B9
:10B1F600AE1512600B124A419009687405F0900969
:10B20600677409F022E52264037003023D16900973
:10B21600687403F09009677409F012CC61227E0904
:10B226007F607D007B017A007900122CB012BCE3AE
:10B23600EF7055901BA0F0A3F0901BA0E0FEA3E0DA
:10B24600FFC3EE9408503974002FF58274003EF562
:10B2560083E0FF12D162501812D0FE901BA0E0FED0
:10B26600A3E02400F58274003EF583E0FF12D117B7
:10B27600901BA1E004F070C1901BA0E004F080B91F
:10B286007BFF7AD679F1800912D0FE7BFF7AD879D6
:10B29600141241F8228F22E4F51412CA0112202654
:10B2A60012D1F612CDC57F011220067F0112CFA65C
:10B2B60012CF4D12BCE3EF7002803C7F2C7E011250
:10B2C600CA3312BCE3EF7002802D7F2C7E0112CAB6
:10B2D6003312BCE3EF7002801E7D12AF16AE15125C
:10B2E600600B7B017A00790012CDE8EF700E7D1CB1
:10B2F600AF16AE1512600BAF2202CD9F12CC619035
:10B3060009687403F09009677409F02212BCE3EF30
:10B316007002801EE4FF1220067FE87E0312CA3305
:10B326007F011220067FE87E0312CA3312BCE3EFC8
:10B33600701112928212CC61E4FDAF16AE15126046
:10B346000B80187F2C7E0112CA3312C9CEEF7018FB
:10B35600FDAF16AE1512600B12CC6190096874022F
:10B36600F09009677409F0229009687403F07D185B
:10B37600AF16AE1512600B9009677409F012CC6116
:10B38600228F268D278A288B2985A72A75A710E55F
:10B396002664AC702412C6D6EF701BAF2712CD52AE
:10B3A600EF7010AF2912CD52EF700512D000800950
:10B3B6007F01227F01227F0122E526648070301200
:10B3C600C6D6EF7027AF2712CD52EF701CE528FFC7
:10B3D60012CD52EF7010AF2912CD52EF700512D078
:10B3E60000800C7F01227F01227F01227F012285BE
:10B3F6002AA77F0022900991E09009AFF090099268
:10B40600E09009B0F0900993E09009B1F0900994AA
:10B41600E09009B2F0900995E09009B3F090099692
:10B42600E09009B4F0900997E09009B5F012D0FECB
:10B43600E4901BA0F0A3F0901BA0E0FEA3E0FFC3E6
:10B446009413EE9400501F74A32FF58274093EF5F1
:10B4560083E0FF12D117901BA1E004F070D9901B76
:10B46600A0E004F080D12212D0FEE4901BA0F0A34D
:10B47600F0901BA0E0FEA3E0FFC3EE9404501F74FF
:10B48600A32FF58274153EF583E0FF12D117901BAA
:10B49600A1E004F070DB901BA0E004F080D3901BC9
:10B4A600A2E0FF12D117E4901BA0F0A3F0901BA01E
:10B4B600E0FEA3E0FFC3EE9404501C74A32FF582B4
:10B4C60074153EF583E4F0901BA1E004F070DE9065
:10B4D6001BA0E004F080D622E4901BA0F0A3F0129B
:10B4E600D1F61220267F011220067FE87E0312CABB
:10B4F60033C29712BC85EF7002800E12BC85EF70C6
:10B5060002800612BC85EF700D7F0112CF9012D11A
:10B51600DEC2AF75A70FE4901BA0F0A3F0901BA0AE
:10B52600E0FEA3E0FFE4FCFD7B407A9CF9F8D31231
:10B5360029EF4010901BA1E004F070E1901BA0E001
:10B5460004F080D9B29780CEE4901BA0F0A3F0124D
:10B55600C3A3EF7055901BA0F0A3F0901BA0E0FED4
:10B56600A3E0FFC3EE9404503974002FF5827400F3
:10B576003EF583E0FF12D162501812D0FE901BA058
:10B58600E0FEA3E02400F58274003EF583E0FF129E
:10B59600D117901BA1E004F070C1901BA0E004F04D
:10B5A60080B97BFF7AD679F1800912D0FE7BFF7ACB
:10B5B600D679F41241F8227E097F607D007B017AFC
:10B5C600007900122CB012C352EF704D901BA0F000
:10B5D600A3F0901BA0E0FEA3E0FFC3EE9408504545
:10B5E60074002FF58274003EF583E0FF12D162509D
:10B5F6001812D0FE901BA0E0FEA3E02400F5827492
:10B60600003EF583E0FF12D117901BA1E004F07015
:10B61600C1901BA0E004F080B912D0FE7BFF7AD85F
:10B6260079141241F8228F388E378D368C358B3946
:10B636008A3A893B8F418E408D3F8C3EE53D2538C9
:10B64600FFE53C3537FEE43536FDE43535FCAB41E8
:10B65600AA40A93FA83EC3122A055037AF41AE40C3
:10B66600AD3FAC3E1291C3AB39AA3AA93BEF1227C4
:10B67600747401253BF53BE4353AF53AE54124017E
:10B68600F541E43540F540E4353FF53FE4353EF518
:10B696003E80A9228E228F23753A607539E375386C
:10B6A600167537007F007E367D6E7C0112C81DE45C
:10B6B600F524C3E524941174809480500EE52490FB
:10B6C600DEDF93FF12D0D8052480E7AF2312D0D84F
:10B6D600E522FF12D0D87F007E537D077C0012AA98
:10B6E600CCEF701A78007C007D017BFF7ADD791C37
:10B6F600122C93EF3395E04F7F017004FF227F01F8
:10B70600227526017527097528787B017A097988BB
:10B7160012842DEF3395E0C3648094807F0050023D
:10B726007F01AD077526017527097528787B017A93
:10B7360009799A12842DEF3395E0C3648094807F53
:10B746000050027F01EDFB7A007006EF70037F0167
:10B7560022EB64014A7006EF70037F0222ED64015A
:10B766007008EF640170037F03227F00228F388EFA
:10B77600378D368C358B398A3A893B8F418E408D91
:10B786003F8C3EE53D2538FFE53C3537FEE4353652
:10B79600FDE43535FCAB41AA40A93FA83EC3122AB9
:10B7A600055035AF41AE40AD3FAC3EAB39053BE54C
:10B7B6003BAA3A7002053A14F91226FBF5461282A4
:10B7C60039E5412401F541E43540F540E4353FF5DE
:10B7D6003FE4353EF53E80AB227FFE7EFF7D007C5A
:10B7E600001291C3EF901BA0F0A3E4F07FFF7EFF51
:10B7F600FDFC1291C3901BA1E02FF0901BA0E0343A
:10B8060000F0A3E004F07006901BA0E004F07FFEB9
:10B816007EFF7D007C00128334901BA0E0F5467FFE
:10B82600FE7EFF7D007C00128239901BA0A3E0F50E
:10B83600467FFF7EFF7D007C00128239E4F5A77506
:10B84600EF10227D19AF16AE1512600B12CF7AEFEC
:10B85600603912BCE3EF700280157F2C7E0112CA9C
:10B866003312BCE3EF7002800612C9CEEF700302FA
:10B87600B1AB12CC617D18AF16AE1512600B9009F4
:10B88600687403F09009677409F0227D1BAF16AE49
:10B896001512600B9009687403F07D18AF16AE158B
:10B8A60012600B9009677409F012CC61228E228F08
:10B8B600237536FF7537DD75381985223985233AA4
:10B8C6007B017A1C79761241F28F25753A607539BB
:10B8D600E37538167537007F007E367D6E7C011263
:10B8E600C81DE4F524C3E524940B74809480500E9F
:10B8F600E52490DE7593FF12D0D8052480E7AF23A8
:10B9060012D0D8E522FF12D0D87FC87E007D007CF9
:10B916000002AACC900991E08F828E83F090099262
:10B92600E08F828E83A3F0900993E08F828E83A3AB
:10B93600A3F0900994E08F828E83A3A3A3F09009CD
:10B9460095E0FDEF2404F582E43EF583EDF09009E1
:10B9560096E0FDEF2405F582E43EF583EDF09009CF
:10B9660097E0FDEF2406F582E43EF583EDF0EF2443
:10B9760007F582E43EF583E4F02285A72CE4F5A7DB
:10B986008FBBD2ECFF20ED0DEFC3946474809480DE
:10B9960050030F80F0C2EDC3EF946474809480402E
:10B9A60006AC2DAD2E8030AFBDAEBEE48F328E31EB
:10B9B600F530F52F7F307E11FDFCAB32AA31A93070
:10B9C600A82F1228C4E47BFF7A0FF9F812294FAC8E
:10B9D60006AD078C2D8D2E852CA7AF05AE0422E46F
:10B9E600B51B14E51AB4080FAF11AE10AD0FAC0EAF
:10B9F600E4F52EF52F8032AF11AE10AD0FAC0EE48C
:10BA0600F52EF52F12851AE5112401F511E43510EE
:10BA1600F510E4350FF50FE4350EF50EAF11AE1047
:10BA2600AD0FFC752E08752F0012851AE51124013D
:10BA3600F511E43510F510E4350FF50FE4350EF584
:10BA46000E22753A607539E37538167537007F0032
:10BA56007E367D6E7C0112C81DE4F527C3E527946A
:10BA66001274809480500EE52790DEF093FF12D07A
:10BA7600D8052780E7E4FF12D0D87F887E137D00A3
:10BA86007C0012AACCEF701A78007C007D017BFF47
:10BA96007ADD791C122C93EF3395E04F7F01700409
:10BAA600FF227F0122AB07AA06901B47A3A3A3E0B0
:10BAB6008B828A83F0901B47E0FCA3E0FDA3E0FEA7
:10BAC600A3E0FF7808122A168B828A83A3EFF090F0
:10BAD6001B47E0FCA3E0FDA3E0FEA3E0FF78101205
:10BAE6002A168B828A83A3A3EFF0901B47E0FCA360
:10BAF600E0FDA3E0FEA3E0FF7818122A168B828AE7
:10BB060083A3A3A3EFF0228D26E5266402701A1202
:10BB160026FB901BA5F0900001122714901BA4F0A1
:10BB2600E0FEA3E0FFE4FCFD22E526640470271294
:10BB360026FB901BA7F0900001122714901BA6F07D
:10BB4600900002122714901BA5F0900003122714F0
:10BB5600901BA4F08003901BA4E0FCA3E0FDA3E0EF
:10BB6600FEA3E0FF22753A607539E375381675371E
:10BB7600007F007E367D6E7C0112C81DE4F527C36A
:10BB8600E527940C74809480500EE52790DDAC93E5
:10BB9600FF12D0D8052780E77F887E137D007C00C2
:10BBA60012AACCEF701A78007C007D017BFF7ADD4B
:10BBB600791C122C93EF3395E04F7F017004FF221E
:10BBC6007F0122753A607539E37538167537007F3F
:10BBD600007E367D6E7C0112C81DE4F522C3E52287
:10BBE600940374809480500EE52290DD4093FF12FA
:10BBF600D0D8052280E77F0A7E007D007C0012AA4D
:10BC0600CCEF701A78007C007D017BFF7ADD791C11
:10BC1600122C93EF3395E04F7F017004FF227F01D2
:10BC260022753A607539E37538167537007F007EE0
:10BC3600367D6E7C0112C81DE4F522C3E522940907
:10BC460074809480500EE52290DD4393FF12D0D885
:10BC5600052280E77F0A7E007D007C0012AACCEFD9
:10BC6600701A78007C007D017BFF7ADD791C122C2E
:10BC760093EF3395E04F7F017004FF227F01227519
:10BC86003A607539E37538167537007F007E367D64
:10BC96006E7C0112C81DE4F522C3E522940B748064
:10BCA6009480500EE52290DF0293FF12D0D8052231
:10BCB60080E77F647E007D007C0012AACCEF701ABC
:10BCC60078007C007D017BFF7ADD791C122C93EFD6
:10BCD6003395E04F7F017004FF227F0122753A60A1
:10BCE6007539E37538167537007F007E367D6E7CB4
:10BCF6000112C81DE4F52AF52B740D252BF5827467
:10BD0600DF352AF583E493FF12D0D8052BE52B7097
:10BD160002052AC3940CE52A940040DD7F887E1331
:10BD26007D007C0012AACCEF700B7E007F007DFFA9
:10BD36007C0302CC377F0122753A607539E375388A
:10BD4600167537007F007E367D6E7C0112C81DE4B5
:10BD5600F526F52774192527F58274DF3526F58330
:10BD6600E493FF12D0D80527E52770020526C39471
:10BD760013E526940040DD7F887E137D007C00124B
:10BD8600AACCEF700B7E007F007DFF7C0302CC37D0
:10BD96007F0122753A607539E37538167537007F6D
:10BDA600007E367D6E7C0112C81DE4F523F52474F1
:10BDB600942524F58274DD3523F583E493FF12D0B0
:10BDC600D80524E52470020523C3940BE5239400CB
:10BDD60040DD7F887E137D007C0012AACCEF700BBD
:10BDE6007E007F007DFF7C0302CC377F0122901B03
:10BDF600A0122A68000130007F007E607D017C0071
:10BE0600901BA0E0F8A3E0F9A3E0FAA3E0FBC312BD
:10BE16002A055033901BA0E0FCA3E0FDA3E0FEA39F
:10BE2600E0FF128334901BA0E0FCA3E0FDA3E0FE3C
:10BE3600A3E02400FFEE3402FEE43DFDE43CFC906A
:10BE46001BA0122A5C80B122421C9D0000441C806B
:10BE560000000E10441C8400000E10441C880000D4
:10BE66000E10441C8C00000E10441C9000000E1096
:10BE7600441C9400000708411C9800411C9900418D
:10BE86001C9C00015A00015900024F00000251009B
:10BE960000025300000155000215097802180991A5
:10BEA60000E4901BA0F0A3F012AB50901BA2EEF0A2
:10BEB600A3EFF04E603F12D0FEE4901BA0F0A3F07B
:10BEC600901BA2E0FEA3E0FF901BA0E0FCA3E0FD18
:10BED600C39FEC9E502274002DF58274003CF583BE
:10BEE600E0FF12D117901BA1E004F070D3901BA0C5
:10BEF600E004F080CB12D093228E328F338C348DB7
:10BF060035E4F560F55FF55EF55DAF03AE029009C9
:10BF160085E0FCA3E0FD12D18EAE32AF33E4FCFD2A
:10BF2600AB60AA5FA95EA85DC3122A055006E55C50
:10BF3600455B60E5AE34AF35E4FCFDAB60AA5FA9B6
:10BF46005EA85DC3122A0540EB53E7F7AE5BAF5C14
:10BF5600228B358A3689378B3B8A3C893DAB350542
:10BF660037E537AA367002053614F91226FB70ED4E
:10BF760074FF2537F53774FF3536F536AB38053A95
:10BF8600E53AAA397002053914F91226FBFFAB35DA
:10BF96000537E537AA367002053614F9EF1227740D
:10BFA60070DAAB3BAA3CA93D228F358E348D338C9B
:10BFB60032E47F03FEFDFCAB35AA34A933A832C3B5
:10BFC600122A055008E47F01FEFDFC801AAF35AE4B
:10BFD60034AD33AC32E41223A47B9A7A997939785A
:10BFE600401223071223E28F398E388D378C36782C
:10BFF6003674FF122A3EEC4D4E4F60030080F0224D
:10C0060085A722E4F5A775981075A70F122ADBC03D
:10C016004E00002580C0460001C200C041000B71E1
:10C02600B0C03C000F4240C0370016E3600000C0BD
:10C036005475ACF8800D75ACF4800875ACF08003CF
:10C0460075AC9875ADFF800675AC1E75ADFB75AB0E
:10C0560043D2AC8522A7228B278A288929753C10D2
:10C06600753D007F007E307D017C0012B62CE4F524
:10C076002AF52BAE2AAF2BE4FCFDFB7A10F9F8D398
:10C08600122A054027AB27AA28A929852B82852AAB
:10C0960083122714F4700B852B82852A8374201251
:10C0A6002786052BE52B70CB052A80C722C0E0C06A
:10C0B60083C082C0D075D000C00630983BC298C3FA
:10C0C600E55C9564E55B9563502B856282856183AB
:10C0D600055CE55CAE5B7002055B142582F582E5C6
:10C0E600833EF583E599F0756000755F00755E0027
:10C0F600755D00800353E7F7D006D0D0D082D08399
:10C10600D0E0327F0A7E007D007C008F278E268D50
:10C11600258C24E4F52BF52AF529F528AF27AE263C
:10C12600AD25AC24AB2BAA2AA929A828C3122A0517
:10C136005025E4FFFE0FBF00010EBE04F8BF38F520
:10C14600E52B2401F52BE4352AF52AE43529F529D2
:10C15600E43528F52880C522E4901BA0F0A3F090D2
:10C166001BA0E475F001122849FE74A325F0F582A0
:10C1760074093EF583E070E712D0FE901BA0E0FE46
:10C18600A3E024A3F58274093EF583E0601D901BAD
:10C19600A0E475F001122849FE74A325F0F5827417
:10C1A600093EF583E0FF12D11780D022E4901BA050
:10C1B600F0A3F0901BA0E475F001122849FE74A3C9
:10C1C60025F0F58274093EF583E070E712D0FE9003
:10C1D6001BA0E0FEA3E024A3F58274093EF583E0EC
:10C1E600601D901BA0E475F001122849FE74A3257A
:10C1F600F0F58274093EF583E0FF12D11780D02254
:10C206007E097F607D007B017A007900122CB07573
:10C216003AE07539937538047537007F007E367DB0
:10C226006E7C0112C81D7F3112D0D87F327E007D10
:10C23600007C0012AACCEF7017FFFE0FEFAC067061
:10C24600010E142400F58274003CF583E070EC22A4
:10C25600E4FEFF227E097F607D007B017A00790083
:10C26600122CB0753AE07539937538047537007F2E
:10C27600007E367D6E7C0112C81D7F3212D0D87FBB
:10C28600327E007D007C0012AACCEF7017FFFE0FF5
:10C29600EFAC0670010E142400F58274003CF583A1
:10C2A600E070EC22E4FEFF2212BCE3EF703F12D0F6
:10C2B600FEE4901BA0F0A3F0900960E0FEA3E0FF6F
:10C2C600901BA0E0FCA3E0FDC39FEC9E502B7400E6
:10C2D6002DF58274003CF583E0FF12D117901BA167
:10C2E600E004F070D3901BA0E004F080CB12D0FEE7
:10C2F6007BFF7AD7795F1241F8228B298A2A892B0C
:10C30600E94A4B60467F1312B980EE3395E0FDFC97
:10C31600E47B0BFAF9F81228C4AB29AA2AA92B90B8
:10C326000002EE8FF01228977F1212B980EE339535
:10C33600E0FDFCE47B0BFAF9F81228C4AB29AA2A23
:10C34600A92B900004EE8FF012289722753A60759B
:10C3560039E37538167537007F007E367D6E7C01B1
:10C3660012C81DE4F522F52374382523F58274DFFF
:10C376003522F583E493FF12D0D80523E523700216
:10C386000522C39410E5226480948040DBE4FF120A
:10C39600D0D87FF47E017D007C0002AACC7E097F86
:10C3A600607D007B017A007900122CB0753A6075C9
:10C3B60039E37538167537007F007E367D6E7C0151
:10C3C60012C81DE4F522C3E52294097480948050B6
:10C3D6000EE52290DE8093FF12D0D8052280E77FFB
:10C3E600327E007D007C0002AACC7E097F607D0043
:10C3F6007B017A007900122CB0753A607539E375C5
:10C4060038167537007F007E367D6E7C0112C81D9A
:10C41600E4F522C3E522941174809480500EE5223F
:10C4260090DE8993FF12D0D8052280E77F647E00D4
:10C436007D007C0002AACC7E097F607D007B017AAC
:10C44600007900122CB0753A607539E375381675A7
:10C4560037007F007E367D6E7C0112C81DE4F52212
:10C46600C3E522941074809480500EE52290DE9AE3
:10C4760093FF12D0D8052280E77F647E007D007C82
:10C486000002AACC7E017FBE7D007B017A0979A3DA
:10C49600122CB0E4900B61F0900B65740BF0900BCE
:10C4A600697404F0E4A3F0A3F0A3F0A3F0A3740965
:10C4B600F0A3743DF0E4A3F07E04FFFD7B017A0B4C
:10C4C6007971122CB0900BA17455F0A374AAF022C6
:10C4D600753A607539E37538167537007F007E3614
:10C4E6007D6E7C0112C81DE4F528F529741E2529E8
:10C4F600F58274DE3528F583E493FF12D0D805293A
:10C50600E52970020528C3940DE528940040DD7FD7
:10C51600E87E037D007C0002AACC753A607539E39B
:10C526007538167537007F007E367D6E7C0112C821
:10C536001DE4F522F523744F2523F58274DE35229A
:10C54600F583E493FF12D0D80523E5237002052274
:10C55600C3940DE522940040DD7FE07E937DFF7C51
:10C56600FF02AACC8D238B2412D05B7A00EF448085
:10C57600FB7D167FAC12B387AF2312D05B7A00EF38
:10C586004480FB7D157FAC12B387AF2412D05B7A53
:10C5960000EF4480FB7D137FAC12B387AF2512D02A
:10C5A6005B7A00EF5401FB7D147FAC02B387E49005
:10C5B6001BA0F0A3F0901BA0E475F001122849FE21
:10C5C60074A325F0F58274093EF583E070E7901BAD
:10C5D600A0E0FEA3E0FF129D54EF700512D081800B
:10C5E6000312D093901BA0E0FEA3E024A3F97409E4
:10C5F6003EFA7B0102D0C7855C82855B83E47F0AB5
:10C60600FEFDFCAB60AA5FA95EA85DD3122A0540B9
:10C616002CD3E5829400E5839400402178237C1C8A
:10C626007D017BFF7AE17969122C93EF3395E04F18
:10C63600700553E7F7FF2253E7F77F01227F0122B8
:10C64600E4901BA0F0A3F012C3A3EF703712D0FE44
:10C65600E4901BA0F0A3F0901BA0E0FEA3E0FFC3B4
:10C66600EE9404502274002FF58274003EF583E0A8
:10C67600FF12D117901BA1E004F070DB901BA0E025
:10C6860004F080D312D093228E228F23753A6075E0
:10C6960039E37538167537007F007E367D6E7C016E
:10C6A60012C81DE4F524C3E52494117480948050C7
:10C6B6000EE52490DEDF93FF12D0D8052480E7AF85
:10C6C6002312D0D8E522FF12D0D812D20C7F002236
:10C6D60012D035E4FDAF2685A72F75A710AE07ED5E
:10C6E6004206E5C830E7FB12D03512D217E4FDED5D
:10C6F600C3940874809480500A12CE2BEE25E0FE77
:10C706000D80EC12CEC88F30E530600312CFFB856A
:10C716002FA7AF3022C2D5E830E70FB2D5E4C39BCE
:10C72600FBE49AFAE499F9E498F8EC30E717B2D505
:10C7360012C75112294FE4C39BFBE49AFAE499F914
:10C74600E498F8800312294F30D50DE4C39FFFE427
:10C756009EFEE49DFDE49CFC22E48F258E24F523B9
:10C76600F522AD23AC227B37FAF9F81228C48F25BF
:10C776008E248D238C22E47BE87A03F9F81228C4F0
:10C786008F258E248D238C22E47B997A09F9F81261
:10C79600294F8F258E248D238C22228D238B2412C4
:10C7A600D05BEFFB7A007D0E7FAC12B387AF23120E
:10C7B600D05BEFFB7A007D0D7FAC12B387AF2412FE
:10C7C600D05BEFFB7A007D0B7FAC12B387AF2512EF
:10C7D600D05BEFFB7A007D0C7FAC02B38785A73078
:10C7E60075A70F53E7F7C28E53C7FD75A710859936
:10C7F60031C298C29975A70F75D4CF75D50343C7B3
:10C8060002852F44852E43852D42852C411276D2F2
:10C8160043E7088530A72285A73B75A70F53E7F79F
:10C82600C28E53C7FD75A71085993CC298C29975EB
:10C83600A70F75D4CFE4F5D543C702853A448539A9
:10C84600438538428537411276D243E708853BA7B0
:10C85600228D228B2312D05B7A00EF4480FB7D125F
:10C866007FAC12B387AF2212D05B7A00EF4480FB15
:10C876007D117FAC12B387AF2312D05B7A00EF44F1
:10C8860080FB7D107FAC02B387900966E06403608D
:10C896002EC29712D15390096BEFF0E4A3F012CC9D
:10C8A60061900966E06402701090096BE0600AE42A
:10C8B600F5149009687402F0229009687403F02256
:10C8C600AEA7E4F5A78FBBD2ECFF20ED0DEFC39426
:10C8D600647480948050030F80F0C2EDEFC39464BB
:10C8E6007480948040067C067D008004ACBEADBD9D
:10C8F6008EA7AF05AE0422128EB38F258E248D230C
:10C906008C22EC4D4E4F601712D0FE7BFF7AD87901
:10C916009685253985243885233785223680091260
:10C92600D0FE7BFF7AD879AB1241F8228B288A2970
:10C93600892A8C2B8D2CE4FFE52C152CAC2B700250
:10C94600152B4C6015AB28052AE52AAA2970020585
:10C956002914F91226FB2FFF80DEEF75F0FFA4FFE6
:10C966002212CF4DE490096CF012BDF4900964E0F8
:10C97600FEA3E0FFE48F288E27F526F5257529FF0F
:10C98600752ADA752B0F7D20AF16AE15125168E4A5
:10C99600FFFE02C68E8E288F29EF2401FFE43EFE9D
:10C9A6008D2E7B01E4FD125A6D78AB7C1B7D017EDA
:10C9B600007F031226D5901BABE08529828528834C
:10C9C600F07B017A1B79AB227D09AF16AE1512609A
:10C9D6000B7B017A00790012CDE8EF700F1292827C
:10C9E6007D1CAF16AE1512600B7F002212D2847D1D
:10C9F60012AF16AE1512600B7F0122AFA775A70FF7
:10CA060075F1FE75F30375F4F875A41275A59575A1
:10CA1600A60375AE7875AF0375D4CF75E10175C7FA
:10CA260042E4F5B575B00775A0FC8FA7228F828EFC
:10CA36008312D00D12CEFC12D048AF82AE83E4FC36
:10CA4600FDAB0DAA0CA90BA80AD3122A0540EB12BE
:10CA5600D20112D271E4F50DF50CF50BF50A228D13
:10CA6600228B2312D05BEFFB7A007D0A7FAC12B3D8
:10CA760087AF2212D05BEFFB7A007D097FAC12B341
:10CA860087AF2312D05BEFFB7A007D087FAC02B341
:10CA960087ABA775A70FC28E53C7FD75A7108599DB
:10CAA60032C298C29975A70F75D4CF75D50F43C7F3
:10CAB600028BA7853144853043852F42852E41025E
:10CAC60076D28F228D237F6F12D1177F6B12D117EB
:10CAD600AF2212D117AF2312D117752404C3E52450
:10CAE6009440748094805009E4FF12D11705248085
:10CAF600EC228F228D237F6E12D1177F6F12D117F2
:10CB0600AF2212D117AF2312D117752404C3E5241F
:10CB16009440748094805009E4FF12D11705248054
:10CB2600EC227E007F007DFF7C0312CC37901BAA8F
:10CB3600EFF0600B12BD99901BABE4F0A3EFF07819
:10CB4600A37C097D017B017A0079007E047F0002C7
:10CB560026D59009A374EBF0A37458F0A37490F053
:10CB6600A37445F0A3744CF0A37449F0A37443F086
:10CB7600A3744FF0A3744DF0E4A3F0A37430F02235
:10CB8600C0E0C083C082C0D075D000C00730981303
:10CB9600C298AF5A055A74002FF582E43400F58323
:10CBA600E599F0D007D0D0D082D083D0E0328F2262
:10CBB60012D0FE7F6F12D1177F6B12D117AF2212E0
:10CBC600D117752303C3E5239440748094805009DC
:10CBD600E4FF12D117052380EC228F2212D0FE7FAC
:10CBE6006E12D1177F6F12D117AF2212D11775238C
:10CBF60003C3E5239440748094805009E4FF12D166
:10CC060017052380EC22AFA7E4F5A743BC0175BE48
:10CC16000475BD7C75BE07F5BD75BE0875BD0153AF
:10CC2600BCFE75BB3075BC3875E8C075D1178FA7CB
:10CC3600228E328F337FFFED1DAA0470011C4A60DD
:10CC4600190533E533AA327002053214F5828A8358
:10CC5600E06FFE90DF6693FF80DD22AFA775A70F1A
:10CC66008FA7E4FF12CF90E4FF122006E4FF122004
:10CC760096E4FF12CFA6E4FF12D26B12D22B12D18A
:10CC86003502D1EA7D027F8012A2F5901B9BE0FE61
:10CC9600A3E02400FFE43EFEEF7803CEC313CE13D9
:10CCA600D8F97802C333CE33CED8F9FF22E4901BED
:10CCB600A0F0A3F0901BA0E475F001122849FE74C1
:10CCC600A325F0F58274093EF583E070E790096CC0
:10CCD60004F002D081C29712BC85EF70137F011257
:10CCE600CF9012D1DE12D0FE7BFF7AD979C38009AC
:10CCF60012D0FE7BFF7AD979D31241F822E517606C
:10CD060006E4F5171288BB1262C1EF700C12D2212D
:10CD1600122CEE12D22B127249E51464017005F53D
:10CD26001412CF4D22AEA775A710E4FDFCECC394F8
:10CD360008748094805010ED25E0FD5305FE12CE58
:10CD4600C8EF42050C80E68EA7AF0522AE07E4FDCC
:10CD5600EDC3940874809480500A12CE2BEE25E021
:10CD6600FE0D80EC12CEC88F2FE52F600312CFFB8D
:10CD7600AF2F2212D0FE7BFF7AD979E390096FE0BC
:10CD8600FCA3E0FDA3E0FEA3E0F5398E388D378CD9
:10CD9600361241F8E4FF02D1178F2312928212D283
:10CDA6007B8F118E108D0F8C0E12D284AD23AF1691
:10CDB600AE1512600B124A419009687405F022AF55
:10CDC600A775A70F759F3075A7107592FF7593FE0F
:10CDD6007594FF7595FE4396104391048FA743E71C
:10CDE60080228B238A248925753C04753D007F00AB
:10CDF6007E507D017C0012B62CAE24AF257D007CD2
:10CE06000402CC37E4FFFE12B69AEF700B12D0FE86
:10CE16007BFF7AD679C1800912D0FE7BFF7AD6795C
:10CE2600D71241F822EEC41313135401FFC287EF41
:10CE360024FF9286E5C830E7FB12D035D287E5C8D5
:10CE460030E7FB02D035C0E0C0D053917FE50D241A
:10CE560001F50DE4350CF50CE4350BF50BE4350A5C
:10CE6600F50AD0D0D0E032C0E0C0D0C2CFE5602411
:10CE760001F560E4355FF55FE4355EF55EE4355D4A
:10CE8600F55DD0D0D0E0328F298E288D278C26AF45
:10CE960029AE28AD27AC26AB0DAA0CA90BA80AD340
:10CEA600122A0540EA22EFFD3395E0FCD3ED9439D2
:10CEB600EC648094805006C3EF9430FF22EF24C9BF
:10CEC600FF22D286C287E5C830E7FB12D035D2876B
:10CED600A286E433FFE5C830E7FB02D035C0E0C0E8
:10CEE60083C08253917F75170190096E7401F0D04B
:0ECEF60082D083D0E03243E640225390F322F4
:07CF080043900C5390F72247
:07CF100043900C5390FB223B
:10CF180043900C227B017A007D017FAC12B3877BA2
:10CF2800017A007D027FAC12B38702D144AFA7E437
:10CF3800F5A775CBFE75CA0B85CBCD85CACCD2CAF1
:10CF4800D2AD8FA722E4FBFA7D017FAC12B387E450
:10CF5800FBFA7D027FAC12B38702D28112D153EF64
:10CF68006401700D12D0FE7F0112D1177FEB12D130
:10CF780017227F907E087D007C0012AEC47E007F61
:10CF8800007DFF7C0302CC378F277F327E0012CAD8
:10CF980033E52724FF92B37F647E0002CA338F27CC
:10CFA8007F327E0012CA33E52724FF92B67FF47ED3
:10CFB8000102CA33E4FFFE1226FB600C0FEF70017A
:10CFC8000E09E970F20A80EF22900968E06408709F
:10CFD800087F0112D26B02D08112D0932212D0FEA8
:10CFE800129A1A7BFF7AD9791F1241F8E4FF02D10D
:10CFF80017EFF07F0112CE33E4FF12CE33E4F5C809
:10D00800D286D28722AFA7E4F5A77593F875922F39
:10D018008593958592948FA722901B9BE0FFEFC480
:10D02800540F75F00AA4FEEF540F2EFF22E4F5C842
:10D0380075CBFF75CAE675CDFF75CCE675C80422B9
:10D04800ABA7E4F50DF50CF50BF50AF5A74391042C
:10D058008BA722EF75F00A84C454F0FEEF75F00A2E
:10D0680084E5F04EFF22EFC394094005EF940E408B
:10D0780003BF2003D38001C32212D0FE7F6F12D1D9
:10D08800177F6B12D117E4FF02D11712D0FE7F6E03
:10D0980012D1177F6F12D117E4FF02D117E4FF12E4
:10D0A800200612D0FE7BFF7AD979400241F87F0131
:10D0B80012200612D0FE7BFF7AD979570241F87503
:10D0C8003C04753D007F007E507D017C0002B773F3
:10D0D800AEA775A710C2998F993099FDC2998EA7EE
:10D0E800227BFF7AD679A61241F8E4F5A775EF10EE
:10D0F80022EEF0A3EFF07F0A12D1177F3E02D1177C
:10D1080012389512D0FE7BFF7AD7794F0241F8AEDC
:10D11800A7E4F5A78F993099FDC2998EA722AEA7EB
:10D12800E4F5A78F993099FDC2998EA7227F047ED6
:10D13800007D007C0012BFAF53B5FD22AFA775A7D5
:10D148000F75E4068FA7D296D2A8227D017FAC1274
:10D15800A2F5901B9BE05401FF22EFC394204007E7
:10D16800EF947F50028001C322EFC394304007EF51
:10D17800943A50028001C3229009687401F0E4FFD8
:10D1880012D26B02D0818E618F62E4F55BF55C8C04
:10D19800638D642243B5027F027E007D007C00021D
:10D1A800BFAF12C5FDEF700302D08112D0932212D7
:10D1B800BC27EF700302D08112D09322AD077FAC59
:10D1C80012A2F5901B9BE0FF22AE05AD07EEFB7A9D
:10D1D800007FAC02B387C2A07FC87E0012CA33D2D8
:10D1E800A02285A72775A70F53ABBFC2AC22AFA754
:10D1F80075A70F75A1C78FA722AFA7E4F5A753910D
:10D20800FB8FA7227E1C7F237D3F7C0002D18EC22C
:10D2180086E5C830E7FB02D03543B5017F017E00C3
:10D2280002CA3353B5FE7F017E0002CA33900968F3
:10D238007408F002D0819009687401F002D081EF7F
:10D248006D90DF6693FF2212CA01D2970279657545
:10D25800140112D28132E4F5A753D9BF2212CF4D5F
:10D2680002D081EF24FF92A12253E6BF220298CA7E
:10D2780002D081028EB3D2AF22C2A82202899F3087
:10D28800002E0020003A00202D2041776169746942
:10D298006E6720726567697374726174696F6E2E48
:10D2A8002E2E00202D20526567697374726174698F
:10D2B8006F6E206D6F6465206163746976652E00FA
:10D2C800202D20526567697374726174696F6E20CE
:10D2D8006D6F646520636F6E636C756465642E00A2
:10D2E800202D20526573746F72696E6720726567AE
:10D2F800697374726174696F6E206D6F64652E2E28
:10D308002E00202D204E6F20726573706F6E73652E
:10D318002066726F6D206465766963652E00202D26
:10D328002053686F7274206369726375697420642E
:10D33800657465637465643A2000202D205A65720F
:10D348006F20706F77657220636F6E73756D707480
:10D35800696F6E3A2000202D204572726F7220721C
:10D368006563656976696E672064617461206672B9
:10D378006F6D206465766963652E00202D20494D08
:10D388005041435420657863656564696E6720641D
:10D3980065746563743A2000202D20556E6B6E6F9E
:10D3A800776E206576656E742E00202D20566F6C82
:10D3B8007461676520526567756C61746F7220448B
:10D3C800726F706F75742064657465637465642E1C
:10D3D80000202D20705F61646472657373206F761E
:10D3E8006572666C6F773A2000202D2048525A5F8C
:10D3F80073697A653A2000202D205761726E696E34
:10D40800672C20536D617274207377697463682088
:10D418006F75743A2000202D205761726E696E670F
:10D428002C207468652066757365206973206372A3
:10D438006173682E00202D205761726E696E672C0B
:10D4480020556261742044726F706F757420646532
:10D45800746563743A2000202D205761726E696EDE
:10D46800673A205265672053746172742077697433
:10D47800682054656D702E00202D205254432041A1
:10D488006C61726D207472696767657265642E00DD
:10D49800202D2045565420666F7220415220746F0B
:10D4A8002053657269616C206E756D6265723A20F1
:10D4B80000202D205374617274205265676973745B
:10D4C800726174696F6E2044756520746F20746989
:10D4D8006D65206D617463682E00202D2045727281
:10D4E8006F722077726974696E6720746F20666C3A
:10D4F8006173682073746F726167652E2000202D38
:10D50800205761746368646F672054696D65722081
:10D518005265736574207472696767657265642EF5
:10D5280000202D2053797374656D207375737065B1
:10D538006E6465642064756520746F20706F77650C
:10D5480072206973737565732E00202D20416C61FC
:10D55800726D206E6F74207365742E00202D20412B
:10D5680077616974696E67206D6F646520286E6FD6
:10D57800206261747465727920706F776572290012
:10D58800202D204865616465722048525A207375C1
:10D59800636365737366756C6C7920726561642E5C
:10D5A80000202D20275461736B272066696C652045
:10D5B8006D697373696E6720696E204E414E442E03
:10D5C80000202D20275461736B272066696C652025
:10D5D8006D697373696E6720696E20466C61736844
:10D5E8002E00202D20275461736B272066696C65F7
:10D5F8002067657420696E20466C6173682E002070
:10D608002D20526567206D6F6465206D65737361A9
:10D6180067653A206E6F2042617474657279207074
:10D628006F77657200202D20526567206D6F6465E5
:10D63800206D6573736167653A2054696D6520656F
:10D648006E6400202D205254432072656164206D61
:10D65800616A6F72697479206661756C742E002036
:10D668002D2053657269616C206E756D626572203C
:10D6780026206669726D77617265207665727369B6
:10D688006F6E3A20006C6F61646572007265736535
:10D69800740065726173650077726974650052651C
:10D6A8007365742053797374656D0A0D004E6F7637
:10D6B80020313320323032350046696C6520737969
:10D6C8007374656D20637265617465640A0D004644
:10D6D800696C652073797374656D206E6F7420634F
:10D6E8007265617465640A0D000A0D004572726FF7
:10D6F800722072656164696E67204F6E6669206189
:10D70800727261790A0D0057726974654C6F6769A6
:10D7180063616C50616765204F4B2C2070616765B1
:10D72800203D20256C640057726974654C6F6769E9
:10D7380063616C50616765204E4F2C20706167658E
:10D74800203D20256C64005365744B6174616C6FD7
:10D7580067204F4B0A0D006E6F7420726573706FEF
:10D768006E73696E6720666F7220636F6D6D616E90
:10D7780064204E616E644765745461736B006E6F0C
:10D788007420726573706F6E73696720666F72209C
:10D79800636F6D6D616E6420526561645068797362
:10D7A8006963616C41646472657373006E6F7420A1
:10D7B800526573706F6E73696E6720666F7220634F
:10D7C8006F6D6D616E64204572617365426C6F6345
:10D7D8006B006E6F7420526573706F6E73696E673D
:10D7E80020666F7220636F6D6D616E64205365747F
:10D7F800446174610A0D0046726565204164647273
:10D80800657373203D20256C640A0D006E6F7420CB
:10D81800726573706F6E73696E6720666F722063CE
:10D828006F6D6D616E64204765745461736B0A0D8A
:10D83800006E6F7420726573706F6E73696E672007
:10D84800666F7220636F6D6D616E64205465726DD2
:10D85800696E616C476574506167650A0D004E6FAB
:10D8680074206D6F7665204B6174616C6F670A0D6B
:10D87800004E6F74206765742048727A0A0D004E56
:10D888006F742077726974652070616765006672CD
:10D8980065652061646472657373203D20256C643E
:10D8A8000A0D006E6F74206672656520616464728B
:10D8B8006573730A0D00777269746520256C64209E
:10D8C80061646472657373203D2073756363657367
:10D8D80073007772697465206661696C65640045D8
:10D8E80072726F7250726570617265526573746F8F
:10D8F8007265004572726F72526573706F6E7365F0
:10D90800526573746F72654661743332636F6D6DFF
:10D91800616E64004F4B006F6B007265616420613B
:10D928006464726573733D256C642000726561647C
:10D93800206661696C656400526567697374726119
:10D9480074696F6E20706F776572204F464600527B
:10D958006567697374617274696F6E20706F77653B
:10D9680072204F4E004D6F76654B6174616C6F6726
:10D9780020737563636573730A0D00476574487295
:10D988007A20737563636573730A0D00577269743F
:10D99800652048525A20426F647920737563636525
:10D9A80073730A0D0057726974652048525A2042F1
:10D9B8006F6479206661696C0A0D0053657455734C
:10D9C800624D6F6465204F4B0A0D005365745573A3
:10D9D800624D6F6465204E4F0A0D00256C6400256A
:10D9E8003032642F253032642F25303264202530C0
:10D9F80032643A253032643A253032640A0D0041E7
:10DA0800525F31353000005F322E3900000000309F
:10DA1800372E30322E3235004572726F7250726571
:10DA280070617265526573746F7265006C6F6164C2
:10DA38006572006669726D776172655F76657200FE
:10DA480074657374007263616C007763616C00675E
:10DA5800657474696D6500636C660067616C00636A
:10DA680068617267657265670073657474696D656E
:10DA780000617574680073657461736D0067640094
:10DA880067645F61300067645F61310067645F618C
:10DA9800320067645F6133007365745F706172613F
:10DAA8006D00666173745F636C656172007772699B
:10DAB800746570616765006261636B75705F74613E
:10DAC800736B00636865636B0063686B6F66660001
:10DAD80063686B6F6E00636F6E00636F66660070DD
:10DAE8006F737473796E6300636C65617200436C65
:10DAF8006561720072656164007265616470616776
:10DB0800650063726561746566696C65004372657A
:10DB180061746546696C6500626174746572795FE9
:10DB28006F6B00626174746572795F696E66007705
:10DB3800726974655F706879736963616C5F70613D
:10DB4800676500726561645F706879736963616CA9
:10DB58005F706167650065726173655F626C6F63B2
:10DB68006B00746573745F72657175657374006EAC
:10DB7800616E645F696E6974006E616E645F6F6E7A
:10DB880066695F726561640065726173655F656E81
:10DB9800640057726974654164647265737354658F
:10DBA800737400526561644164647265737354658B
:10DBB800737400706567697374726174696F6E5FFE
:10DBC800706F7765725F646F776E007265676973EF
:10DBD80074726174696F6E5F706F7765725F75706C
:10DBE800006E616E645F6C6F616465720047657496
:10DBF8004E616E64436F6D70696C65566572004E58
:10DC0800616E644765745461736B00526573746F19
:10DC1800726546617433320057726974654C6F6778
:10DC28006963616C5061676500526561644C6F6738
:10DC38006963616C50616765004765744576656E18
:10DC4800745061676500726566617400726566612B
:10DC5800745F7374617475730047657452756E6E82
:10DC6800696E6754696D6500526573657452756EA7
:10DC78006E696E6754696D65004765744F6E6669B5
:10DC88000047657450616765004765745061676552
:10DC980031004765745061676532005365744661A9
:10DCA8007433320052657365740047657454617348
:10DCB8006B005365745461736B005365744B6174E6
:10DCC800616C6F6700536574506F737473796E631A
:10DCD80000476574467265654164647265737300D4
:10DCE8005365745573624D6F646500536574446180
:10DCF80074610047657454696D6500556E6B6E6F8D
:10DD0800776E20636F6D6D616E640A0D00256C641B
:10DD1800002564004F4B00253032642F25303264D3
:10DD28002F2530326420253032643A253032643A67
:10DD380025303264006F6B004154004E616E6449B7
:10DD48006E69740041545F575F315F48414C46002B
:10DD580041545F575F325F48414C460045726173DA
:10DD6800655461736B426F647900476574467265E8
:10DD780065416464726573730052656164506167DC
:10DD880065466F72506879506167650047657448E9
:10DD9800727A426F647900457261736548727A429B
:10DDA8006F6479004D6F76654B6174616C6F6700C5
:10DDB800476574467265654164647265737354653A
:10DDC8007374005265616441646472657373546569
:10DDD800737400577269746541646472657373542F
:10DDE80065737400476574436F6D70696C65446151
:10DDF8007461005F6C6F61646572000016E3600017
:10DE08001E8480536574526573746F7265546173B0
:10DE18006B426F6479005365744576656E74426F22
:10DE2800647900536574526573746F726548525A09
:10DE3800426F647900536574526573746F72654BF1
:10DE48006174616C6F6700526573746F72654661C7
:10DE58007433320057726974655068795061676528
:10DE68000052656164506879506167650045726168
:10DE78007365426C6F636B00526561644F6E6669CF
:10DE880000537461727452656275696C644E616E98
:10DE9800640052656275696C6450726F677265736D
:10DEA80073005465726D696E616C53657444617476
:10DEB800610053657445767400526561645061670A
:10DEC80065005772697465506167650057726974B7
:10DED8006532506167650043726561746546696CB7
:10DEE8006553797374656D0052657365744576651D
:10DEF8006E744C6F6746696C650053657455736240
:10DF08004D6F6465004765745461736B426F647943
:10DF18000047657448727A426F6479576974684437
:10DF2800617465005365745461736B426F64790062
:10DF38005465726D696E616C5365745461736B00DE
:10DF480053657448727A426F64795769746844619A
:10DF580074650053657448727A426F647900005E94
:10DF6800BCE2613FDD83C29C7E20A3FD1F419DC3AF
:10DF7800217FFCA2401E5F01E3BD3E6082DC237D61
:10DF88009FC1421CFEA0E1BF5D0380DE3C62BEE093
:10DF9800025CDF81633D7C22C09E1D43A1FF4618C1
:10DFA800FAA427799BC584DA3866E5BB5907DB856F
:10DFB8006739BAE406581947A5FB7826C49A653B21
:10DFC800D987045AB8E6A7F91B45C6987A24F8A653
:10DFD800441A99C7257B3A6486D85B05E7B98CD281
:10DFE800306EEDB3510F4E10F2AC2F7193CD114F2F
:10DFF800ADF3702ECC92D38D6F31B2EC0E50AFF1E1
:10E00800134DCE90722C6D33D18F0C52B0EE326C12
:10E018008ED0530DEFB1F0AE4C1291CF2D73CA9440
:10E028007628ABF517490856B4EA6937D58B5709EE
:10E03800EBB536688AD495CB2977F4AA4816E9B7A0
:10E04800550B88D6346A2B7597C94A14F6A8742AD2
:10E05800C896154BA9F7B6E80A54D7896B354220FC
:10E068000049006E0066006F000F007272006D00BC
:10E078006100740069006F0000006E000000015329
:10E088000079007300740065000F00726D002000B5
:10E0980056006F006C00750000006D006500535954
:10E0A8005354454D7E3120202016009F13918F55E3
:10E0B8008F55000014918F55030000000000544153
:10E0C800534B2020202020202020000126918F550E
:10E0D8008F5500008A5E8F550A00000400004556DF
:10E0E800454E544C4F4754585420006C5C89525745
:10E0F8005257000070875257060000100000414731
:10E1080047432020202048525A2000B333918F558E
:10E118008F550000A4788F550B0000E06CF76D4117
:10E128002E006D562E007061676500000001000129
:10E1380000010000000000000000000000010000D5
:10E1480000000000000000000000000000010001C5
:10E1580000000000000000000000000000006D4703
:04E16800004F4B0019
:00000001FF
